:020000040800F2
:100000000000022029B90008B1A70008B3A7000822
:10001000B5A70008B7A70008B9A7000800000000AE
:100020000000000000000000000000001186000831
:10003000BBA7000800000000B18600081587000873
:1000400079B9000879B9000879B9000879B90008C8
:10005000BDA7000879B9000879B9000879B9000886
:1000600079B90008C5A70008CFA7000879B900082A
:10007000D9A70008E9A70008F9A7000809A80008FF
:1000800079B9000879B9000879B9000879B9000888
:1000900019A8000829A8000879B9000839A800089B
:1000A00079B9000879B9000879B9000879B9000868
:1000B00079B9000879B9000879B9000879B9000858
:1000C00079B9000845A8000855A8000865A80008E7
:1000D00075A8000885A8000879B9000895A8000847
:1000E00079B9000879B9000879B9000879B9000828
:1000F00079B90008A5A8000879B90008BDA80008CA
:1001000079B9000879B9000879B9000879B9000807
:1001100079B9000879B9000879B9000879B90008F7
:10012000CDA8000879B90008DDA80008EDA80008EE
:10013000FDA8000879B9000879B9000879B9000864
:100140000DA900081DA9000879B900082DA900080B
:100150003DA900084DA900085DA900086DA9000887
:100160007DA900088DA9000879B9000879B90008AF
:1001700079B9000879B9000879B9000800000000D1
:0801800079B9000879B9000803
:1001900010B5054C237833B9044B13B10448AFF3C1
:1001A00000800123237010BD080D00200000000016
:1001B000E8C3010808B5034B1BB103490348AFF37B
:1001C000008008BD000000000C0D0020E8C30108FD
:1001D00081F0004102E000BF83F0004330B54FEAF8
:1001E00041044FEA430594EA050F08BF90EA020F65
:1001F0001FBF54EA000C55EA020C7FEA645C7FEAF8
:10020000655C00F0E2804FEA5454D4EB5555B8BF1A
:100210006D420CDD2C4480EA020281EA030382EA8B
:10022000000083EA010180EA020281EA0303362D1D
:1002300088BF30BD11F0004F4FEA01314FF4801CF0
:100240004CEA113102D0404261EB410113F0004F02
:100250004FEA03334CEA133302D0524263EB4303B9
:1002600094EA050F00F0A780A4F10104D5F1200E57
:100270000DDB02FA0EFC22FA05F2801841F10001B2
:1002800003FA0EF2801843FA05F359410EE0A5F186
:1002900020050EF1200E012A03FA0EFC28BF4CF0B7
:1002A000020C43FA05F3C01851EBE37101F000456D
:1002B00007D54FF0000EDCF1000C7EEB00006EEB7A
:1002C0000101B1F5801F1BD3B1F5001F0CD3490804
:1002D0005FEA30004FEA3C0C04F101044FEA44525B
:1002E00012F5800F80F09A80BCF1004F08BF5FEAE2
:1002F000500C50F1000041EB045141EA050130BDC2
:100300005FEA4C0C404141EB0101013C28BFB1F5D3
:10031000801FE9D291F0000F04BF01460020B1FA1E
:1003200081F308BF2033A3F10B03B3F120020CDAF1
:100330000C3208DD02F1140CC2F10C0201FA0CF0CF
:1003400021FA02F10CE002F11402D8BFC2F1200C34
:1003500001FA02F120FA0CFCDCBF41EA0C019040EA
:10036000E41AA2BF01EB0451294330BD6FEA040433
:100370001F3C1CDA0C340EDC04F11404C4F120021E
:1003800020FA04F001FA02F340EA030021FA04F330
:1003900045EA030130BDC4F10C04C4F1200220FA87
:1003A00002F001FA04F340EA0300294630BD21FAC5
:1003B00004F0294630BD94F0000F83F4801306BF8B
:1003C00081F480110134013D4EE77FEA645C18BF7F
:1003D0007FEA655C29D094EA050F08BF90EA020F16
:1003E00005D054EA000C04BF1946104630BD91EA0E
:1003F000030F1EBF0021002030BD5FEA545C05D111
:100400004000494128BF41F0004130BD14F580044F
:100410003CBF01F5801130BD01F0004545F0FE41C3
:1004200041F470014FF0000030BD7FEA645C1ABFF8
:10043000194610467FEA655C1CBF0B46024650EA2F
:10044000013406BF52EA033591EA030F41F400215B
:1004500030BD00BF90F0000F04BF0021704730B5E1
:100460004FF4806404F132044FF000054FF00001B6
:1004700050E700BF90F0000F04BF0021704730B577
:100480004FF4806404F1320410F0004548BF40424C
:100490004FF000013EE700BF42004FEAE2014FEAA1
:1004A00031014FEA02701FBF12F07F4393F07F4F7C
:1004B00081F06051704732F07F4208BF704793F07F
:1004C0007F4F04BF41F40021704730B54FF4607492
:1004D00001F0004521F000411CE700BF50EA010295
:1004E00008BF704730B54FF000050AE050EA01023E
:1004F00008BF704730B511F0004502D5404261EBAE
:1005000041014FF4806404F132045FEA915C3FF4EE
:10051000D8AE4FF003025FEADC0C18BF03325FEA8B
:10052000DC0C18BF033202EBDC02C2F1200300FA3C
:1005300003FC20FA02F001FA03FE40EA0E0021FA61
:1005400002F11444BDE600BF70B54FF0FF0C4CF44F
:10055000E06C1CEA11541DBF1CEA135594EA0C0F01
:1005600095EA0C0F00F0DEF82C4481EA030621EA3C
:100570004C5123EA4C5350EA013518BF52EA033577
:1005800041F4801143F4801338D0A0FB02CE4FF029
:100590000005E1FB02E506F00042E0FB03E54FF059
:1005A0000006E1FB03569CF0000F18BF4EF0010E51
:1005B000A4F1FF04B6F5007F64F5407404D25FEA4D
:1005C0004E0E6D4146EB060642EAC62141EA555100
:1005D0004FEAC52040EA5E504FEACE2EB4F1FD0C42
:1005E00088BFBCF5E06F1ED8BEF1004F08BF5FEAC0
:1005F000500E50F1000041EB045170BD06F0004672
:1006000046EA010140EA020081EA0301B4EB5C041E
:10061000C2BFD4EB0C0541EA045170BD41F4801116
:100620004FF0000E013C00F3AB8014F1360FDEBF3B
:10063000002001F0004170BDC4F10004203C35DA17
:100640000C341BDC04F11404C4F1200500FA05F39A
:1006500020FA04F001FA05F240EA020001F000423B
:1006600021F0004110EBD37021FA04F642EB0601B1
:100670005EEA430E08BF20EAD37070BDC4F10C04DB
:10068000C4F1200500FA04F320FA05F001FA04F29F
:1006900040EA020001F0004110EBD37041F100018B
:1006A0005EEA430E08BF20EAD37070BDC4F1200596
:1006B00000FA05F24EEA020E20FA04F301FA05F2FE
:1006C00043EA020321FA04F001F0004121FA04F2A6
:1006D00020EA020000EBD3705EEA430E08BF20EA76
:1006E000D37070BD94F0000F0FD101F000464000B0
:1006F00041EB010111F4801F08BF013CF7D041EA32
:10070000060195F0000F18BF704703F00046520035
:1007100043EB030313F4801F08BF013DF7D043EA06
:100720000603704794EA0C0F0CEA135518BF95EABC
:100730000C0F0CD050EA410618BF52EA4306D1D143
:1007400081EA030101F000414FF0000070BD50EA62
:10075000410606BF1046194652EA430619D094EAEC
:100760000C0F02D150EA013613D195EA0C0F05D1D6
:1007700052EA03361CBF104619460AD181EA03012A
:1007800001F0004141F0FE4141F470014FF00000E2
:1007900070BD41F0FE4141F4780170BD70B54FF07D
:1007A000FF0C4CF4E06C1CEA11541DBF1CEA1355FD
:1007B00094EA0C0F95EA0C0F00F0A7F8A4EB0504DF
:1007C00081EA030E52EA03354FEA013100F08880D6
:1007D0004FEA03334FF0805545EA131343EA12639F
:1007E0004FEA022245EA111545EA10654FEA002654
:1007F0000EF000419D4208BF964244F1FD0404F50D
:10080000407402D25B084FEA3202B61A65EB030568
:100810005B084FEA32024FF480104FF4002CB6EB25
:10082000020E75EB030E22BFB61A754640EA0C00A5
:100830005B084FEA3202B6EB020E75EB030E22BFE5
:10084000B61A754640EA5C005B084FEA3202B6EB26
:10085000020E75EB030E22BFB61A754640EA9C00E5
:100860005B084FEA3202B6EB020E75EB030E22BFB5
:10087000B61A754640EADC0055EA060E18D04FEA73
:10088000051545EA16754FEA06164FEAC30343EA13
:1008900052734FEAC2025FEA1C1CC0D111F4801FE0
:1008A0000BD141EA00014FF000004FF0004CB6E7D9
:1008B00011F4801F04BF01430020B4F1FD0C88BF78
:1008C000BCF5E06F3FF6AFAEB5EB030C04BFB6EB83
:1008D000020C5FEA500C50F1000041EB045170BD76
:1008E0000EF0004E4EEA113114EB5C04C2BFD4EBA3
:1008F0000C0541EA045170BD41F480114FF0000E27
:10090000013C90E645EA060E8DE60CEA135594EAA2
:100910000C0F08BF95EA0C0F3FF43BAF94EA0C0FA5
:100920000AD150EA01347FF434AF95EA0C0F7FF41A
:1009300025AF104619462CE795EA0C0F06D152EA6E
:1009400003353FF4FDAE1046194622E750EA410652
:1009500018BF52EA43067FF4C5AE50EA41047FF463
:100960000DAF52EA43057FF4EBAE12E74FF0FF3CC8
:1009700006E000BF4FF0010C02E000BF4FF0010C99
:100980004DF804CD4FEA410C7FEA6C5C4FEA430C12
:1009900018BF7FEA6C5C1BD001B050EA410C0CBF61
:1009A00052EA430C91EA030F02BF90EA020F0020C3
:1009B000704710F1000F91EA030F58BF994208BF2A
:1009C00090422CBFD8176FEAE37040F001007047E7
:1009D0004FEA410C7FEA6C5C02D150EA013C07D13E
:1009E0004FEA430C7FEA6C5CD6D152EA033CD3D089
:1009F0005DF8040B704700BF8446104662468C4683
:100A00001946634600E000BF01B5FFF7B7FF0028B5
:100A100048BF10F1000F01BD4DF808EDFFF7F4FFDE
:100A20000CBF012000205DF808FB00BF4DF808ED69
:100A3000FFF7EAFF34BF012000205DF808FB00BF8C
:100A40004DF808EDFFF7E0FF94BF012000205DF8AE
:100A500008FB00BF4DF808EDFFF7CEFF94BF012063
:100A600000205DF808FB00BF4DF808EDFFF7C4FF5C
:100A700034BF012000205DF808FB00BF4FEA410CA5
:100A80007FEA6C5C02D150EA013C0AD14FEA430C88
:100A90007FEA6C5C02D152EA033C02D14FF00000C5
:100AA00070474FF0010070474FEA410212F5001203
:100AB00015D211D56FF47873B3EB625212D94FEAA5
:100AC000C12343F0004343EA505311F0004F23FA8F
:100AD00002F018BF404270474FF00000704750EAE4
:100AE000013005D111F0004008BF6FF000407047A1
:100AF0004FF00000704700BF4FEA4102B2F1E043FF
:100B000024BFB3F5001CDCF1FE5C0DD901F0004CF4
:100B10004FEAC0024CEA5070B2F1004F40EB830044
:100B200008BF20F00100704711F0804F21D113F170
:100B30003872BCBF01F00040704741F480114FEAA9
:100B40005252C2F11802C2F1200C10FA0CF320FA32
:100B500002F018BF40F001004FEAC1234FEAD3234F
:100B600003FA0CFC40EA0C0023FA02F34FEA4303B9
:100B7000CCE77FEA625307D150EA01331EBF4FF042
:100B8000FE4040F44000704701F0004040F0FE405D
:100B900040F40000704700BF53B94AB9002908BFAC
:100BA00000281CBF4FF0FF314FF0FF3000F06AB952
:100BB000ADF1080C6DE904CE00F006F8DDF804E0B4
:100BC000DDE9022304B070472DE9F047089D0C468B
:100BD000002B4ED194468C458646B2FA82F262D9F9
:100BE0004AB1C2F12003914020FA03F30CFA02FC4F
:100BF000194300FA02FE4FEA1C471FFA8CF6B1FBBC
:100C0000F7F44FEA1E4307FB141143EA014304FBC8
:100C100006F199420AD91CEB030304F1FF3080F07E
:100C20001281994240F20F81023C6344591A1FFA23
:100C30008EF3B1FBF7F007FB101143EA014300FB11
:100C400006F69E420AD91CEB030300F1FF3180F047
:100C5000FC809E4240F2F980634402389B1B40EACC
:100C6000044000211DB1D3400022C5E90032BDE897
:100C7000F0878B4205D90DB1C5E900010021084676
:100C8000F5E7B3FA83F1002946D1A34202D390429B
:100C9000C0F0F080861A64EB03030120002DE6D03B
:100CA000C5E90063E3E7002A40F09080A1EB0C0463
:100CB0004FEA1C481FFA8CF70121B4FBF8F64FEA03
:100CC0001E4308FB164443EA044307FB06F0984220
:100CD00008D91CEB030306F1FF3402D2984200F25C
:100CE000CD8026461C1A1FFA8EF3B4FBF8F008FBE1
:100CF000104443EA044300FB07F79F4208D91CEB6A
:100D0000030300F1FF3402D29F4200F2B08020467C
:100D1000DB1B40EA0640A5E7C1F120068B4022FA22
:100D200006F71F4320FA06FC04FA01F343EA0C031A
:100D3000F44000FA01F8380C4FEA1349B4FBF0FE16
:100D40001FFA87FC00FB1E4449EA04440EFB0CF921
:100D5000A14502FA01F20AD93C190EF1FF3A80F0DE
:100D60008480A14540F28180AEF1020E3C44A4EBA8
:100D700009041FFA83F9B4FBF0F300FB134449EABA
:100D8000044403FB0CFCA44507D93C1903F1FF30D4
:100D900067D2A44565D9023B3C4443EA0E40A0FB20
:100DA0000293A4EB0C049C42CE469C4651D34ED0F9
:100DB00055B1B8EB0E0364EB0C0404FA06F6CB4015
:100DC0001E43CC40C5E90064002150E7C2F1200376
:100DD00020FA03F10CFA02FC24FA03F394400C43CA
:100DE0004FEA1C4800FA02FE1FFA8CF7B3FBF8F03A
:100DF00008FB1031230C43EA014300FB07F1994241
:100E000008D91CEB030300F1FF362CD299422AD9F2
:100E1000023863445B1AA4B2B3FBF8F108FB113348
:100E200044EA034401FB07F3A34208D91CEB040482
:100E300001F1FF3613D2A34211D902396444E41AF6
:100E400041EA004139E70446F0E6084606E7C845AE
:100E5000AED2B9EB020E63EB070C0138A8E73146BE
:100E6000EDE7034699E73046D4E7D6467FE763448B
:100E700002384DE70646234608460FE7023E634424
:100E800030E700BF704700BF10F8012B11F8013B9D
:100E9000012A28BF9A42F7D0D01A7047034613F8A8
:100EA000012B002AFBD1181A0138704700000000FE
:100EB00001F0FF01102A2BDB10F0070F08D010F80B
:100EC000013B013A8B422DD010F0070F42B3F6D10F
:100ED000F0B441EA012141EA014122F007047FF028
:100EE00000070023F0E80256083C85EA010586EA7F
:100EF000010685FA47F5A3FA87F586FA47F6A5FABB
:100F000087F68EB9EED1F0BC01F0FF0102F00702C6
:100F100032B110F8013B013A83EA010313B1F8D171
:100F20000020704701387047002D06BF3546033852
:100F3000073815F0010F07D1013015F4807F02BF8B
:100F4000013015F4C03F0130F0BC0138704700BFDC
:100F500008B50B4B1A6842F400721A601A6842F422
:100F600080621A601A6842F480721A60032000F0EE
:100F7000F5FD0F2009F0CAFB09F09EFB002008BD1B
:100F8000003C0240034A1168034B1B780B4413607A
:100F9000704700BF240D002000000020014B18689E
:100FA000704700BF240D002038B50446FFF7F6FF58
:100FB0000546B4F1FF3F02D0044B1B781C44FFF7F9
:100FC000EDFF401BA042FAD338BD00BF0000002057
:100FD0004A4B5A6822F440325A605A6841680A43C0
:100FE0005A600268536823F4807353600268536840
:100FF000016943EA012353600268536823F0407398
:1010000053600268536881680B43536002689368B9
:1010100023F40063936002689368C1680B43936094
:10102000826A374B9A4257D00268936823F0706304
:10103000936002689368816A0B43936002689368C7
:1010400023F04053936002689368C16A0B43936036
:101050000268936823F00203936002689368017E3C
:1010600043EA4103936090F82030002B3FD00268A0
:10107000536843F4006353600268536823F4604389
:10108000536001684B68426A013A43EA42334B605D
:101090000268D36A23F47003D3620168CB6AC26921
:1010A000013A43EA0253CB620268936823F4007367
:1010B00093600268936890F8301043EA412393608C
:1010C0000268936823F480639360026893684169BF
:1010D00043EA8123936070470268936823F070634A
:1010E00093600268936823F040539360B0E702680E
:1010F000536823F400635360CAE700BF0023014034
:101100000100000F38B310B50446036C43B1236CE3
:1011100013F0100F0BD00120002384F83C3010BDD9
:1011200008F030FC0023636484F83C30EFE7236C64
:1011300023F4885323F0020343F002032364204680
:10114000FFF746FF00206064236C23F0030343F0A5
:1011500001032364E0E701207047000030B482B04F
:101160000022019290F83C20012A00F0B68003464C
:10117000012280F83C200A68092A40D90468E06806
:1011800092B202EB42021E3A4FF0070C0CFA02F246
:1011900020EA0202E2601C68E0680A8802EB420270
:1011A0001E3A8D6805FA02F20243E2604A68062A96
:1011B0003CD81C68606B02EB8202053A4FF01F0CB2
:1011C0000CFA02F220EA020262631C68606B4A6851
:1011D00002EB8202053AB1F800C00CFA02F20243B7
:1011E000626318683E4A904250D018683C4A904268
:1011F00055D0002083F83C0002B030BC7047046832
:10120000206992B202EB42024FF0070C0CFA02F294
:1012100020EA020222611C6820690A8802EB42026D
:101220008D6805FA02F202432261BFE70C2A16D844
:101230001D68286B02EB8202233A1F2404FA02F293
:1012400020EA02022A631D68286B4A6802EB8202C8
:10125000233A0C8804FA02F202432A63C1E71D68AC
:10126000E86A02EB8202413A1F2404FA02F220EA01
:101270000202EA621D68E86A4A6802EB8202413AA9
:101280000C8804FA02F20243EA62AAE70A68122A08
:10129000ABD11448426842F480024260A5E70A6874
:1012A000103A012AA5D80F48426842F40002426071
:1012B0000A68102A9DD10C4A12680C49A1FB02123F
:1012C000920C02EB82025200019202E0019A013A72
:1012D0000192019A002AF9D18BE702208CE700BF26
:1012E00000200140002301409400002083DE1B43C6
:1012F000002800F0A18038B5044690F82030D3B122
:101300002268136843F001031360FFF747FE0546A8
:1013100023685A6812F0010F10D1FFF73FFE401BFF
:101320000A28F5D9636A43F400336362052384F81D
:101330002030012038BD08F0A3FBE1E71A6822F055
:1013400002021A60FFF72AFE054623685A6812F067
:10135000020F0DD0FFF722FE401B0A28F5D9636A61
:1013600043F400336362052384F820300120E1E771
:10137000227E012A3DD01A6822F080021A60637E24
:10138000012B3BD02268136823F040031360A37E37
:10139000012B39D02268136823F020031360E37E09
:1013A000012B37D02268136843F010031360237FAA
:1013B000012B35D02268136823F008031360637F84
:1013C000012B33D02268136823F004031360A36851
:1013D000E268134322691343626913436268013A66
:1013E00021681343CB6100206062012384F8203020
:1013F000A0E71A6842F080021A60C0E7226813680A
:1014000043F040031360C2E72268136843F02003EF
:101410001360C4E72268136823F010031360C6E763
:101420002268136843F008031360C8E72268136852
:1014300043F004031360CAE70120704790F820309E
:10144000013BDBB2012B05D9436A43F4802343629D
:101450000120704730B5464BD3F8002242F001021C
:10146000C3F80022D3F8002222F47C52C3F80022F1
:10147000D3F80022486A42EA0022C3F800224A69EF
:1014800002F01F02012000FA02F2D3F81C026FEAF8
:10149000020C20EA0200C3F81C02CB69C3B9344B2A
:1014A000D3F80C020CEA0000C3F80C028C884869DF
:1014B000CD6844EA0544483043F830408C680888D9
:1014C00040EA04404C6904F1480E03EBCE03586037
:1014D000CB69012B1ED08B69002B33D12448D0F867
:1014E00004320CEA0303C0F804320B698BBB2048BA
:1014F000D0F814320CEA0303C0F814320B6A012B43
:101500002ED01B4AD2F8003223F00103C2F8003279
:10151000002030BD164BD3F80C021043C3F80C0268
:101520008C8848690D6844EA0544483043F83040E7
:1015300088894C698D6840EA0540483403EBC40350
:101540005860C8E70A48D0F804321343C0F80432A0
:10155000CBE70748D0F814321343C0F81432CDE774
:101560000349D1F81C321343C1F81C32C9E700BF4C
:101570000064004070B5044690F82050EDB2012D93
:1015800006D0436A43F4002343620125284670BD18
:10159000022380F820300268136823F001031360EF
:1015A000FFF7FCFC064623685B6813F0010F0CD0C4
:1015B000FFF7F4FC831B0A2BF5D9636A43F400336D
:1015C0006362052384F82030E0E700256562DDE7EB
:1015D00030B590F820C00468A4680CF1FF3C5FFAB5
:1015E0008CFCBCF1010F6BD814F0E05F62D0C4F347
:1015F000016CBCF1020F05D9436A43F40003436256
:10160000012062E0012404FA0CF41C608B68002BBA
:101610003DD10D68CB68046843EA45550CF11803C9
:101620001B01E55003680C690CF1180E03EB0E1357
:101630005C600B7D012B35D0D17993791B0443EA93
:101640000163517943EA012314790168234301EBD3
:101650000C11C1F88C31D17893781B0443EA0163F3
:10166000517843EA0123117802680B4302EB0C1214
:10167000C2F8883102680CF1180C4FEA0C1C52F8C1
:101680000C3043F0010342F80C3000201DE04C68A0
:1016900043EAC403CC6823430CF118042401056811
:1016A0002B51BFE7036803EB0E13596841F48071B7
:1016B0005960C1E7436A43F400134362012004E028
:1016C000436A43F480234362012030BD90F8203008
:1016D000013BDBB2012B01D90020704703689868F9
:1016E00010F0806000D001209A6812F0006F00D0E6
:1016F00001309B6813F0805FEFD00130704790F8A5
:1017000020C00CF1FF3C5FFA8CFCBCF1010F00F231
:10171000958030B451B90468E46814F0030F10D117
:10172000436A43F400134362012077E004682469AC
:1017300014F0030F05D1436A43F400134362012000
:101740006CE001F11B04240105682C5904F0040429
:101750009460002C64D101F11B04240105682C590C
:10176000640D1460046801F11B0C4FEA0C1C54F862
:101770000C4004F00204D46004686444646804F01B
:101780000F041461046864446468C4F3072494611A
:10179000046864446468240C5461026802EB01121A
:1017A000D2F8B8211A70026802EB0112D2F8B821FF
:1017B000C2F307225A70026802EB0112D2F8B82174
:1017C000C2F307429A70026802EB0112D2F8B82104
:1017D000120EDA70026802EB0112D2F8BC211A7103
:1017E000026802EB0112D2F8BC21C2F307225A713F
:1017F000026802EB0112D2F8BC21C2F307429A71CF
:10180000026802EB0112D2F8BC21120EDA7179B92A
:101810000268D36843F02003D360002030BC7047D7
:1018200001F11B04240105682C59E408546099E770
:101830000268136943F020031361EEE7436A43F43F
:10184000802343620120704790F82030013BDBB2D7
:10185000012B01D90020704721B90368D86800F036
:10186000030070470368186900F00300704790F8A0
:101870002030013BDBB2012B05D9436A43F48023BE
:10188000436201207047026853690B435361002093
:101890007047704770477047704770477047704790
:1018A00070477047704770472DE9F84F0546036849
:1018B0005C69D3F804809F68D3F80CB0D3F810A00B
:1018C000D3F8189014F001063BD017F0010616D09B
:1018D00001229A6017F0020F08D117F0040F0CD103
:1018E00017F0080606D04FF4805608E0FFF7D1FF46
:1018F000002604E0FFF7D0FF01E04FF4006617F484
:10190000807F0DD02B684FF480729A6017F4007FAF
:1019100040F0868017F4806F00F0868046F4005611
:1019200017F4803F0DD02B684FF480329A6017F483
:10193000003F40F0838017F4802F00F0838046F44E
:10194000004614F0080F07D01BF0100F04D046F427
:1019500000762B681022DA6014F0040F02D01BF01E
:10196000080F79D114F0020F04D02B68DB6813F054
:10197000030F78D114F0400F07D01AF0100F04D0E5
:1019800046F480662B6810221A6114F0200F02D0F2
:101990001AF0080F6BD114F0100F04D02B681B69DC
:1019A00013F0030F6AD114F4003F02D018F0100FA7
:1019B00068D114F4803F02D018F0080F69D114F4F4
:1019C000004F7AD018F0040F74D014F4807F04D044
:1019D00019F0010F01D046F0010614F4007F04D085
:1019E00019F0020F01D046F0020614F4806F04D003
:1019F00019F0040F01D046F0040614F4006F59D01A
:101A000019F0700956D0B9F1400F65D058D8B9F126
:101A1000200F5ED0B9F1300F42D146F0200644E0ED
:101A20002846FFF737FF7BE717F4006F02D046F434
:101A3000804675E72846FFF730FF71E72846FFF735
:101A40002AFF7EE717F4002F02D046F4803678E7AD
:101A50002846FFF723FF74E72B680822DA60284640
:101A6000FFF71DFF7EE728460BF0E2FB82E72B68BD
:101A700008221A612846FFF713FF8CE728460BF06F
:101A8000DCFB90E72B6810225A602846FFF709FF1D
:101A90008FE72B6808225A602846FFF703FF8EE77E
:101AA000B9F1100F01D146F008062A68936923F0B6
:101AB000700393612B6804225A609EB9BDE8F88FC9
:101AC000B9F1500F0BD0B9F1600FEED146F480762A
:101AD000EBE746F01006E8E746F04006E5E746F09B
:101AE0008006E2E76B6A33436B622846FFF7DBFE52
:101AF000E4E70000002808DB0901C9B200F16040FA
:101B000000F5614080F80013704700F00F000901F4
:101B1000C9B2014B1954704714ED00E000B500F054
:101B20000700C0F1070CBCF1040F28BF4FF0040CF4
:101B3000031D062B0FD9C31E4FF0FF3E0EFA0CF00B
:101B400021EA000199400EFA03FE22EA0E0241EA60
:101B500002005DF804FB0023EEE70000074AD368AB
:101B600023F4E0631B041B0C000200F4E060034359
:101B700043F0BF6343F40033D360704700ED00E0EF
:101B800010B50446054BD868C0F30220FFF7C6FF26
:101B900001462046FFF7AEFF10BD00BF00ED00E09C
:101BA000002807DB00F01F02400901239340024A8E
:101BB00042F82030704700BF00E100E058B110B596
:101BC000044643791BB101236371002010BD0371EA
:101BD00008F006F8F7E70120704770B110B5044629
:101BE000037933B102232371002020610123237183
:101BF00010BD437108F02EF8F4E70120704703464A
:101C000008465979012924D010B54FF0010E83F808
:101C100005E0022119711C68216802F0100240F6EB
:101C2000FE7C0CFA02FC21EA0C0C016840680143BE
:101C3000914041EA0C0121601C682168C02000FA33
:101C400002F221EA0202226083F804E000205871C7
:101C500010BD0220704730B405682C6824F480243D
:101C60002C60046863608368402B05D0036899602A
:101C70000368DA6030BC704703689A600368D96013
:101C8000F8E7000010B40368D9B210390C4AA2FB7F
:101C9000014212090B4CA25CC2655F2909D923F4E9
:101CA0007F7323F0030304338365806D5DF8044B79
:101CB000704723F47F7323F003038365F5E700BFC8
:101CC000ABAAAAAAD8C40108836A826992B9012B77
:101CD0000AD0022B02D00BB100207047C36A13F068
:101CE000807F28D100207047C36AB3F1C07F24D021
:101CF00000207047B2F5005F09D0022B25D9032BD5
:101D000025D1C36A13F0807F23D100207047032BB5
:101D100003D8DFE803F01404140A00207047C36AF4
:101D200013F0807F0DD100207047C36AB3F1C07FEC
:101D300009D0002070470120704701207047012022
:101D40007047012070470120704701207047002034
:101D5000704701207047000070B50446FFF71EF978
:101D6000002C5BD00546022384F83530002384F82C
:101D700034302268136823F00103136023681A6863
:101D800012F0010F0AD0FFF709F9431B052BF5D913
:101D900020236365032084F8350070BD1A6820494C
:101DA00011406268A0680243E06802432069024370
:101DB00060690243A0690243E0690243206A02436A
:101DC0000A43616A04291ED01A602668756925F0E5
:101DD0000705636A1D43042B07D1A36A1D43E36A09
:101DE0001BB12046FFF770FF90B975612046FFF7E1
:101DF00049FFE26D3F23934083600020606501232B
:101E000084F83530C9E7E16A206B01430A43DBE718
:101E100040236365012084F83500BEE70120BCE75C
:101E20003F8010F038B50446856D90F834000128E5
:101E30002BD0012084F8340094F83500C0B201287A
:101E400004D0002384F83430022038BD022084F806
:101E50003500002060652046FFF7FDFEE26D3F2360
:101E60009340AB602268136843F016031360236C41
:101E700023B12268136843F00803136022681368D3
:101E800043F0010313600020DFE70220DDE770B5B7
:101E90000446866DFFF782F894F83530DBB2022BEA
:101EA00006D080236365002384F83430012070BDA0
:101EB00005462268136823F01603136022685369ED
:101EC00023F080035361236CE3B12268136823F08D
:101ED000080313602268136823F00103136023686A
:101EE0001B6813F0010F11D0FFF758F8431B052BA7
:101EF000F5D920236365032084F83500002384F896
:101F00003430D4E7A36C002BDFD1E3E7E26D3F234D
:101F10009340B360012384F83530002084F8340006
:101F2000C5E790F83530DBB2022B03D08023436540
:101F300001207047052380F835300268136823F0CC
:101F40000103136000207047F0B583B004460023FE
:101F50000193724B1D68724BA3FB0535AD0A876D6B
:101F60003E68C26D08239340334210D003681A685C
:101F700012F0040F0BD01A6822F004021A60C26D2E
:101F800008239340BB60436D43F001034365E26D5A
:101F900001239340334209D02268526912F0800F26
:101FA00004D0BB60636D43F002036365E26D0423FC
:101FB0009340334209D02268126812F0020F04D015
:101FC000BB60636D43F004036365E26D10239340CF
:101FD000334224D02268126812F0080F1FD0BB6071
:101FE00023681A6812F4802F0DD01B6813F4002F99
:101FF00004D1236C9BB12046984710E0A36C73B1C9
:10200000204698470BE01A6812F4807F03D11A68C3
:1020100022F008021A60236C0BB120469847E26D4B
:1020200020239340334255D02268126812F0100FDB
:1020300050D0BB6094F83530DBB2052B0ED023684E
:102040001A6812F4802F33D01B6813F4002F2AD1A2
:10205000636C002B3ED0204698473BE02268136813
:1020600023F0160313602268536923F08003536141
:10207000236CA3B12268136823F008031360E26D98
:102080003F239340BB60012384F83530002384F85C
:102090003430236D002B3FD0204698473CE0A36CA2
:1020A000002BE7D1EBE7E36BA3B12046984711E0A3
:1020B0001A6812F4807F09D11A6822F010021A609F
:1020C000012384F83530002384F83430E36B0BB1FE
:1020D00020469847636DFBB1636D13F0010F17D075
:1020E000052384F835302268136823F00103136058
:1020F000019B01330193AB4204D823681B6813F0A2
:10210000010FF5D1012384F83530002384F83430F1
:10211000E36C0BB12046984703B0F0BD940000205B
:10212000B5814E1B90F8350070470000204BDB68EE
:1021300013F0100F07D01F4AD36943F01003D36187
:102140001B4B1022DA601A4BDB6813F0200F07D00C
:10215000184AD36943F00803D361154B2022DA6093
:10216000134BDB6813F0400F07D0124AD36943F0DA
:102170000403D3610E4B4022DA600D4BDB6813F091
:10218000800F07D00B4AD36943F00203D361084B99
:102190008022DA60064BDB6813F0020F07D0054A95
:1021A000D36943F02003D361014B0222DA60704708
:1021B000003C0240280D00207047704710B53A4B94
:1021C000DB6813F0F20F13D0384B1B78DBB2012B16
:1021D0003BD0364B1B78DBB2022B3CD0334B5C69D7
:1021E000FFF7A4FF2046FFF7E8FF304B00221A70EC
:1021F0002D4BDB6813F0010F13D02B4B0122DA605B
:102200002A4B1B78DBB2934228D0284B1B78DBB2D9
:10221000022B41D0254B5869FFF7CEFF234B0022FC
:102220001A70224B1B787BB91F4B1A6922F0FF02F0
:102230001A611A6922F080721A611A6922F000721A
:102240001A611A4B00221A7610BD184BDC684FF049
:10225000FF32DA60C4E7154B1C69C1E7134B5A68BB
:10226000013A5A605B685BB1104CE068FFF7A4FF6D
:10227000E3680133E360E068217A00F019F8D0E701
:102280000A4B4FF0FF34DC6000221A7000F036F881
:102290002046FFF791FFC4E700F030F8034B1869C0
:1022A000FFF78AFFBAE700BF003C0240280D00207C
:1022B00001291BD002291CD009B14FF440710E4BEB
:1022C0001A6922F440721A611A690A431A611A697A
:1022D00022F0F8021A611A6942EAC00040F00200D6
:1022E00018611A6942F480321A6170474FF48071A4
:1022F000E5E74FF40071E2E7003C0240164B1B6833
:1023000013F4007F10D0144B1A6822F400721A6084
:102310001A6842F400621A601A6822F400621A60B5
:102320001A6842F400721A600B4B1B6813F4806F3A
:1023300010D0094B1A6822F480621A601A6842F4BD
:1023400080521A601A6822F480521A601A6842F4A5
:1023500080621A60704700BF003C024000230F2BD0
:1023600000F2E98070B582B065E085684FEA430EFF
:10237000032404FA0EF425EA0405CC6804FA0EF4EA
:102380002C438460446824EA02044A68C2F30012C1
:102390009A40224342605CE0DC08083450F8242074
:1023A00003F00705AD004FF00F0E0EFA05FE22EA0E
:1023B0000E0E0A69AA4042EA0E0240F824205CE0B0
:1023C000072200E0002202FA0EF22A4302345A4D9C
:1023D00045F82420594A94686FEA0C0224EA0C0557
:1023E0004E6816F4801F01D04CEA0405534CA560DA
:1023F000E46802EA04054E6816F4001F01D04CEAB6
:1024000004054E4CE560646802EA04054E6816F463
:10241000003F01D04CEA0405484C65602468224026
:102420004D6815F4803F01D04CEA0402434C226011
:1024300001330F2B7DD801229A400C6804EA020C6C
:1024400032EA0404F4D14C6804F00304013C012C8A
:102450008BD94A6802F00302032A09D0C4685D00E0
:102460000322AA4024EA02048A68AA402243C260E6
:102470004A6802F00302022A8ED004684FEA430E33
:10248000032202FA0EF224EA02044A6802F003026E
:1024900002FA0EF2224302604A6812F4403FC7D0AB
:1024A00000220192264A546C44F480445464526CD5
:1024B00002F480420192019A9C08A51C1E4A52F81F
:1024C000255003F0030E4FEA8E0E0F2202FA0EF291
:1024D00025EA02051B4A90423FF474AF02F5806280
:1024E00090421AD002F58062904218D002F58062C4
:1024F000904216D002F58062904214D002F58062BC
:10250000904212D002F58062904210D002F58062B3
:1025100090423FF455AF082255E7012253E70222CB
:1025200051E703224FE704224DE705224BE706223D
:1025300049E702B070BD704700380140003C0140DF
:1025400000380240000002400AB18161704709046E
:102550008161704708B5054B5B69034200D108BD36
:10256000024B58610AF0B8FFF9E700BF003C014098
:1025700090F83E30DBB2402B10D00369B3F5804FAA
:102580001BD0036D002B39D1436CC3F3C813026811
:1025900003F0060343F0F00313617047036D2BB99A
:1025A000436C026803F0FE0313617047436C0268DA
:1025B00043F00103DBB21361704790F83D30DBB2AA
:1025C000212B0FD0436C026843F00103DBB213618F
:1025D000436B6BB1DB6B5BB10268536843F4006320
:1025E00053607047436C026803F0FE031361EFE72A
:1025F000836B33B1DB6B002BEED102E0036D012B5B
:1026000000D07047436CC3F3C813026803F006039D
:1026100043F0F1031361F4E7436C0268DBB213612A
:10262000436B3BB1DB6B2BB10268536843F400632F
:1026300053607047836B002BFBD0DB6B002BF3D117
:10264000F7E7000010B48BB090F83E30DAB2C16A00
:10265000046B90F83D30DBB2222B0BD000230993A2
:1026600003685A6909929B690993099B0BB05DF84D
:10267000044B7047036D0BB9402A17D0036D1BB98B
:102680000369B3F5404F19D0438D9BB2002B25D180
:10269000029303685A6902929A690292029A1A682E
:1026A00042F400721A6000230365DFE700930368B9
:1026B0005A6900929B690093009BD7E7002301931E
:1026C00003685A6901929A690192019A1A6842F460
:1026D00080721A60036D01330365C7E7438D9BB2B7
:1026E000012B1CD0438D9BB2022B72D00268136861
:1026F00043F48063136003685A6812F4006F00F0BB
:10270000A980202900F2AF80082980F09C8001294F
:1027100040F0A0805A6842F480525A609AE011F565
:10272000803F11D0082934D0202932D0122C2ED04D
:10273000042940D002293ED010293CD002681368F9
:1027400023F4806313603BE00268136823F4806322
:10275000136003685A6812F4006F0CD01A6822F4F0
:1027600080621A600023039303685A6903929B698D
:102770000393039B97E7002204925A6904929A6993
:102780000492049A1A6842F400721A608BE70129D5
:10279000D0D00268136823F480631360002306938B
:1027A00003685A6906929A690692069A1A6842F470
:1027B00000721A6077E70268136843F4806313605D
:1027C0000023059303685A6905929B690593059B4D
:1027D00069E7102904D8264BCB4013F0010F19D11B
:1027E0000268136823F4806313600268136843F47B
:1027F0000063136003685A6812F4006F16D0202932
:102800001DD808290CD2012910D15A6842F48052EF
:102810005A600BE00268136843F480631360E9E7D1
:102820000839144ACA4012F0010FEED10023079371
:1028300003685A6907929B690793079B33E711F571
:10284000803FF3D1E1E708390A4ACA4012F0010F8C
:102850007FF460AF0023089303685A6908929B696C
:102860000893089B1FE711F5803FF3D152E700BFA3
:102870001400010001010001438D9BB25BB1426A6B
:10288000036812781A61436A01334362438D9BB235
:10289000013B9BB243857047438D9BB25BB103689C
:1028A0001A69436A1A70436A01334362438D9BB2CB
:1028B000013B9BB24385704782B0002301930E4BCE
:1028C0001B68DB080D4AA2FB03231B0A03EB8303EF
:1028D0000193019B013B0193019B33B103681B688A
:1028E00013F4007FF5D1002004E0036C43F02003D3
:1028F0000364012002B070479400002089B5F814E9
:10290000C36AB3F52A0F04D0C36AB3F12A4F03D0C8
:1029100070470123C36270470823C362F8E70000D1
:10292000002800F0CC8070B5044690F83D30002BB4
:1029300077D0242384F83D302268136823F0010304
:1029400013602268136843F400431360226813681D
:1029500023F40043136002F04BF862685A4B9A422A
:1029600064D85A4B98428CBF00230123002B40F0BF
:10297000A8805749A1FB00318B0C25686A6822F0BA
:102980003F0242EA91426A6021680A6A22F03F02ED
:1029900066684D4DAE424FD8013313430B62216838
:1029A000CA6922F44F4222F0FF026568464B9D42FD
:1029B0004CD8431E6D00B3FBF5F3013340F6FC70B9
:1029C000034278D0C3F30B031A43CA6121680B6832
:1029D00023F0C003E269206A024313430B602168BD
:1029E0008B6823F4034323F0FF032269E06802436A
:1029F00013438B602168CB6823F0FF036269A069F1
:102A000002431343CB602268136843F00103136051
:102A100000202064202384F83D30206384F83E00A9
:102A200070BD80F83C3007F001FB82E7294B9842EB
:102A30008CBF0023012399E74FF4967505FB03F340
:102A4000254DA5FB03539B090133A6E7A668BEB934
:102A5000431E05EB450CB3FBFCF30133C3F30B033F
:102A6000B3FA83F35B0943BBC6B9431E05EB4505C7
:102A7000B3FBF5F30133C3F30B0343F40043A3E7C4
:102A8000431E05EB850C0CEB8C0CB3FBFCF3013304
:102A9000C3F30B03B3FA83F35B09E4E7431E05EBCF
:102AA000850505EB8505B3FBF5F30133C3F30B0394
:102AB00043F4404388E7042386E7012384E70120A9
:102AC00070470120ACE700BFA08601007F841E0094
:102AD00083DE1B43FF083D00D34D621070477047F3
:102AE00008B590F83D30DAB2438D9BB283B1416AAC
:102AF000036809781961436A01334362438D9BB2CD
:102B0000013B9BB24385438D9BB20BB9292A00D070
:102B100008BD0268536823F4806353602123036374
:102B2000282380F83D30FFF7DAFFF1E7704708B55A
:102B300090F83D30DAB2438D9BB283B103681969D6
:102B4000436A1970436A01334362438D9BB2013B70
:102B50009BB24385438D9BB20BB92A2A00D008BD96
:102B60000268536823F4806353602223036328239D
:102B700080F83D30FFF7DAFFF1E7704700B583B02A
:102B800090F83D3003F02803282B0CD0002301934C
:102B900002685169019192690192019A80F83C3072
:102BA00003B05DF804FB0268536823F4806353604C
:102BB00011F0040F0BD0002311F0800F09D182898E
:102BC000002180F83C101946FFF7D7FFE8E7012302
:102BD000F2E7028BF4E7704708B590F83D30DBB2BE
:102BE000C26A082A01D0202A01D1282B06D0212B25
:102BF0001ED003686FF480625A6108BD1A4BC3622D
:102C00000268536823F4E063536003686FF48062E2
:102C10005A610268136823F480631360002303631E
:102C2000202280F83D2080F83E30FFF7D4FFE4E713
:102C30000D4BC36221230363202380F83D30002322
:102C400080F83E300268536823F4E0635360036801
:102C50006FF480625A610268136823F48063136022
:102C6000FFF73DFFC9E700BF0000FFFF704708B551
:102C7000C26A90F83D30DBB2212B00D008BD438DF5
:102C80009BB263B1426A036812781A61436A0133E6
:102C90004362438D9BB2013B9BB24385EEE7082A1A
:102CA00004D0202A02D012F5803F19D1026853685F
:102CB00023F4E06353600268136843F40073136005
:102CC00000230363202380F83D3090F83E30DBB2D0
:102CD000402B15D0002380F83E30FFF7FFFECDE7F4
:102CE0000268536823F4E0635360112303630023F5
:102CF00080F83E30202380F83D30FFF7EFFEBDE73F
:102D0000002380F83E30FFF7B1FFB7E708B590F831
:102D10003D30026D9AB9C36C012B08D0836CC3F3AC
:102D2000072302681361036D0133036508BD836CDB
:102D30000268DBB21361036D02330365F6E7DBB2B1
:102D4000026D012A23D0026D022AEFD1222B26D058
:102D5000428D92B20AB1212B2AD0428D92B2002A22
:102D6000E4D1212BE2D10268536823F4E06353607D
:102D70000268136843F40073136000230363202286
:102D800080F83D2080F83E30FFF770FFCEE7836C7F
:102D90000268DBB21361036D01330365C6E70268A5
:102DA000136843F480731360036D01330365BDE75B
:102DB000426A036812781A61436A01334362438DA1
:102DC0009BB2013B9BB24385B0E710B590F83D3014
:102DD000DBB290F83E20D2B2C46A018D00293BD10B
:102DE000212B02D0402A42D010BD082C04D0202C28
:102DF00002D014F5803F19D10268536823F4E063D0
:102E000053600268136843F4007313600023036384
:102E1000202380F83D3090F83E30DBB2402B15D0B7
:102E2000002380F83E30FFF759FEDDE70268536863
:102E300023F4E063536011230363002380F83E30E2
:102E4000202380F83D30FFF749FECDE7002380F8CE
:102E50003E30FFF70BFFC7E7212BC3D1438D9BB259
:102E600043B90268536823F480635360BCE7222BA4
:102E7000BAD1F3E790F83E30DBB2402B0CD0426A77
:102E8000036812781A61436A01334362438D9BB22F
:102E9000013B9BB24385A7E7FFF738FFA4E708B5DE
:102EA000C26A438D9BB2042B14D0438D9BB2032B7B
:102EB00022D0438D9BB2022B39D003681A69436A32
:102EC0001A70436A01334362438D9BB2013B9BB24C
:102ED000438510E00268536823F4806353600368FD
:102EE0001A69436A1A70436A01334362438D9BB285
:102EF000013B9BB2438508BD01684B6823F48063A6
:102F00004B60042A06D0022A04D00268136823F416
:102F10008063136003681A69436A1A70436A013355
:102F20004362438D9BB2013B9BB24385E3E7013A89
:102F30000F2A40D8DFE802F008393F393F3F3F3FD2
:102F40003F3F3F3F3F3F3F080268136823F48063E1
:102F5000136003681A69436A1A70426A531C436219
:102F6000438D9BB2013B9BB2438503681B69537041
:102F7000436A01334362438D9BB2013B9BB243855D
:102F80000268536823F440735360202380F83D3077
:102F900090F83E30DBB2402B13D0002380F83E3057
:102FA000122303630AF0B0FAA5E70268136843F43A
:102FB00080631360CDE70268136843F40073136005
:102FC000C7E7002380F83E3003630AF0C7FA92E7B0
:102FD000704790F83D30DBB2222B00D0704710B51F
:102FE0000446438D9BB2032B15D903681A69436AC3
:102FF0001A70436A01334362438D9BB2013B9BB21B
:103000004385438D9BB2032B0FD10268536823F491
:103010008063536009E0C26A022A01D0012B05D9FE
:103020002268536823F48063536010BDFFF744FCAB
:1030300000282ED12268136823F48063136022686D
:10304000536823F4E063536023681A69636A1A7053
:10305000636A01336362638D9BB2013B9BB26385FC
:10306000202384F83D3094F83E30DBB2402B08D06A
:10307000002384F83E301223236320460AF044FAEA
:10308000D3E7002384F83E30236320460AF066FA33
:10309000CBE72268536823F4E063536023681A691E
:1030A000636A1A70636A01336362638D9BB2013B8A
:1030B0009BB26385202384F83D30002384F83E30A2
:1030C0002046FFF785FFB0E77047000000B583B0EA
:1030D00000230193806B90F83D20D2B2324B1B68E5
:1030E000DB083249A1FB03131B0A03EB8303C3EB89
:1030F000C3030193019B43B1019B013B019303680F
:103100001B6813F4007FF5D103E0036C43F0200348
:103110000364436B0BB10021D963836B0BB10021B6
:10312000D96301680B6823F480630B600023438537
:10313000436B0BB100211965836B0BB1002119653D
:1031400001680B6823F001030B6090F83D30DBB29F
:10315000602B0ED002F02802282A14D0202380F8F9
:103160003D30002380F83E30FFF732FF03B05DF8BA
:1031700004FB202380F83D30002380F83E300364B8
:10318000FFF7A2FFF2E70268136843F00103136040
:103190000268136843F480631360002303632823E9
:1031A00080F83D30E0E700BF9400002089B5F814B6
:1031B00010B5044690F83D30DBB290F83E20D2B214
:1031C000102A36D0402A34D003F02802282A38D0DA
:1031D0002268526812F4006F07D1602B05D02023BB
:1031E00084F83D30002384F83E30002323632368B5
:1031F0005A6812F4006F48D05A6822F400625A608C
:10320000626B92F83530DBB2012B20D0444B136552
:10321000606BFEF786FE002849D02268136823F011
:1032200001031360202384F83D30606B036D9847E1
:103230003DE0222BC8D121680A6822F400620A60AE
:10324000C2E700232363282384F83D30CFE7A36B34
:10325000334A1A65A06BFEF764FE40B323685A69CF
:1032600012F0400F05D01A69636A1A70636A01335D
:1032700063622268136823F001031360202384F83B
:103280003D30A06B036D984711E094F83D20D2B219
:10329000602A1FD05A6912F0400F05D01A69636A7C
:1032A0001A70636A013363622046FFF791FE236C54
:1032B00013F00F0F04D02268536823F4E0635360C7
:1032C00094F83D30DBB2226C12F0040F01D0282BB1
:1032D00018D010BD202284F83D20002222645A69B3
:1032E00012F0400F05D01A69636A1A70636A0133DD
:1032F00063622268136823F0010313602046FFF71E
:10330000E3FED4E7074BE36200232363202284F823
:103310003D2084F83E302046FFF75DFCD9E700BF32
:10332000CD3000080000FFFF30B583B0044690F8B0
:103330003D50EDB20268536823F4E063536000230C
:10334000019303685A6901921A6842F001021A60F7
:10335000019B0268136823F48063136003685A6852
:1033600012F4006F38D0222D21D02A2D1FD0426BAD
:103370001268526892B24285428D92B21AB1026CC2
:1033800042F0040202645A6822F400625A60606BE0
:10339000FEF7C8FE01281FD0636B444A1A65606BB4
:1033A000FEF7BFFDC0B1606B036D984714E0A26BE0
:1033B0001268526892B26285628D92B21AB1226C22
:1033C00042F0040222645A6822F400625A60A06B40
:1033D000FEF7A8FE012842D1638D9BB233B3236868
:1033E0005A6912F0040F0AD01A69636A1A70636A84
:1033F00001336362638D9BB2013B9BB2638523689B
:103400005A6912F0400F0AD01A69636A1A70636A27
:1034100001336362638D9BB2013B9BB26385638D15
:103420009BB21BB1236C43F004032364236C13BBD6
:103430002A2D25D094F83D30DBB2282B29D0236BE0
:10344000222B01D0222D19D100232363202284F8BE
:103450003D2084F83E302046FFF768FB0EE0A36B6A
:10346000124A1A65A06BFEF75CFD0028B4D0A06B71
:10347000036D9847B0E72046FFF79AFE03B030BDD2
:1034800000232363282384F83D302046FFF74EFBBA
:10349000D0E7074BE36200232363202284F83D201A
:1034A00084F83E302046FFF796FBE7E7CD30000872
:1034B0000000FFFFF8B5044602685568C66A90F838
:1034C0003E30DBB290F83D10C8B2102B13D0402B29
:1034D00011D0236C002B7AD05369002113F0020F16
:1034E00078D015F4007F75D0236C03B19169204624
:1034F000FFF744FBF8BDD2F818C0516911F001077D
:1035000005D1B6F52A0FF5D0B6F12A4FF2D017B192
:1035100015F4007F29D111F0080F02D015F4007FB7
:103520002AD111F0020F02D015F4007F28D11CF02F
:10353000040F31D0526812F4006FDBD111F0800F0C
:1035400005D015F4806F02D011F0040F1CD011F0DB
:10355000040FCFD015F4007FCCD0212818D0402BF9
:10356000C8D12046FFF7D2FBC4E72046FFF7C8F9D1
:103570002046FEF7FDFFBDE72046FFF74DF8B9E70F
:103580002046FFF75FF8B5E72046FFF71EFCB1E7DE
:103590002046FFF76CFBADE7536813F4006FA9D129
:1035A00011F0400F05D015F4806F02D011F0040F18
:1035B00009D011F0040F9DD015F4007F9AD0204659
:1035C000FFF76DFC96E72046FFF703FD92E7916950
:1035D000536983E713F0100F02D015F4007F18D160
:1035E00021281AD0292818D013F0400F05D015F43F
:1035F000806F02D013F0040F28D013F0040F3FF4B3
:1036000079AF15F4007F3FF475AF2046FFF744F91A
:1036100070E72046FFF788FE6CE713F0800F05D0B7
:1036200015F4806F02D013F0040F0BD013F0040FC9
:103630003FF460AF15F4007F3FF45CAF2046FFF726
:103640001BF957E72046FFF74BFA53E72046FFF7F1
:103650006EFA4FE7F8B5044603685D695F6890F855
:103660003E20D2B215F4807606D017F4807603D0CF
:103670006FF480715961012615F4007F08D017F4AA
:10368000807F05D046F0020623686FF4007159610F
:1036900015F4806F19D017F4807F16D0638D99B21E
:1036A00094F83D30DBB2206B202A1BD023686FF4E6
:1036B0008061596146F00406102A01D0402A04D1E5
:1036C0002268136843F40073136015F4006F17D079
:1036D00017F4807F14D046F0080623686FF4006268
:1036E0005A610EE00029E1D1212B05D0292B03D00E
:1036F000282BDBD12128D9D12046FFF76DFAE4E74A
:103700002EB1236C334323642046FFF751FDF8BDEF
:103710002DE9F04383B0D0F8008001EBC10300EB4A
:103720008303DA6D5B6D9A4254D807460C469B1AA8
:1037300001EBC10200EB8202926C9A4200D31A465E
:1037400002F103094FEA990915E006F103094FEA6E
:10375000990904EBC40507EB8505E96C3B7C0093F4
:10376000B3B2E2B2404603F0B2FBEB6C3344EB641D
:10377000EB6D3344EB6508EB441303F510639B6971
:103780009BB24B4512D304EBC40307EB8303DA6D02
:103790005B6D9A420AD24BB19B1A04EBC40207EB51
:1037A0008202966C9E42D0D31E46CEE704EBC40341
:1037B00007EB83077A6DFB6D9A420FD804F00F0474
:1037C0000122A240D8F8343823EA0203C8F834387A
:1037D000002000E0012003B0BDE8F0830020FAE7FC
:1037E00070B58AB0002800F090800546046890F813
:1037F000BD343BB3032385F8BD34E36B13F4807F02
:1038000001D100232B61286803F07EF82C4654F880
:10381000106BEC460FCCACE80F000FCCACE80F00FF
:1038200094E803008CE803002B1D0ECB304602F019
:10383000ADFF044658B1022385F8BD34012420466B
:103840000AB070BD80F8BC3407F07CFED2E70021DE
:10385000286803F04AFD234616E003EBC30205EB9C
:103860008202012182F83D1082F83C30A2F84430F7
:10387000002182F840109164D16403EBC30205EB90
:10388000820251650133DBB269688B42E5D316E0F1
:1038900004EBC40305EB8303002283F87D2283F845
:1038A0007C4283F88022C3F88822C3F88C2204EB80
:1038B000C40305EB8303C3F894220134E4B2A142AC
:1038C000E6D82C4654F8106BEC460FCCACE80F0051
:1038D0000FCCACE80F0094E803008CE803002B1D2C
:1038E0000ECB304603F06CF8044620B1022385F875
:1038F000BD340124A3E7002385F83830012385F87F
:10390000BD34286803F0B0FC99E7012497E702680A
:1039100090F8BC34012B19D010B50446012380F86F
:10392000BC34836A012B09D0206802F0E7FF2068CD
:1039300003F08CFC002084F8BC0410BD8369012BCB
:10394000F2D0936B43F480339363EDE7022070472A
:1039500070B504460D460068066C00EB411303F594
:1039600030639A682169012911D038498E4256D0B6
:103970003DB905EBC50304EB8303D3F89432002B68
:103980005ED0E9B2204607F027FE002070BD12F09D
:10399000080F09D02E498E42F7D912F4004FF4D007
:1039A0004FF400429A60F0E712F0200F02D020227C
:1039B0009A60EAE712F0280FE7D125498E4206D92E
:1039C00012F4004F03D04FF400429A60DDE705EB9C
:1039D000C50204EB8202D2F898121B69C3F31203EA
:1039E000CB1AC2F89C327DB905EBC50204EB82020A
:1039F000D2F894226AB105EBC50204EB8202D2F838
:103A00008C121944C2F88C12E9B2204607F0E4FD8A
:103A1000BBE704F2C442012103F0A8FCF4E712F46E
:103A2000004F03D04FF400429A60AEE712F0200F2F
:103A300001D020229A60E9B2204607F0CDFDA4E72C
:103A400004F2C442002103F091FC9AE70A31544F7A
:103A50000A30544F38B5044603681D6C03EB41131C
:103A6000D3F8081B0E4A954207D903F5306311F4C9
:103A7000004F02D04FF400429A60204607F0A4FDA8
:103A8000074B9D4202D92369012B01D0002038BD8C
:103A900004F2C4420121206803F068FCF6E700BF8D
:103AA0000A30544F90F8BC34012B0DD010B50446A9
:103AB000012380F8BC3480F83810006803F0B6FBAE
:103AC000002084F8BC0410BD0220704738B50546BC
:103AD0008C4611F0800F29D101F00F0E0EEBCE04B1
:103AE000A40004F51E740444211D0EEBCE0E00EB61
:103AF0008E0E00208EF87D020CF00F0C81F800C0B5
:103B0000CA600B714A780AB1A1F808C0022B1DD017
:103B100095F8BC34012B1CD0012385F8BC342868EF
:103B200003F027F8002085F8BC0438BD01F00F0031
:103B300000EBC001890038312944043100EBC0009A
:103B400005EB8000012480F83D40D5E700234B7150
:103B5000DEE70220E9E710B504460A4611F0800FBF
:103B600020D101F00F0000EBC0039B0003F51E7392
:103B70002344191D00EBC00004EB8000002380F8F3
:103B80007D3202F00F020A7094F8BC34012B19D078
:103B9000012384F8BC34206803F038F8002084F84E
:103BA000BC0410BD01F00F0000EBC0039B003833D4
:103BB0002344191D00EBC00004EB8000012380F8B2
:103BC0003D30DEE70220ECE710B501F00F0404EB16
:103BD000C401890001F51E710144043104EBC40CD9
:103BE00000EB8C0CCCF88C22CCF894320023CCF86F
:103BF0009C328CF87D328CF87C420369012B06D014
:103C000064B9DAB2006803F071F8002010BD04EB6B
:103C1000C40C00EB8C0CCCF89022F1E7DAB200680F
:103C200003F06CF9F1E701F00F0101EBC10100EBCA
:103C30008100D0F89C02704710B501F00F0404EB2E
:103C4000C401890038310144043104EBC40C00EB99
:103C50008C0CCCF84C20CCF854300023CCF85C30E1
:103C600001238CF83D308CF83C400369012B06D0D1
:103C700064B9DAB2006803F039F8002010BD04EB33
:103C8000C40C00EB8C0CCCF85020F1E7DAB20068E1
:103C900003F034F9F1E738B501F00F0542689542B9
:103CA00039D804460B4611F0800F1FD101EBC1013A
:103CB000890001F51E710144043103EBC30300EBDD
:103CC0008303002283F87D2201238B700D7094F80A
:103CD000BC34012B21D0012384F8BC34206803F0CC
:103CE0004AFA8DB1002084F8BC0438BD05EBC5014B
:103CF000890038310144043105EBC50300EB83032F
:103D0000012283F83D20DFE704F2C442217C2068D1
:103D100003F02CFBE6E70120E7E70220E5E701F0EE
:103D20000F034268934231D810B5044611F0800F5A
:103D30001ED103EBC301890001F51E71014404315A
:103D400003EBC30200EB8202002082F87D02002216
:103D50008A700B7094F8BC34012B19D0012384F8BD
:103D6000BC34206803F034FA002084F8BC0410BD91
:103D700003EBC301890038310144043103EBC30272
:103D800000EB8202012082F83D00E0E7012070474D
:103D90000220ECE708B511F0800F0CD101F00F0103
:103DA00001EBC101890001F51E7101440431006875
:103DB00003F02EF808BD01F00F0101EBC1018900ED
:103DC000383101440431F2E72DE9F04F83B0044665
:103DD0000568284603F085FA10B103B0BDE8F08FFE
:103DE0000646206803F04EFA0028F6D005F5006775
:103DF000BB68C3F30D23C4F8FC34206803F042FA17
:103E000010F0020F04D02268536903F002035361DB
:103E1000206803F037FA10F0100F13D0226893696E
:103E200023F010039361D5F8208008F00F09C8F340
:103E30004343022B4BD0062B6FD02268936943F08B
:103E400010039361206803F01DFA10F4002F76D15F
:103E5000206803F017FA10F4802F40F0E08020680B
:103E600003F010FA0028C0F26381206803F00AFA18
:103E700010F4006F09D0BB6813F0010F40F070819F
:103E80002268536903F400635361206803F0FAF970
:103E900010F4805F40F06881206803F0F3F910F4BB
:103EA000005F40F0B581206803F0ECF910F0080FD6
:103EB00040F0C681206803F0E5F910F0800F00F0B3
:103EC000D981AB6923F08003AB610126C2E147F6DB
:103ED000F07318EA030FB0D04FEA181A4FEAC9037B
:103EE000019309EBC90B04EB8B0BC8F30A12DBF847
:103EF0008C12284603F01CF9DBF88C32CAF30A0A4C
:103F00005344CBF88C32DBF89C32019A4A4404EBE0
:103F100082025344C2F89C328FE7082204F2C44163
:103F2000284603F005F909EBC90304EB8303D3F832
:103F30009C22C8F30A184244C3F89C227DE72068FB
:103F400003F0A4F98046B14635E005EB49130122A0
:103F5000C3F8082B49462046FFF7FAFC3CE005EB86
:103F600049130822C3F8082B49462046FFF772FD83
:103F700035E009EBC90304EB830393F87F32012B8F
:103F800041D005EB49130222C3F8082B1AF0200F89
:103F900004D005EB49132022C3F8082B1AF4005F64
:103FA00005D005EB49134FF40052C3F8082B09F173
:103FB00001094FEA5808B8F1000F3FF449AF18F073
:103FC000010FF4D05FFA89FB5946206803F06EF9BF
:103FD000824610F0010FB8D11AF0080FBFD11AF0C5
:103FE000100F04D005EB49131022C3F8082B1AF068
:103FF000020FCBD06B6913F0800FBAD07B6843F40B
:1040000080637B60B5E709EBC90304EB83030022FF
:1040100083F87F225946204607F030FBB1E720683D
:1040200003F03CF98046B14625E05946204607F0AA
:10403000DFFA1AF0080F04D005EB49130822C3F881
:1040400008291AF0100F04D005EB49131022C3F809
:1040500008291AF0400F04D005EB49134022C3F899
:1040600008291AF0020F40D11AF0800F5BD109F134
:1040700001094FEA5808B8F1000F3FF4F0AE18F00C
:10408000010FF4D05FFA89FB5946206803F017F955
:10409000824610F0010FCCD009F00F02012101FA85
:1040A00002F27B6B23EA02037B6305EB4913C3F83F
:1040B000081923698B42B8D109EBC90304EB8303C8
:1040C000DA6C996C0A44DA64B9F1000FADD109EBEE
:1040D000C90304EB83035B6D002BA6D104F2C44239
:1040E0000121206803F042F99FE74946284602F083
:1040F00011FC09EBC90304EB830393F83F30012B58
:1041000005D005EB49130222C3F80829ACE709EBF7
:10411000C90304EB8303002283F83F20594620465D
:1041200007F0B2FAEDE749462046FFF7F1FA9EE7BD
:104130007B6823F001037B6094F8F434012B08D0F2
:10414000204607F095FA2268536903F00043536153
:104150008BE6002184F8F414204600F041F9F2E7E0
:10416000204607F06DFA8BE67B6823F001037B6045
:104170001021206802F0CEFB1AE005EB46134FF643
:104180007F31C3F80819D3F8002922F40012C3F8CC
:104190000029C3F8081BD3F8002B22F40012C3F83F
:1041A000002BD3F8002B42F00062C3F8002B01363D
:1041B0006368B342E1D8FB6943F00113FB61236BF1
:1041C000DBB1D7F8843043F00B03C7F884307B6C45
:1041D00043F00B037B64D5F8003823F4FE63C5F885
:1041E000003804F2C442217C206803F0BFF8226842
:1041F000536903F4805353614EE67B6943F40053E3
:1042000043F02B037B613B6943F00B033B61E2E727
:10421000206803F09BF8206802F09AFCE0602668B2
:1042200000F0E0FB0146227B304602F0F5FA204622
:1042300007F0EFF92268536903F40053536132E643
:10424000204607F0E0F92268536903F00803536140
:1042500030E601366368B3420CD906EBC60304EBC3
:10426000830393F87F32012BF3D1F1B22046FFF79D
:1042700091FDEEE7206803F005F810F4801F27D1C8
:10428000206802F0FFFF10F4001F5BD0012328E03C
:1042900001366368B3421DD905EB4613D3F80029F4
:1042A00006EBC60304EB830393F84030012BEFD1F8
:1042B000002AEDDA06EBC60304EB8303012283F840
:1042C0003F2066F07F01C9B22046FFF763FDDFE7BC
:1042D0000126DEE72268536903F480135361CFE7B8
:1042E000013362689A4228D905EB4312D2F8001BC9
:1042F00003EBC30204EB820292F88022012AEFD181
:104300000029EDDA01F48031D4F8FC2402F0010236
:104310009142E5D103EBC30204EB8202012182F852
:104320007F12AA6942F08002AA616A6912F0800FC6
:10433000D6D17B6843F400737B602268536903F431
:1043400000135361206802F09DFF10F0804F10D1E0
:10435000206802F097FF10F0040F3FF43EAD236891
:104360005D6815F0040F0DD1226853682B4353602C
:1043700033E5204607F08EF92268536903F0804345
:104380005361E5E7204607F08BF9EDE710B40468C8
:10439000606A31B940EA0240A06200205DF8044B37
:1043A00070478C46A36A00EB1340002308E003F13A
:1043B000400104EB8101496800EB11400133DBB29D
:1043C0000CF1FF318B42F2D340EA02400CF13F0185
:1043D00004EB81046060E0E70368596200207047E5
:1043E00070470000002800F0E08170B582B00446FC
:1043F000036813F0010F3BD09F4B9B6803F00C0345
:10440000042B2CD09C4B9B6803F00C03082B21D071
:104410006368B3F5803F4FD0B3F5A02F52D0964BD1
:104420001A6822F480321A601A6822F480221A6014
:104430006368002B50D0FCF7B1FD05468E4B1B681E
:1044400013F4003F14D1FCF7A9FD401B6428F5D9F3
:104450000320B1E1884B5B6813F4800FD8D0864B02
:104460001B6813F4003F03D06368002B00F09F81AA
:10447000236813F0020F54D07F4B9B6813F00C0F8E
:104480003ED07D4B9B6803F00C03082B33D0E368D0
:10449000002B68D0794B01221A60FCF77FFD05469E
:1044A000754B1B6813F0020F54D1FCF777FD401BCE
:1044B0000228F5D903207FE16F4A136843F4803363
:1044C0001360B5E76C4B1A6842F480221A601A68D0
:1044D00042F480321A60ABE7FCF760FD0546664B9C
:1044E0001B6813F4003FC3D0FCF758FD401B642841
:1044F000F5D9032060E1604B5B6813F4800FC6D1EF
:104500005D4B1B6813F0020F03D0E368012B40F0F2
:104510005081594A136823F0F803216943EAC10323
:104520001360236813F0080F42D063696BB3534BD9
:104530000122C3F8802EFCF731FD05464E4B5B6F20
:1045400013F0020F34D1FCF729FD401B0228F5D9E6
:10455000032031E1484A136823F0F803216943EA54
:10456000C1031360DDE7454B00221A60FCF716FD1E
:104570000546414B1B6813F0020FD2D0FCF70EFD2D
:10458000401B0228F5D9032016E13C4B0022C3F85A
:10459000802EFCF703FD0546374B5B6F13F0020FCF
:1045A00006D0FCF7FBFC401B0228F5D9032003E1F1
:1045B000236813F0040F77D02F4B1B6C13F0805F30
:1045C00033D1002301932C4B1A6C42F080521A64B1
:1045D0001B6C03F080530193019B0125284B1B6842
:1045E00013F4807F23D0A368012B34D0052B38D05F
:1045F000214B1A6F22F001021A671A6F22F004028F
:104600001A67A368002B3DD0FCF7C8FC06461A4B7E
:104610001B6F13F0020F46D1FCF7C0FC801B41F268
:1046200088339842F3D90320C6E00025D6E7144A20
:10463000136843F480731360FCF7B0FC0646104B1C
:104640001B6813F4807FCED1FCF7A8FC801B0228E6
:10465000F5D90320B0E0084A136F43F00103136754
:10466000CFE7054B1A6F42F004021A671A6F42F047
:1046700001021A67C5E700BF003802400000474248
:1046800000700040FCF78AFC0646524B1B6F13F08B
:10469000020F08D0FCF782FC801B41F2883398425D
:1046A000F3D9032088E0EDB9A369002B00F08380E3
:1046B000484A926802F00C02082A51D0022B17D007
:1046C000454B00221A66FCF769FC0446414B1B6807
:1046D00013F0007F42D0FCF761FC001B0228F5D9E3
:1046E000032069E03B4A136C23F080531364DBE73B
:1046F000394B00221A66FCF751FC0546354B1B6806
:1047000013F0007F06D0FCF749FC401B0228F5D9C6
:10471000032051E0E369226A1343626A43EA821389
:10472000A26A5208013A43EA0243E26A43EA026398
:10473000284A5360284B01221A66FCF72FFC0446D6
:10474000244B1B6813F0007F06D1FCF727FC001BED
:104750000228F5D903202FE000202DE000202BE0D7
:10476000012B2BD01B4B5B6803F48001E269914263
:1047700026D103F03F02216A8A4223D1616A47F6BB
:10478000C0721A40B2EB811F1ED103F44031A26AFD
:104790005208013AB1EB024F18D103F07063E26A9C
:1047A000B3EB026F14D1002006E001207047012016
:1047B00002E0012000E0002002B070BD0120FBE714
:1047C0000120F9E70120F7E70120F5E70120F3E7F1
:1047D0000120F1E7003802400000474208B5264BAF
:1047E0009B6803F00C03042B41D0082B41D1224BD2
:1047F0005A6802F03F025B6813F4800F12D01E4B20
:104800005968C1F388111D480023A1FB0001FCF782
:10481000C3F9194B5B68C3F3014301335B00B0FB81
:10482000F3F027E0144B5868C0F388104FEA401C9F
:10483000BCEB000C6EEB0E0E4FEA8E1343EA9C634A
:104840004FEA8C11B1EB0C0163EB0E03DB0043EA82
:104850005173C90011EB000C43F1000399020023CE
:104860004FEA8C2041EA9C51FCF796F9D1E70348C6
:1048700000E0034808BD00BF00380240001BB7003D
:104880000024F400002800F09B8070B50D4604461B
:104890004F4B1B6803F007038B4208D2CBB24C4A44
:1048A0001370136803F007038B4240F08B8023687A
:1048B00013F0020F17D013F0040F04D0454A936889
:1048C00043F4E0539360236813F0080F04D0414A87
:1048D000936843F4604393603E4A936823F0F00387
:1048E000A1680B439360236813F0010F32D0636813
:1048F000012B21D09A1E012A25D9364A126812F0BE
:10490000020F61D033498A6822F0030213438B609F
:10491000FCF744FB06462F4B9B6803F00C036268D0
:10492000B3EB820F16D0FCF739FB801B41F28833C2
:104930009842F0D9032042E0264A126812F4003F60
:10494000E0D101203BE0234A126812F0007FD9D168
:10495000012034E01E4B1B6803F00703AB4207D96C
:10496000EAB21B4B1A701B6803F00703AB422DD150
:10497000236813F0040F06D0164A936823F4E0531B
:10498000E1680B439360236813F0080F07D0114AC6
:10499000936823F46043216943EAC1039360FFF7FE
:1049A0001DFF0C4B9B68C3F303130B4AD35CD84029
:1049B0000A4B18600A4B186805F0A8FE002070BD6D
:1049C000012070470120FAE70120F8E70120F6E70F
:1049D000003C02400038024074C5010894000020E9
:1049E00004000020014B1868704700BF94000020AD
:1049F00008B5FFF7F7FF044B9B68C3F38223034A14
:104A0000D35CD84008BD00BF003802406CC5010827
:104A100008B5FFF7E7FF044B9B68C3F34233034A33
:104A2000D35CD84008BD00BF003802406CC5010807
:104A30000F2303600B4B9A6802F0030242609A68EE
:104A400002F0F00282609A6802F4E052C2609B6851
:104A5000DB0803F4E0530361034B1B6803F0070317
:104A60000B60704700380240003C024030B583B014
:104A70000446036813F0050F06D1236813F0020FF4
:104A80002ED1002003B030BD4A4B00229A66FCF7BD
:104A900085FA0546484B1B6813F0006F06D0FCF7FB
:104AA0007DFA431B022BF5D90320EBE76268A3686C
:104AB0001B0743EA8213404AC2F884303D4B01226F
:104AC0009A66FCF76BFA05463B4B1B6813F0006FC8
:104AD000D3D1FCF763FA431B022BF5D90320D1E7AE
:104AE00000230193344B1A6C42F080521A641B6C01
:104AF00003F080530193019B304A136843F48073A1
:104B00001360FCF74BFA05462C4B1B6813F4807FAF
:104B100006D1FCF743FA431B022BF5D90320B1E77A
:104B2000254B1B6F13F4407314D0E26802F44072FB
:104B30009A420FD0204B1A6F22F440721D49012077
:104B4000C1F8400E0020C1F8400E1A671B6F13F029
:104B5000010F13D1E36803F44072B2F5407F1ED019
:104B6000154A936823F4F813936013490B6FE268B6
:104B7000C2F30B0213430B67002083E7FCF70EFA26
:104B800005460D4B1B6F13F0020FE3D1FCF706FA3D
:104B9000401B41F288339842F3D9032072E706495B
:104BA0008A6822F4F81223F0704323F4407313430D
:104BB0008B60DAE700004742003802400070004096
:104BC00098B110B5044643795BB102236371226842
:104BD000136843F004031360012363710020A06095
:104BE00010BD037105F0B6FBEFE70120704738B543
:104BF00004460268D36823F0A003D360FCF7CEF923
:104C000005462368DB6813F0200F07D1FCF7C6F9CF
:104C1000401BB0F57A7FF4D9032000E0002038BDB6
:104C200070B50368DA6812F0400F02D000252846FC
:104C300070BD0446DA6842F08002DA60FCF7AEF933
:104C4000064600252368DB6813F0400FEFD1002DE6
:104C5000EDD1FCF7A3F9831BB3F57A7FF2D90423D6
:104C600063770125EEE70268D36823F08003D36001
:104C700003689B6813F0200F01D00020704710B527
:104C80000446FFF7B4FF10B104236377012010BD81
:104C9000002842D010B50446437F7BB102236377DE
:104CA0002368CA225A62236853225A622046FFF7B9
:104CB000B7FF38B12368FF225A6210BD037705F0B1
:104CC0007BFBEBE72268936823F4E00323F04003C7
:104CD000936021688A6863682069034360690343BD
:104CE00013438B602368E2681A6122681369A16824
:104CF00043EA014313612046FFF7B5FF0028D9D1ED
:104D00002268136C23F4802313642268136CA16956
:104D10000B43136401236377CCE701207047000045
:104D20002DE9F04782B00546884617461E46FCF737
:104D300035F90A9B1B1A03EB0609FCF72FF982468B
:104D4000284B1B68C3F3CB3309FB03F301932B6898
:104D50009C6838EA04040CBF01230023BB423DD009
:104D6000B6F1FF3FF3D0FCF719F9A0EB0A00484574
:104D700007D2019A02B14A46019B013B0193914639
:104D8000E5E72A68536823F0E00353606B68B3F5E6
:104D9000827F0BD0AB6AB3F5005F14D0012385F896
:104DA0005130002385F85030032018E0AB68B3F58C
:104DB000004F02D0B3F5806FECD12A68136823F05E
:104DC00040031360E6E72A68136823F40053136076
:104DD0002A68136843F400531360DFE7002002B031
:104DE000BDE8F0879400002010B584B00446164B4F
:104DF0001868164BA3FB0030400D4FF47A7303FB89
:104E000000F003906368B3F5827F0BD0039BBBB1C6
:104E1000039B013B039323689B6813F0800FF5D13C
:104E200000200EE000920B46002280212046FFF772
:104E300077FF30B1636D43F020036365032000E02A
:104E4000002004B010BD00BF94000020819F5E16BA
:104E500000285AD010B50446436A33B94368B3F505
:104E6000827F05D00023C36102E000230361436118
:104E70000023A36294F85130002B40D0022384F821
:104E800051302268136823F040031360636803F411
:104E90008273A26802F404421343E26802F40062DF
:104EA0001343226902F002021343626902F0010215
:104EB0001343A26902F400721343E26902F038025C
:104EC0001343226A02F080021343A26A02F40052E2
:104ED000216813430B60638B03F00403626A02F0E2
:104EE0001002216813434B602268D36923F40063E6
:104EF000D36100206065012384F8513010BD84F82F
:104F00005030204605F0C4FAB8E7012070472DE97B
:104F1000F04383B01F460A9D90F85030012B00F0FB
:104F20001081044688469146012380F85030FCF7F2
:104F300035F8064694F85130DBB26268012B0AD08E
:104F4000B2F5827F40F0E380A268002A40F0E98059
:104F5000042B40F0E880B8F1000F00F0E680B9F1D2
:104F6000000F00F0E480002F00F0E38094F851304F
:104F7000DBB2042B02D0052384F851300023636593
:104F8000C4F83890E787A787C4F83080E786A786FB
:104F90002364636423681A6812F0400F03D11A680F
:104FA00042F040021A60E368B3F5006F11D0636805
:104FB0000BB1012F0BD1226B236812781A73236B6C
:104FC00001332363E38E9BB2013B9BB2E38601274F
:104FD0006BE063680BB1012F0BD1226B2368128841
:104FE000DA60236B02332363E38E9BB2013B9BB2F7
:104FF000E38601271CE023689A6812F0010F0ED0A7
:10500000E28F92B25AB1DA68A36B1A80A36B0233B3
:10501000A363E38F9BB2013B9BB2E3870127FBF7BE
:10502000BDFF801BA84203D3B5F1FF3F40F0838052
:10503000E38E9BB21BB9E38F9BB2002B53D0236846
:105040009A6812F0020FD6D0E28E92B2002AD2D025
:10505000002FD0D0226B1288DA60236B02332363D7
:10506000E38E9BB2013B9BB2E3860027C3E7236834
:105070009A6812F0010F0ED0E28F92B25AB1DA683C
:10508000A36B1A70A36B0133A363E38F9BB2013B45
:105090009BB2E3870127FBF781FF831BAB4202D35F
:1050A000B5F1FF3F49D1002D49D0E38E9BB213B932
:1050B000E38F9BB2BBB123689A6812F0020FD6D07F
:1050C000E28E92B2002AD2D0002FD0D0226B12787A
:1050D0001A73236B01332363E38E9BB2013B9BB2B4
:1050E000E3860027C3E7324629462046FFF77CFEC9
:1050F00048B9A36863B901932368DA6801929B6891
:105100000193019B04E020236365012000E002205D
:10511000012384F85130002384F8503003B0BDE8F7
:10512000F0830220F4E70220F2E70120F0E70120FB
:10513000EEE70120ECE70320EAE70320E8E703209D
:10514000E6E70220EAE7704710B584B0044602683B
:105150005168936803F04100012867D013F0020FF3
:1051600002D011F0800F68D113F4B07F68D011F035
:10517000200F65D013F0400F0FD094F85100C0B24B
:1051800003285FD0606D40F004006065002000904F
:10519000D068009090680090009813F0200F0CD019
:1051A000606D40F001006065002002909068029000
:1051B000106820F040001060029A13F4807F09D03C
:1051C000636D43F0080363650023039323689B68C2
:1051D0000393039B636D002B32D02268536823F046
:1051E000E0035360012384F8513011F0030F31D0F4
:1051F0002268536823F003035360E36C4BB1174AF2
:105200001A65E06CFCF78DFE18B1636D43F0400346
:105210006365A36CA3B1114A1A65A06CFCF781FE0B
:1052200070B1636D43F04003636509E011F0400F16
:1052300094D0236C2046984702E0636C2046984740
:1052400004B010BD00230193D368019393680193C8
:10525000019BF5E72046FFF776FFF1E76152000872
:1052600008B5806B0023C387C386FFF76CFF08BDBA
:1052700030B4036A23F001030362036A426884695D
:1052800024F0730C0C6844EA0C0423F0020C8B68C5
:1052900043EA0C03114DA84203D005F58065A842EE
:1052A00005D123F00803CD682B4323F004030B4DF5
:1052B000A84203D005F58065A84207D122F44072C8
:1052C0004D6945EA020C8A6942EA0C024260846137
:1052D0004A684263036230BC704700BF000001406F
:1052E00030B4036A23F480730362036A4268C469BA
:1052F00024F0730C0C6844EA0C0523F400738C68EA
:1053000043EA0423114CA04203D004F58064A04278
:1053100006D123F40063CC6843EA042323F48063BA
:105320000A4CA04203D004F58064A04207D122F4C5
:1053300040524C6942EA04128C6942EA041242600B
:10534000C5614A68C263036230BC70470000014017
:1053500030B4036A23F480530362036A4468C26969
:1053600022F4E6420D6842EA052223F400538D68D8
:1053700043EA0533094DA84203D005F58065A842EC
:1053800004D124F480444D6944EA85144460C26128
:105390004A680264036230BC704700BF00000140ED
:1053A00010B4036A046A24F001040462846924F0DE
:1053B000F00C4CEA021223F00A030B4382610362F1
:1053C0005DF8044B704710B4036A23F010030362C6
:1053D0008469036A24F4704C4CEA023223F0A0037F
:1053E00043EA0113826103625DF8044B70478368EE
:1053F00023F070030B4343F0070383607047000002
:1054000090F83D30DBB2012B37D1022380F83D30DC
:105410000268D36843F00103D3600368194A9342DA
:1054200020D0B3F1804F1DD0A2F57C42934219D019
:1054300002F58062934215D002F58062934211D04A
:1054400002F5784293420DD002F57052934209D092
:10545000A2F59432934205D01A6842F001021A6014
:10546000002070479A6802F00702062A07D01A68DF
:1054700042F001021A6000207047012070470020AE
:10548000704700BF00000140704770477047704789
:10549000704710B5044603681A6912F0020F11D064
:1054A000DA6812F0020F0DD06FF002021A610123C8
:1054B000037703689B6913F0030F70D0FFF7E7FFD2
:1054C0000023237723681A6912F0040F12D0DA68D8
:1054D00012F0040F0ED06FF004021A61022323773A
:1054E00023689B6913F4407F5FD02046FFF7CFFF0E
:1054F0000023237723681A6912F0080F12D0DA68A4
:1055000012F0080F0ED06FF008021A6104232377FF
:105510002368DB6913F0030F4ED02046FFF7B7FF77
:105520000023237723681A6912F0100F12D0DA686B
:1055300012F0100F0ED06FF010021A6108232377BB
:105540002368DB6913F4407F3DD02046FFF79FFFBF
:105550000023237723681A6912F0010F03D0DA6859
:1055600012F0010F36D123681A6912F0800F03D0B0
:10557000DA6812F0800F34D123681A6912F0400FF4
:1055800003D0DA6812F0400F32D123681A6912F0A2
:10559000200F03D0DA6812F0200F30D110BDFFF7D2
:1055A00075FF204608F01CF88AE72046FFF76EFFDB
:1055B000204608F015F89BE72046FFF767FF2046D6
:1055C00008F00EF8ACE72046FFF760FF204608F031
:1055D00007F8BDE76FF001021A61204604F000FEF3
:1055E000C1E76FF080021A61204600F059FBC3E763
:1055F0006FF040021A612046FFF74AFFC5E76FF0DF
:1056000020021A61204600F04AFBC7E70368304ACF
:10561000904212D0B0F1804F0FD0A2F57C42904260
:105620000BD002F58062904207D002F58062904272
:1056300003D002F57842904203D123F070034A6808
:105640001343234A90422AD0B0F1804F27D0A2F5CD
:105650007C42904223D002F5806290421FD002F536
:10566000806290421BD002F57842904217D002F53A
:105670007052904213D002F5806290420FD002F532
:10568000806290420BD0A2F59832904207D002F58A
:105690008062904203D002F58062904203D123F4ED
:1056A0004073CA68134323F080034A6913430360BD
:1056B0008B68C3620B688362054B984203D003F585
:1056C0008063984201D10B690363012343617047F2
:1056D0000000014040B310B5044690F83D30F3B1EE
:1056E000022384F83D30214651F8040BFFF78EFF6A
:1056F000012384F8463084F83E3084F83F3084F843
:10570000403084F8413084F8423084F8433084F8E3
:10571000443084F8453084F83D30002010BD80F8D6
:105720003C3005F0A3F9DBE70120704740B310B52A
:10573000044690F83D30F3B1022384F83D30214611
:1057400051F8040BFFF762FF012384F8463084F818
:105750003E3084F83F3084F8403084F8413084F89B
:10576000423084F8433084F8443084F8453084F87B
:105770003D30002010BD80F83C30FFF785FEDBE7B0
:105780000120704740B310B5044690F83D30F3B1A6
:10579000022384F83D30214651F8040BFFF736FF11
:1057A000012384F8463084F83E3084F83F3084F892
:1057B000403084F8413084F8423084F8433084F833
:1057C000443084F8453084F83D30002010BD80F826
:1057D0003C30FFF75AFEDBE70120704730B4036A24
:1057E00023F010030362036A4468826922F4E642EC
:1057F0000D6842EA052223F020038D6843EA051371
:10580000114DA84203D005F58065A84206D123F0CA
:105810008003CD6843EA051323F040030A4DA842F4
:1058200003D005F58065A84207D124F440644D6992
:1058300044EA85048D6944EA8504446082614A68CB
:105840008263036230BC70470000014090F83C3036
:10585000012B28D010B50446012380F83C300C2AD7
:105860001CD8DFE802F0071B1B1B0C1B1B1B111BAA
:105870001B1B16000068FFF7FBFC00200FE0006810
:10588000FFF7ACFF00200AE00068FFF729FD0020C9
:1058900005E00068FFF75CFD002000E00120002328
:1058A00084F83C3010BD0220704738B590F83C3089
:1058B000012B66D004460D46012380F83C300C2AAB
:1058C0005AD8DFE802F0075959591B59595930592C
:1058D000595944000068FFF7CBFC2268936943F0F4
:1058E000080393612268936923F00403936122689B
:1058F000936929690B43936100203EE00068FFF73C
:105900006DFF2268936943F4006393612268936991
:1059100023F48063936122689369296943EA012330
:105920009361002029E00068FFF7DAFC2268D36960
:1059300043F00803D3612268D36923F00403D361E1
:105940002268D36929690B43D361002015E0006800
:10595000FFF7FEFC2268D36943F40063D361226839
:10596000D36923F48063D3612268D369296943EA48
:105970000123D361002000E00120002384F83C30A3
:1059800038BD0220FCE710B4846824F47F4C42EA5E
:1059900003220A4342EA0C0282605DF8044B70471E
:1059A00090F83C30012B78D010B50446012380F8E4
:1059B0003C30022380F83D300268936823F47F4333
:1059C00023F0770393600B68602B4CD029D8402BD1
:1059D00054D00CD9502B22D1CA6849680068FFF70F
:1059E000DFFC50212068FFF702FD002005E0202B9E
:1059F0000DD009D9302B0AD00120012384F83D3085
:105A0000002384F83C3010BD0BB1102B05D1194692
:105A10002068FFF7ECFC0020EFE70120EDE7012014
:105A2000EBE7B3F5805F34D0B3F5005F0CD1CB6802
:105A30004A6889680068FFF7A6FF2268936843F404
:105A4000804393600020D8E7702B24D1CB684A684C
:105A500089680068FFF797FF2268936843F077032F
:105A600093600020C9E7CA6849680068FFF7ABFC8B
:105A700060212068FFF7BBFC0020BEE7CA684968C8
:105A80000068FFF78DFC40212068FFF7B0FC002084
:105A9000B3E70020B1E70120AFE70220704701F033
:105AA0001F014FF0010C0CFA01FC036A23EA0C03FE
:105AB0000362036A8A4013430362704710B50446C9
:105AC0000846002942D194F83E30DBB2013B18BFB2
:105AD0000123002B6ED1002851D1022384F83E30DF
:105AE000012201462068FFF7DAFF2368334A934218
:105AF00003D002F58062934203D15A6C42F4004213
:105B00005A6423682D4A934249D0B3F1804F46D05E
:105B1000A2F57C42934242D002F5806293423ED08D
:105B200002F5806293423AD002F57842934236D031
:105B300002F57052934232D0A2F5943293422ED0A5
:105B40001A6842F001021A60002032E0042908D0ED
:105B500008290DD094F84130DBB2013B18BF012376
:105B6000B7E794F83F30DBB2013B18BF0123B0E741
:105B700094F84030DBB2013B18BF0123A9E70428A9
:105B800005D0082807D0022384F84130A8E7022373
:105B900084F83F30A4E7022384F84030A0E79A68F5
:105BA00002F00702062A07D01A6842F001021A60C2
:105BB000002010BD0120FCE70020FAE700000140B2
:105BC00090F83C20012A3DD010B40346012280F811
:105BD0003C20022280F83D2002685068946820F042
:105BE000700C086840EA0C0050601A68164882423F
:105BF0001AD0B2F1804F17D0A0F57C40824213D06A
:105C000000F5806082420FD000F5806082420BD0A8
:105C100000F57840824207D000F57050824203D0F0
:105C2000A0F59430824204D124F0800449682143D5
:105C30009160012283F83D20002083F83C005DF84C
:105C4000044B70470220704700000140024690F864
:105C50003C30012B21D0012380F83C30CB6823F469
:105C600040738868034323F480634868034323F444
:105C700000630868034323F480530869034323F453
:105C800000534869034323F48043C9690B431168F7
:105C90004B64002082F83C00704702207047704738
:105CA0007047026802F10C0353E8003F23F0C00381
:105CB0000C3242E800310029F3D1202380F83D3036
:105CC0007047026802F10C0353E8003F23F490731D
:105CD0000C3242E800310029F3D1026802F11403CA
:105CE00053E8003F23F00103143242E80031002959
:105CF000F3D1036B012B05D0202380F83E30002325
:105D000003637047026802F10C0353E8003F23F07D
:105D100010030C3242E800310029F3D1ECE790F88F
:105D20003D30DBB2212B01D0022070478368B3F5F0
:105D3000805F17D0036A5A1C02621A7803685A609F
:105D4000C38C9BB2013B9BB2C3844BB90268D3683E
:105D500023F08003D3600268D36843F04003D3602C
:105D6000002070470369002BE4D1036A1B88026896
:105D7000C3F308035360036A02330362E0E70000E1
:105D800010B504460268136923F44053C1680B43FD
:105D90001361836802691A4343691A43C3691A434A
:105DA0000168CB6823F4164323F00C031343CB6044
:105DB0000268536923F4407381690B43536103689C
:105DC000314A934206D002F58062934202D0FEF738
:105DD0000FFE01E0FEF71CFEE369B3F5004F29D08A
:105DE0000021031849411B1841F10001C90041EA93
:105DF0005371DB00181863684FEA83024FEA93730C
:105E000041F10001FAF7C8FE204AA2FB003149091E
:105E1000642303FB11031B013233A2FB03235B0941
:105E200003F0F00202EB011203F00F0321681344A8
:105E30008B6010BD0023021843EB0301121841F1DF
:105E40000001C90041EA5271D200101841F100016D
:105E5000626892185B41FAF79FFE0C4AA2FB003180
:105E60004909642303FB1103DB003233A2FB032344
:105E70005B095A0002F4F87202EB011203F0070307
:105E8000216813448B60D4E7001001401F85EB515B
:105E90002DE9F84305460F4616469946DDF8208061
:105EA0002B681C6837EA04040CBF01240024B442A8
:105EB0002DD1B8F1FF3FF3D0B8F1000F05D0FBF7BB
:105EC0006DF8A0EB09004045EAD92A6802F10C03FD
:105ED00053E8003F23F4D0730C3242E8003100292C
:105EE000F3D12A6802F1140353E8003F23F00103C1
:105EF000143242E800310029F3D1202385F83D30E7
:105F000085F83E30002385F83C30032000E0002077
:105F1000BDE8F88358B310B5044690F83D300BB394
:105F2000242384F83D302268D36823F40053D360DF
:105F30002046FFF725FF2268136923F4904313617D
:105F40002268536923F02A0353612268D36843F41B
:105F50000053D36000202064202384F83D3084F86F
:105F60003E3010BD80F83C3005F014F9D8E7012030
:105F700070472DE9F04182B01E4690F83D30DBB20B
:105F8000202B54D104460D469046002953D0002AB8
:105F900053D090F83C30012B51D0012380F83C3095
:105FA00000230364212380F83D30FAF7F7FF07460A
:105FB000A4F82480A4F82680A368B3F5805F05D0F8
:105FC0004FF00008002384F83C3012E0236913B13D
:105FD0004FF00008F6E7A8460025F3E738F8023B43
:105FE0002268C3F308035360E28C92B2013A92B282
:105FF000E284E38C9BB273B100963B460022802181
:106000002046FFF745FFE0B9002DE7D015F8012B3A
:1060100023685A60E8E700963B460022402120466C
:10602000FFF736FF78B9202384F83D3000E00220E6
:1060300002B0BDE8F0810120FAE70120F8E7022074
:10604000F6E70320F4E70320F2E790F83D30DBB2F7
:10605000202B19D1D1B1DAB190F83C30012B19D0F5
:10606000012380F83C3001628284C28400230364EF
:10607000212280F83D2080F83C300168CA6842F057
:106080008002CA601846704702207047012070479E
:10609000012070470220704738B5134690F83D2024
:1060A000D2B2202A37D10446002936D0002B36D070
:1060B00090F83C20012A34D0012280F83C20016273
:1060C0008384C38400250564212280F83D20426B2F
:1060D0001548D063626B15481064626B1448D06435
:1060E000626B156522680432606BFBF79BFE2368C8
:1060F0006FF040021A6084F83C50226802F11403E9
:1061000053E8003F43F08003143242E80031002995
:10611000F3D1002000E0022038BD0120FCE701207F
:10612000FAE70220F8E700BF376100089F61000826
:10613000AD610008704708B50346806B1B681B689B
:1061400013F4807F1AD10023C384026802F1140380
:1061500053E8003F23F08003143242E80031002965
:10616000F3D1026802F10C0353E8003F43F040030F
:106170000C3242E800310029F3D108BDFFF7DAFF05
:10618000FBE708B50168CA6822F04002CA60202215
:1061900080F83D20FFF7CEFF002008BD704708B50E
:1061A000806BFFF7FBFF08BD7047704710B5846B2D
:1061B00023685A6994F83D30DBB2212B10D0236854
:1061C0005A6902F0400294F83E30DBB2222B11D023
:1061D000236C43F010032364204607F071FB10BDCD
:1061E00002F08002002AEAD00023E3842046FFF771
:1061F00058FDE4E7002AEBD00023E3852046FFF7B3
:1062000060FDE5E708B5806B0023C385C38407F014
:1062100057FB08BD90F83E30DBB2222B67D1836874
:10622000B3F5805F4DD0826AB3F5805F04D0002B58
:1062300054D10369002B51D103685B681370836AE2
:1062400001338362C38D9BB2013B9BB2C385002B9C
:106250004FD100B583B00268D36823F02003D36028
:106260000268D36823F48073D3600268536923F013
:1062700001035361202380F83E30036B012B33D19F
:1062800000230363026802F10C0353E8003F23F08C
:1062900010030C3242E800310029F3D103681A6878
:1062A00012F0100F06D0002201921A6801925B686A
:1062B0000193019B818D07F0CDFA002003B05DF8BA
:1062C00004FB0269002AAED1826A03685B68C3F3EB
:1062D00008031380836A02338362B3E703685B6851
:1062E00003F07F031370AAE7FFF75EFFE5E70220E4
:1062F000704700207047000010B582B00446026865
:106300001368D068516913F00F0F09D113F0200FF3
:106310000CD010F0200F09D02046FFF77BFF16E0CD
:1063200011F0010115D110F4907F12D1216B0129D8
:1063300079D013F0800F03D010F0800F40F010815F
:1063400013F0400F03D010F0400F40F00D8102B069
:1063500010BD13F0010F06D010F4807F03D0226C23
:1063600042F00102226413F0040F04D019B1226C30
:1063700042F00202226413F0020F04D019B1226C21
:1063800042F00402226413F0080F07D010F0200F2F
:1063900000D119B1226C42F008022264226C002A5A
:1063A000D5D013F0200F02D010F0200F29D1236890
:1063B0005B6903F04003226C12F0080F00D163B355
:1063C0002046FFF77EFC23685B6913F0400F20D066
:1063D000226802F1140353E8003F23F04003143213
:1063E00042E800310029F3D1A36B73B1604A1A650A
:1063F000A06BFBF796FD0028A9D0A06B036D984712
:10640000A5E72046FFF706FFD1E7204607F058FA38
:106410009DE7204607F054FA99E7204607F050FA26
:106420000023236493E713F0100F82D010F0100FB5
:106430003FF47FAF002301931368019353680193E6
:10644000019B536913F0400F50D0A26B13685B6837
:106450009BB2002B3FF47BAFA18D99427FF677AFC3
:10646000E385D369B3F5807F37D0226802F10C034E
:1064700053E8003F23F480730C3242E800310029D6
:10648000F3D1226802F1140353E8003F23F0010323
:10649000143242E800310029F3D1226802F11403DA
:1064A00053E8003F23F04003143242E80031002952
:1064B000F3D1202384F83E3000232363226802F1C5
:1064C0000C0353E8003F23F010030C3242E8003184
:1064D0000029F3D1A06BFBF7DAFCA18DE38D9BB211
:1064E000C91A89B2204607F0B5F930E7A18DE38DCE
:1064F0009BB2C91A89B2E38D9BB2002B3FF427AF40
:1065000000293FF424AF226802F10C0353E8003F56
:1065100023F490730C3242E800300028F3D1226853
:1065200002F1140353E8003F23F00103143242E860
:1065300000300028F3D1202384F83E300023236369
:10654000226802F10C0353E8003F23F010030C32E1
:1065500042E800300028F3D1204607F07BF9F6E648
:106560002046FFF7DCFBF2E62046FFF70AFEEEE6E8
:106570000562000808B5806B036B012B02D0FFF7A2
:1065800014FE08BD818D490807F064F9F9E708B5E4
:106590000346806B1B681B6813F4807F2BD100239C
:1065A000C385026802F10C0353E8003F23F48073B3
:1065B0000C3242E800310029F3D1026802F11403E1
:1065C00053E8003F23F00103143242E80031002970
:1065D000F3D1026802F1140353E8003F23F04003B3
:1065E000143242E800310029F3D1202380F83E30F4
:1065F000036B012B05D0036B012B0FD0FFF7D4FDEC
:1066000008BD026802F10C0353E8003F23F01003B9
:106610000C3242E800310029F3D1ECE7818D07F01C
:1066200019F9EDE730B583B00446134681628285DF
:1066300000250564222280F83E20826B2048D0632A
:10664000A26B20481064A26B1F48D064A26B156532
:1066500020680A46011DA06BFBF7E4FB0195236847
:106660001A6801925B680193019B84F83C5023698E
:106670005BB1226802F10C0353E8003F43F48073DE
:106680000C3242E800310029F3D1226802F11403F0
:1066900053E8003F43F00103143242E8003100297F
:1066A000F3D1226802F1140353E8003F43F04003A2
:1066B000143242E800310029F3D1002003B030BD8C
:1066C0008F65000875650008AD61000890F83E30E0
:1066D000DBB2202B29D110B582B0044639B342B3C6
:1066E00090F83C30012B27D0012380F83C30036325
:1066F000FFF798FFF0B9236B012B01D0012019E0BF
:106700000023019323681A6801925B680193019B3F
:10671000226802F10C0353E8003F43F010030C32EF
:1067200042E800310029F3D104E002207047012043
:1067300000E0012002B010BD0220FBE782B0002380
:106740000193019B01330193019A0F4B9A4215D893
:106750000369002BF5DA00230193036943F0010379
:106760000361019B01330193019A074B9A4208D8B8
:10677000036913F0010FF4D1002000E0032002B000
:1067800070470320FBE700BF400D030084B010B545
:10679000044603A880E80E00089B012B1FD1A36BC1
:1067A00023F48033A363E36823F4840323F04003DA
:1067B000E360E36823F44013E3600F9B012B09D0EF
:1067C0002046FFF7BBFF069B012B1BD0BDE8104006
:1067D00004B07047E36843F48013E360F0E7E368D4
:1067E00043F04003E3602046FFF7A8FF0C9B23B96A
:1067F000A36B43F48033A363E5E7A36B23F48033F7
:10680000A363E0E7A36843F00603A360A36843F033
:106810002003A360DAE70000022A0AD00922C36835
:1068200023F47053C360C36843EA8223C36000202B
:106830007047234B0B44234A93422FD9224B0B44DE
:10684000224A93422CD9A1F57403A3F51053204A90
:10685000934227D9A1F18373A3F5E7431D4A9342DD
:1068600022D31D4B0B441D4A93421FD91C4B0B4492
:106870001C4A93421CD31C4B0B441C4A934219D311
:10688000A1F1B773A3F55853194A934214D3194B86
:106890000B44194A934211D20722C0E70F22BEE7E8
:1068A0000E22BCE70D22BAE70C22B8E70B22B6E7AE
:1068B0000A22B4E70922B2E70822B0E70622AEE7CF
:1068C000405327FFFF340C00401E1BFF3F420F00C8
:1068D0007F4F120020D6130060B6E5FE5FE316007E
:1068E00000D3CEFE40771B00C05BB3FEC0912100F9
:1068F00020753800E05459FEE09C4100836843F065
:106900000103836000207047836823F001038360E4
:106910000020704782B000230193019B0133019353
:10692000019A0F4B9A4215D80369002BF5DA002320
:106930000193890141F020010161019B0133019321
:10694000019A074B9A4208D8036913F0200FF4D13B
:10695000002000E0032002B070470320FBE700BFE7
:10696000400D030082B000230193019B013301938A
:10697000019A0E4B9A4213D80369002BF5DA0023D3
:10698000019310230361019B01330193019A074B8B
:106990009A4208D8036913F0100FF4D1002000E0E8
:1069A000032002B070470320FBE700BF400D030047
:1069B000D0F800381943C0F80018002070470000D4
:1069C00084B02DE9F041044607A880E80E000023BA
:1069D00006E003F1400204EB820200215160013322
:1069E0000E2BF6D9119F27BBD4F8043843F00203CD
:1069F000C4F80438A36B43F40013A363A36B23F41C
:106A00000023A363A36B23F48023A3630023C4F8B0
:106A1000003E04F50065D4F80038C4F800380C9B3B
:106A2000012B14D1099B6BB900212046FFF7C0FF51
:106A300011E0A36B23F40013A363A36B43F40023BF
:106A4000A363E3E701212046FFF7B2FF03E0032140
:106A50002046FFF7ADFF10212046FFF75BFF804681
:106A600008B14FF001082046FFF77CFF08B14FF056
:106A7000010800232B616B61EB610AE0C3B94FF0A1
:106A80000060C2F8000900220A614FF67F328A6076
:106A900001330799994210D904EB431202F51061B2
:106AA000D2F800090028E9DB0020C2F80009EAE773
:106AB0004FF09040C2F80009E5E700230AE0C3B1B7
:106AC0004FF0904CC2F800CB002202614FF67F32AB
:106AD00082600133994211D904EB431202F5306010
:106AE000D2F8006B002EEADB4FF0000CC2F800CBAE
:106AF000EAE74FF0006CC2F800CBE5E72B6923F41E
:106B000080732B610023A3616FF0804363610A9B54
:106B10001BB9A36943F01003A361A2690B4B134394
:106B2000A3610D9B1BB1A36943F00803A361012F6F
:106B300004D04046BDE8F04104B07047A36943F07B
:106B4000804343F00403A361F3E700BF00383C80B7
:106B5000D0F8083813F0060307D0022B07D0062B15
:106B600001D00F207047022070470020704702209C
:106B7000704710B591F800C04B78012B23D000F579
:106B8000006ED0F81C380CF00F040122A24043EA3A
:106B90000243C0F81C3800EB4C10D0F8003B13F453
:106BA000004F0ED1D0F8003BCA68C2F30A0209793F
:106BB00042EA8142134343F0805343F40043C0F858
:106BC000003B002010BDD0F81C280CF00F0E03FA7B
:106BD0000EF39BB21343C0F81C3800EB4C10D0F8F6
:106BE000003913F4004FECD1D0F80039CA68C2F371
:106BF0000A02097942EA814242EA8C52134343F085
:106C0000805343F40043C0F80039DAE730B40B781E
:106C10004A78012A26D000EB4313D3F8002B002A30
:106C200052DBD0F83C480A7802F00F024FF0010C1A
:106C30000CFA02F224EA0242C0F83C28D0F81C28E0
:106C4000097801F00F010CFA01FC22EA0C42C0F8AD
:106C50001C28D3F8001B234A0A40C3F8002B00204D
:106C600030BC704700EB4313D3F80029002A1EDB29
:106C7000D0F83C580A7802F00F02012404FA02F21C
:106C800092B225EA0202C0F83C28D0F81C28097804
:106C900001F00F018C40A4B222EA0402C0F81C28C3
:106CA000D3F80019104A0A40C3F80029D7E7D3F8EF
:106CB000002942F00062C3F80029D3F8002942F00D
:106CC0008042C3F80029D3E7D3F8002B42F00062DA
:106CD000C3F8002BD3F8002B42F08042C3F8002BFE
:106CE0009FE700BF0078F3EF007833EC70B40B78C7
:106CF0004C78012C29D000EB431000F530631C695F
:106D0000E40CE4041C611C6924F0FF5424F4C01456
:106D10001C618C690CB1CC688C61CC68CC611C693D
:106D200044F400241C611C69CD69C5F3120C44EACB
:106D30000C041C61012A66D0D0F8003B43F00443E8
:106D4000C0F8003B002070BC70478C696CBB00EB46
:106D50004314D4F8105925F0FF5525F4C015C4F894
:106D60001059D4F8105945F40025C4F81059D4F836
:106D70001059ED0CED04C4F81059012A34D000EB81
:106D80004313D3F8002942F00442C3F800298B6969
:106D9000002BD7D0D0F83438097801F00F01012248
:106DA0008A401343C0F83438CCE700EB431404F5B1
:106DB00010642569ED0CED042561256925F0FF556A
:106DC00025F4C0152561CD688E69AE4200D98D616C
:106DD000256945F40025256125698E69C6F3120CE5
:106DE00045EA0C052561C8E74A691AB100EB431171
:106DF000C1F8142900EB4313D3F8002942F00442F0
:106E0000C3F800299EE70A69002A95D05A6193E7E2
:106E100010B483B0024600230193487801280BD0B8
:106E20000B7802EB4313D3F8000B00282DDB002076
:106E300003B05DF8044B70470B7802EB4313D3F8B3
:106E40000049002C01DB0020F2E7D3F8004944F0B0
:106E50000064C3F800490B7802EB4313D3F80049F0
:106E600044F08044C3F80049019B01330193019C25
:106E700042F210739C42DBD80B7802EB4313D3F839
:106E80000039002BF0DB0020D2E7D3F8000B40F0F4
:106E90000060C3F8000B0B7802EB4313D3F8000B30
:106EA00040F08040C3F8000B019B0133019301982F
:106EB00042F21073984208D80B7802EB4313D3F8D0
:106EC000003B002BF0DB0020B2E70120B0E710B55B
:106ED0009DF8084084B903334FEA930E4FF0000C3D
:106EE00008E000EB023303F5805351F8044B1C60BB
:106EF0000CF1010CF445F4D3002010BDF0B583B0C3
:106F00000B784C78012C33D000EB431303F5306C35
:106F1000DCF81040E40CE404CCF81040DCF810403D
:106F200024F0FF5424F4C014CCF810408C69002CD9
:106F300040F0C780DCF81040CD68C5F312052C4343
:106F4000CCF81040DCF8104044F40024CCF8104099
:106F5000012A00F0D0800A79012A00F0D380D3F80A
:106F6000002B42F00442C3F8002B002003B0F0BD18
:106F70008C6984BB00EB4314D4F8105925F0FF55FD
:106F800025F4C015C4F81059D4F8105945F400255B
:106F9000C4F81059D4F81059ED0CED04C4F8105988
:106FA000012A4CD000EB4313D3F8004944F00444C9
:106FB000C3F800490C79012C6AD08B69002BD4D01E
:106FC000D0F83438097801F00F0101228A401343C8
:106FD000C0F83438C9E700EB4314D4F81059ED0C6D
:106FE000ED04C4F81059D4F8105925F0FF5525F4D4
:106FF000C015C4F81059D4F810698D69CF683D44A4
:10700000013DB5FBF7F5494F07EAC5453543C4F8DF
:107010001059D4F810598E69C6F312063543C4F8D6
:10702000105904F510640D79012DB9D1256925F0A9
:10703000C0452561256945F000552561B0E74A69DD
:107040001AB100EB4314C4F814290A79012A08D0B4
:1070500000EB4313D3F8002942F00442C3F800299F
:1070600083E7D0F8082812F4807F08D100EB4311A1
:10707000D1F8002942F00052C1F80029E8E700EBFE
:107080004311D1F8002942F08052C1F80029DFE70E
:10709000D0F8084814F4807F0CD1D3F8004944F0AC
:1070A0000054C3F8004900920B8B0A780969FFF776
:1070B0000EFF5AE7D3F8004944F08054C3F8004962
:1070C000F1E7CD682C44013CB4FBF5F4A4B204FB19
:1070D00005F5CD61DCF81050144E06EAC4442C438B
:1070E000CCF81040DCF81040CD69C5F312052C43F4
:1070F000CCF810402CE70A69002A3FF42CAFCCF8FA
:10710000142028E7D0F8082812F4807F06D1D3F89D
:10711000002B42F00052C3F8002B20E7D3F8002BDD
:1071200042F08052C3F8002B19E700BF0000F81F9F
:1071300010B5844608464FEA920E02F0030200237F
:1071400005E00CF58051096840F8041B01337345D4
:10715000F7D37AB10CF5805CDCF800400021CBB2AB
:10716000DB0024FA03F300F8013B0131013A92B24B
:10717000002AF4D110BD0B784A78012A14D000EB14
:107180004310D0F8002B002A06DB2BB1D0F8003BCF
:1071900023F08043C0F8003BD0F8003B43F40013D9
:1071A000C0F8003B0020704700EB4310D0F80029E6
:1071B000002A06DB2BB1D0F8003923F08043C0F859
:1071C0000039D0F8003943F40013C0F80039E9E77A
:1071D0000B784A78012A0ED000EB4310D0F8003B20
:1071E00023F40013C0F8003B0B79023BDBB2012B08
:1071F00015D90020704700EB4310D0F8003923F474
:107200000013C0F800390B79023BDBB2012BF0D838
:10721000D0F8003943F08053C0F80039E9E7D0F8DE
:10722000003B43F08053C0F8003BE2E7D0F8003861
:1072300023F4FE63C0F80038D0F80038090101F4E7
:10724000FE610B43C0F8003800207047D0F8003EC4
:1072500023F00303C0F8003ED0F8043823F0020303
:10726000C0F8043800207047D0F8003E23F0030334
:10727000C0F8003ED0F8043843F00203C0F80438E8
:10728000002070474269806910407047D0F8183874
:1072900000F50060C0691840000C7047D0F818383D
:1072A00000F50060C069184080B2704700EB4111E2
:1072B000D1F8082B00F50060406910407047D0F805
:1072C0001028D0F8343801F00F0C23FA0CF3DB014E
:1072D000DBB2134300EB411000F5106080681840EA
:1072E0007047406900F00100704738B50546C36833
:1072F00023F0C043C360012913D019BBC36843F016
:107300008043C36000240120F9F74EFE0134284673
:10731000FFF7E7FF08B1312CF5D9322C14D000204B
:1073200038BDC36843F00053C36000240120F9F75F
:107330003BFE01342846FFF7D4FF0128EDD0312C65
:10734000F4D9EAE70120EBE70120E9E7D0F80039BA
:1073500023F4FF6323F00703C0F80039D0F80438A2
:1073600043F48073C0F804380020704710B4046CF4
:10737000154B9C4203D9D0F8003B002B16DB0024B0
:10738000C0F8104BD0F8104B44F40024C0F8104B58
:10739000D0F8104B44F01804C0F8104BD0F8104B44
:1073A00044F0C044C0F8104B012903D000205DF820
:1073B000044B7047C0F8142BD0F8003B43F08023F7
:1073C000C0F8003BF2E700BF0A30544F10B5D0F8C8
:1073D000D43203F1B00250F822408CB100EB8200AD
:1073E00043687BB194F80002FF280DD09B6894F8A5
:1073F000012221469847FF2384F80032002010BD67
:107400000320FCE70020FAE70020F8E70A230380C6
:107410000048704784000020F8B506460F4F8221CF
:10742000384600F01FFC05460121384600F01AFCE2
:1074300004468121384600F015FC0DB11022AA71D6
:107440001CB1402222710022627118B140220271E7
:1074500000224271432333800048F8BD0800002019
:10746000F8B506460F4F8221384600F0FBFB054673
:107470000121384600F0F6FB04468121384600F031
:10748000F1FB0DB11022AA711CB140222271002221
:10749000627118B14022027100224271432333808D
:1074A0000048F8BD08000020F8B506460F4F8221BD
:1074B000384600F0D7FB05460121384600F0D2FBE4
:1074C00004468121384600F0CDFB0DB11022AA718F
:1074D0001CB1002222710222627118B100220271D5
:1074E00002224271432333800048F8BD0800002087
:1074F00038B5D0F8D432B03350F8235095B10446A3
:1075000004F01FF9C5F80C02D4F8D432B03304EB00
:1075100083046368DB6805F50371D5F804029847B6
:10752000002038BD0320FCE738B5D0F8C852D0F8A9
:10753000D432B03350F8234084B301F00F0303EB8F
:10754000830200EB820292694AB103EBC30C05EBA4
:107550008C05AD6CB2FBF5FC05FB1C2292B100233F
:10756000C4F81432D0F8D432B03300EB830043684F
:107570001B69ABB10A4604F50471D4F808029847B8
:10758000002038BD03EB830300EB830300249C61E0
:107590002346224604F01EF92046F2E70320F0E7D6
:1075A0000020EEE7F0B583B0D0F8D43203F1B0029A
:1075B00050F8227000228DF80720ADF80420002F2B
:1075C0007BD004460D46097811F0600634D0202E99
:1075D0006CD1EA882AB311F0800F07D16B7887F855
:1075E0000032EA883F2A13D8D2B212E0B03300EB5F
:1075F00083035B689B68394668789847EA88072A5E
:1076000028BF07223946204600F0DCFE002651E064
:10761000402287F801223946204600F0E8FE002685
:1076200048E0B03300EB83035B689B680022294687
:107630006878984700263DE06F780B2F31D8DFE857
:1076400007F006393030303030303030162690F8C0
:107650009C32DBB2032B04D0294600F040FB03260A
:1076600028E0022201A900F0ADFE3E4622E090F89B
:107670009C32DBB2032B04D0294600F030FB0326FA
:1076800018E001220DF1070100F09CFE12E090F8D5
:107690009C32DBB2032B0DD0294600F020FB0326E1
:1076A00008E0294600F01BFB032603E0294600F012
:1076B00016FB0326304603B0F0BD0326FAE738B5C3
:1076C0000446812104F066F8002525870121204623
:1076D00004F060F8A4F878518221204604F05AF8AA
:1076E000A4F84C50A4F84E50D4F8D43203F1B002B0
:1076F00054F822209AB1B03304EB83035B685B68D3
:107700009847D4F8D432B03354F8230004F024F866
:10771000D4F8D432B03344F82350C4F8BC5200201B
:1077200038BD70B504464FF4077004F011F8002816
:1077300049D005464FF40772002110F07BFCD4F8C5
:10774000D432B03344F82350C4F8BC52237C002B0D
:1077500041D14FF4007302228121204604F00FF83A
:10776000012626874FF4007302223146204604F09A
:1077700006F8A4F878611023A4F84E3008230322F9
:107780008221204603F0FBFF0123A4F84C300026A1
:10779000C5F80462D4F8D432B03304EB83035B68D9
:1077A0001B689847C5F81462C5F81862D5F804221A
:1077B00062B3257C1DBB4FF400730121204604F009
:1077C00011F8284670BDD4F8D432B033002244F802
:1077D00023200225F5E7402302228121204603F0E1
:1077E000CEFF01262687402302223146204603F0A1
:1077F000C6FFA4F878611023A4F84E30BEE74023FA
:107800000121204603F0EEFF0025DAE70225D8E744
:1078100039B1D0F8D432B03300EB8300416000209E
:10782000704703207047D0F8D432B03350F823307B
:107830002BB1C3F80812C3F81022002070470320B0
:107840007047D0F8D432B03350F823301BB1C3F8AE
:107850000412002070470320704710B5D0F8D432CE
:10786000B03350F8232092B1047C44B94FF4007334
:10787000D2F80422012103F0B5FF204610BD4023B9
:10788000D2F80422012103F0ADFF0024F5E7032420
:10789000F3E798B108B503460020C3F8B802C3F86F
:1078A000C402C3F8D00209B1C3F8B412012183F8AD
:1078B0009C121A70184603F0F9FE08BD03207047A9
:1078C00010B582B00023ADF8063089B10446C0F887
:1078D000B812CB6A23B10DF106009847C4F8D00264
:1078E000D4F8D8320133C4F8D832002002B010BD29
:1078F0000320FBE708B503F03AFF08BD08B5D0F850
:10790000B83213B11B68984708BD0020FCE708B5E2
:10791000D0F8B8325B68984700B908BD0320FCE78F
:1079200038B5044600F2AA25284600F0C4F9012320
:10793000C4F89432B4F8B032C4F8983294F8AA1269
:1079400001F01F03012B0DD0022B10D02BB101F041
:107950008001204603F026FF03E02946204600F080
:107960007FFB38BD2946204600F0B5FBF9E72946E4
:10797000204600F0F2FBF4E7F8B50446012380F856
:107980009C320023C0F894324360C0F8A43280F8DF
:10799000A032D0F8B832DBB15B68DBB10021984788
:1079A0000746C8B9402300221146204603F0E7FEEF
:1079B0000126A4F864614025C4F860512B460022DA
:1079C0008021204603F0DBFEA68425623846F8BD00
:1079D0000027E7E70027E5E70327E3E70174002036
:1079E000704790F89C32DBB280F89D32042380F817
:1079F0009C320020704790F89C32DBB2042B01D0FF
:107A00000020704790F89D32DBB280F89C32F7E797
:107A100008B590F89C32DBB2032B01D0002008BDE2
:107A2000D0F8B832002BF9D0DB69002BF6D098479C
:107A3000F4E708B5D0F8D432AE3350F823205AB169
:107A400090F89C32DBB2032B01D0002008BD136AF2
:107A500023B198470020F9E70320F7E70020F5E776
:107A600008B5D0F8D432AE3350F823205AB190F88C
:107A70009C32DBB2032B01D0002008BD536A23B136
:107A800098470020F9E70320F7E70020F5E70020FA
:107A9000704708B5012380F89C32D0F8B83223B182
:107AA0005B680179984710B908BD0020FCE7032006
:107AB000FAE7002070470020704738B504460D46AD
:107AC000002943D11346D0F89422032A01D0084656
:107AD00038BDD0F85C11D0F86021914212D890F8EE
:107AE000AA3203F01F03012B17D0022B1CD028460B
:107AF00094F89C32DBB2032B1BD0204600F08EFCA6
:107B00002846E5E7891AC0F85C118A4228BF0A4670
:107B1000194600F07BFC2846DAE790F8AE12FFF732
:107B2000C8FF0028E9D1E3E790F8AE12FFF7C3FFE2
:107B3000F7E700F1AE0354F823301A69002ADCD0CD
:107B4000C4F8D4021B6920469847D6E701F07F01AC
:107B5000FFF7B1FF90B994F89C32DBB2032BB7D199
:107B600000F1AE0354F823309A69002AB0D0C4F86B
:107B7000D4029B69294620469847A9E70020A7E739
:107B800038B504460D4600294BD11346D0F894224F
:107B9000022A07D094F8A00218B1002384F8A0327A
:107BA000284638BDC269016A8A420ED88A4218D076
:107BB00094F89C32DBB2032B27D08021204603F0BF
:107BC000F1FD204600F035FCE4E7521AC261194687
:107BD00000F005FC00231A461946204603F002FE79
:107BE000D8E783699942E3D8D0F898229342DFD24C
:107BF0000022114600F0F3FB0021C4F898120B4656
:107C00000A46204603F0EEFDC4E7D4F8B832DA683D
:107C1000002AD2D00022C4F8D422DB68204698473C
:107C2000CBE741F08001FFF746FF90B994F89C3212
:107C3000DBB2032BB5D100F1AE0354F823305A69FF
:107C4000002AAED0C4F8D4025B6929462046984782
:107C5000A7E70020A5E70B88027813440B80037880
:107C600018447047428803789A4218D930B583B0D7
:107C700004460D46ADF806306388BDF806209A42EA
:107C80000AD20DF10601FFF7E6FF4378052BF3D189
:107C90008378AB42F0D100E0002003B030BD00207B
:107CA00070470346002002E00130C0B201331A7869
:107CB000002AF9D170470B7803704B7843708B78AA
:107CC000CA7843EA022343800B794A7943EA0223C4
:107CD00083808B79CA7943EA0223C380704710B549
:107CE0000446802103F05EFD0021204603F05AFD8A
:107CF00010BD30B583B004460D460023ADF8063004
:107D00004A88130A013B062B00F2AB80DFE803F040
:107D1000041F33A9A98D9A00D0F8B4321B680DF165
:107D20000601007C9847EA88002A00F0A380BDF88D
:107D30000630002B00F099809A4228BF1A46ADF811
:107D400006200146204600F03DFB03B030BD037C19
:107D500043B9D0F8B8329B6A0DF106009847022368
:107D60004370E0E7D0F8B832DB6A0DF106009847BF
:107D700002234370D7E7D2B2052A52D8DFE802F0D7
:107D800003101D2A3744D0F8B4325B6823B10DF1DB
:107D90000601007C9847C6E72946FFF7A0FFD4E715
:107DA000D0F8B4329B6823B10DF10601007C9847EE
:107DB000B9E72946FFF793FFC7E7D0F8B432DB688D
:107DC00023B10DF10601007C9847ACE72946FFF787
:107DD00086FFBAE7D0F8B4321B6923B10DF1060172
:107DE000007C98479FE72946FFF779FFADE7D0F879
:107DF000B4325B6923B10DF10601007C984792E72C
:107E00002946FFF76CFFA0E7D0F8B4329B6923B195
:107E10000DF10601007C984785E72946FFF75FFFD3
:107E200093E72946FFF75BFF8FE7037C33B9D0F870
:107E3000B8325B6B0DF10600984774E72946FFF7EF
:107E40004EFF82E7037C43B9D0F8B8321B6B0DF1CB
:107E5000060098470723437065E72946FFF73FFF71
:107E600073E72946FFF73BFF6FE729462046FFF7F8
:107E700036FF6AE7204600F0D1FA66E738B50446D7
:107E80008B88FBB9CB88EBB94B887F2B1AD803F0D2
:107E90007F0590F89C32DBB2032B0CD080F89E5209
:107EA000294603F08FFC204600F0B8FA35B10223D2
:107EB00084F89C3209E0FFF712FF06E0012384F802
:107EC0009C3202E02046FFF70AFF38BD70B5044639
:107ED0000E468D782F4B1D70012D10D890F89C32D6
:107EE000DBB2022B0FD0032B26D0FFF7F8FE294B75
:107EF00019782046FFF70BFD0325284670BDFFF7D4
:107F0000EEFE0325F9E7A5B145602946FFF7F6FC2B
:107F1000054638B131462046FFF7E1FE022384F8DA
:107F20009C32EAE7204600F079FA032384F89C3279
:107F3000E3E700F073FAE0E7CDB141688D4225D068
:107F4000C9B2FFF7E4FC134B197861602046FFF7D4
:107F5000D5FC0546B0B131462046FFF7C0FE217979
:107F60002046FFF7D4FC022384F89C32C5E70223A5
:107F700080F89C3245602946FFF7C9FC204600F096
:107F80004DFABAE7204600F049FAB6E700F046FAA3
:107F90000025B2E7480D002008B5CB88012B0BD196
:107FA00090F89C32DBB2022B09D9032B09D10122B4
:107FB000011D00F007FA01E0FFF791FE08BD5BB27A
:107FC00013B9FFF78CFEF9E70146002341F8083F9B
:107FD000012200F0F7F9F1E708B590F89C32013B77
:107FE000022B12D8CB88022B0CD10123C360D0F80E
:107FF000A4320BB10323C360022200F10C0100F094
:10800000E1F908BDFFF76BFEFBE7FFF768FEF8E755
:1080100008B54B88012B04D0022B07D0FFF75FFE79
:1080200008BDC0F8A43200F0F9F9F9E78B881B0A03
:1080300080F8A03200F0F2F9F2E708B590F89C322F
:10804000013B022B09D84B88012B00D008BD00232F
:10805000C0F8A43200F0E2F9F8E7FFF740FEF5E7D8
:1080600038B50C7804F06004202C06D0402C04D0E5
:108070006CB1FFF734FE002407E0D0F8D432AE3301
:1080800050F823309B6898470446204638BD4D7809
:10809000092D1DD8DFE805F012191C161C08051C57
:1080A0000F0BFFF726FEF0E7FFF7E8FEEDE7FFF71F
:1080B0000DFF0446E9E7FFF76FFFE6E7FFF78CFFE8
:1080C0002C46E2E7FFF7A4FFDFE7FFF7B6FFDCE7A8
:1080D000FFF705FED9E770B505460C460B7803F0AF
:1080E0006003202B07D0402B05D023B1FFF7F7FD0D
:1080F0000026304670BD95F89C32013B022B26D8F5
:108100002179012905D921462846FFF7E8FD0026F7
:10811000EFE72846FFF7CDFC68B900F1AE0255F84D
:108120002220916889B1C5F8D40293682146284677
:108130009847064600E00326E388002BD9D1002E9D
:10814000D7D1284600F06AF9D3E70326F4E72146A1
:108150002846FFF7C4FD0026CBE72DE9F04106468F
:108160000D468B88DFB20C7804F06004202C08D018
:10817000402C06D0DCB1FFF7B2FD00242046BDE85C
:10818000F08139463046FFF796FC0446002840F05F
:10819000F880C6F8D40200F1AE0356F823309B688D
:1081A000002BEBD02946304698470446E6E791F885
:1081B0000180B8F1010F31D0B8F1030F05D0B8F14B
:1081C000000F67D0FFF78BFDD8E790F89C32DBB249
:1081D000022B04D0032B12D0FFF781FDCEE70FB1A5
:1081E000802F04D129463046FFF779FDC6E739468E
:1081F00003F0D8FA8021304603F0D4FABEE74B886A
:1082000023B91FB1802F01D0CB881BB1304600F0BD
:1082100005F9B3E7394603F0C5FAF7E790F89C3261
:10822000DBB2022B04D0032B12D0FFF758FDA5E7D9
:108230000FB1802F04D129463046FFF750FD9DE74E
:10824000394603F0AFFA8021304603F0ABFA95E7E8
:108250004B88002B92D117F07F0F17D1304600F0DA
:10826000DDF839463046FFF726FC002886D1C6F8EF
:10827000D40200F1AE0256F822209268002A00F0E3
:108280008280294630469047044677E7394603F016
:1082900091FAE3E790F89C22D2B2022A05D0032A91
:1082A00027D0FFF71CFD444668E70FB1802F13D19C
:1082B00013F0800F14D107F07F0707EB8707B90091
:1082C00001F5A8713144043100230B6002223046CD
:1082D00000F078F8444651E7FFF701FD44464DE7CA
:1082E00007F07F0707EB8707B900103131440431ED
:1082F000EAE75BB2002B1FDB07F00F0202EB820202
:1083000000EB8202B2F864211AB3002B25DB07F0E0
:108310007F0303EB83039C0004F5A8743444043406
:108320000FB1802F22D10023236002222146304644
:1083300000F048F8444621E707F00F0202EB820202
:1083400000EB8202928C002ADFD1FFF7C8FC444682
:1083500014E7FFF7C4FC444610E707F07F0303EB84
:1083600083039C00103434440434D9E73946304642
:1083700003F0D0F910B101232360D6E70023236076
:10838000D3E70024FAE60446F8E6D0B170B50D460E
:1083900016460446FFF785FC431C5B009BB2338006
:1083A0002B7003236B70022307E0EA5401345A1C3C
:1083B000D2B20021A9540233DBB22278002AF4D1D0
:1083C00070BD704708B513460222C0F8942283613D
:1083D000C3610A46002103F0FDF9002008BD08B57D
:1083E00013460A46002103F0F5F9002008BD08B540
:1083F00013460322C0F89422C0F85831C0F85C310B
:108400000A46002103F0EEF9002008BD08B5134626
:108410000A46002103F0E6F9002008BD08B5042251
:10842000C0F8942200231A46194603F0D3F900201D
:1084300008BD08B50522C0F8942200231A46194643
:1084400003F0D0F9002008BD842801D00330704724
:108450000020704708B500F0A5FD002008BD2DE9FB
:10846000F04387B00E464469C4B18569B5B1476829
:10847000D0F80080D0F81090B0F90800FFF7E4FFC2
:1084800002950194009033464A464146384600F032
:10849000ABFC0590059807B0BDE8F083446805681B
:1084A0000769B0F90800FFF7CFFF05AB0193009013
:1084B0003346BAB22946204600F0D1FC0128E9D063
:1084C0000020E8E708B500B9012000F0B5FE002063
:1084D00008BD00F1080343604FF0FF328260C360C3
:1084E0000361002303607047002303617047436802
:1084F0004B609A688A605160996008610368013333
:108500000360704730B40D68B5F1FF3F11D000F142
:1085100008031C465B681A68AA42FAD963684B6074
:1085200099608C606160086103680133036030BC4E
:1085300070470469F2E70369416882688A604168AC
:1085400051605A68824206D0002202611A68013ADC
:108550001A601868704782685A60F5E782B0002395
:1085600001930D4B1B68B3F1FF3F08D04FF0500350
:1085700083F31188BFF36F8FBFF34F8FFEE74FF088
:10858000500383F31188BFF36F8FBFF34F8F019BAD
:10859000002BFCD002B07047900000200848006813
:1085A000006880F308884FF0000080F3148862B6FA
:1085B00061B6BFF34F8FBFF36F8F00DF00BF0000C6
:1085C00008ED00E0DFF80C00016841F47001016083
:1085D0007047000088ED00E04FF0807340F8043CE5
:1085E00021F0010140F8081C054B40F80C3C40F814
:1085F000202C6FF0020340F8243C4438704700BF41
:108600005D85000800000000000000000000000080
:10861000074B19680868B0E8F04F80F30988BFF38A
:108620006F8F4FF0000080F311887047AFF3008028
:10863000BC5C00204FF0500383F31188BFF36F8FB1
:10864000BFF34F8F0B4A136801331360012B00D027
:1086500070474FF0E023D3F8043D13F0FF0FF7D03D
:108660004FF0500383F31188BFF36F8FBFF34F8F29
:10867000FEE700BF90000020094B1B6843B94FF094
:10868000500383F31188BFF36F8FBFF34F8FFEE763
:10869000013B034A13600BB983F31188704700BF95
:1086A000900000200000000000000000000000001A
:1086B000EFF30980BFF36F8F154B1A681EF0100F90
:1086C00008BF20ED108A20E9F04F10602DE9090065
:1086D0004FF0500080F31188BFF34F8FBFF36F8FBF
:1086E00000F0D0FD4FF0000080F3118809BC19683C
:1086F0000868B0E8F04F1EF0100F08BFB0EC108A09
:1087000080F30988BFF36F8F704700BFAFF300801D
:10871000BC5C002008B54FF0500383F31188BFF311
:108720006F8FBFF34F8F00F07FFC28B14FF0E02335
:108730004FF08052C3F8042D002383F3118808BD45
:108740004FF0E022002313619361054B1B6805493C
:10875000A1FB03139B09013B53610723136170477E
:1087600094000020D34D62104FF0E023D3F8002D89
:108770003D4B9A421CD04FF0E023D3F8002D3B4BE9
:108780009A421ED030B583B0394B1A78D2B20192DA
:10879000FF221A701B78DBB28DF803309DF803308E
:1087A00003F05003334A1370334B07221A601BE067
:1087B0004FF0500383F31188BFF36F8FBFF34F8FD8
:1087C000FEE74FF0500383F31188BFF36F8FBFF3C1
:1087D0004F8FFEE7284A1368013B13609DF8033072
:1087E0005B00DBB28DF803309DF8033013F0800F8F
:1087F000F0D1214B1B68032B08D04FF0500383F3BB
:108800001188BFF36F8FBFF34F8FFEE71B021A4A29
:10881000136003F4E0631360019BDBB2144A13702E
:108820004FF0E024D4F8203D43F47003C4F8203D19
:10883000D4F8203D43F07043C4F8203DFFF780FF9B
:1088400000250E4B1D60FFF7BDFED4F8343F43F00A
:108850004043C4F8343FFFF7A1FE00F013FDFFF7DB
:108860007DFE284603B030BD71C20F4170C20F417A
:1088700000E400E0500D00204C0D0020900000208E
:10888000134A12F0070F1FD0D11D21F00701C1F5C7
:108890009C43203313440A460E4802600021416085
:1088A0001344083B23F007030B4803605960196029
:1088B000991A51601360094B1960094B1960094BF3
:1088C0004FF000421A60704744F62063E4E700BFAF
:1088D000740D00206C0D0020680D0020600D00203C
:1088E000640D0020540D0020164B1A461B6883426D
:1088F000FBD3516802EB010C844509D0416800EBC1
:10890000010C634509D00360904219D01060704794
:108910004068014451601046F0E710B40A4C2468E6
:10892000A3420BD05B681944416013681B68036065
:10893000904200D010605DF8044B70470460F7E788
:10894000704700BF6C0D0020680D002038B504464C
:1089500000F062FB384B1B68B3B1384B1B681C42FC
:1089600050D1002C50D004F1080214F0070F02D0AF
:1089700022F007020832002A55D0314B1B6893427F
:1089800053D330490C6804E0FFF77AFFE5E721464E
:108990001C466368934202D22368002BF7D1264B12
:1089A0001B68A34243D00D68083523680B606368D9
:1089B0009B1A102B10D9A01810F0070F08D04FF0F9
:1089C000500383F31188BFF36F8FBFF34F8FFEE720
:1089D00043606260FFF788FF626819490B689B1A61
:1089E0000B60194909688B4201D217490B60134B80
:1089F0001B681343636000232360144A1368013328
:108A0000136002E0002500E0002500F099FB15F05E
:108A1000070F0ED04FF0500383F31188BFF36F8F11
:108A2000BFF34F8FFEE70025EFE70025EDE70025B8
:108A3000EBE7284638BD00BF680D0020540D00202C
:108A4000640D00206C0D0020600D00205C0D0020E6
:108A5000002834D038B50446A0F1080550F8043C8D
:108A6000174A1268134208D14FF0500383F311885C
:108A7000BFF36F8FBFF34F8FFEE750F8081C41B173
:108A80004FF0500383F31188BFF36F8FBFF34F8F05
:108A9000FEE723EA020340F8043C00F0BDFA54F874
:108AA000041C084A13680B4413602846FFF71CFF98
:108AB000054A13680133136000F042FB38BD70476C
:108AC000540D0020640D0020580D0020084B1B6839
:108AD0001B6823B9074B4FF0FF321A607047044BF5
:108AE0001B68DB68DB685A68024B1A60704700BF7E
:108AF000045C00209C5B00202DE9F0470746984667
:108B0000089DDDF824900A9C266B02F18042013A10
:108B100006EB820626F00706C1B308464FF0000CAC
:108B2000BCF11F0F09D810F80C2004EB0C0383F8DC
:108B3000342012B10CF1010CF2E7002384F8533019
:108B4000062D00D90625E56265654FF0000AC4F8D8
:108B500058A0201DFFF7C8FC04F11800FFF7C4FC63
:108B60002461C5F10705A5616462C4F85CA084F8BE
:108B700060A0424639463046FFF72EFD2060B9F12D
:108B8000000F01D0C9F80040BDE8F087002384F849
:108B90003430D5E738B5002407E004EB84029300B5
:108BA0000E481844FFF795FC0134062CF5D90C4DFE
:108BB0002846FFF78EFC0B4C2046FFF78AFC0A483C
:108BC000FFF787FC0948FFF784FC0948FFF781FCA1
:108BD000084B1D60084B1C6038BD00BF305C002096
:108BE0001C5C0020085C0020EC5B0020D85B0020AF
:108BF000C05B0020045C0020005C002010B504462F
:108C0000FFF718FD214A136801331360204B1B68DE
:108C10005BB1204B1B686BB91D4B1B68DA6AE36ABA
:108C20009A4207D81A4B1C6004E0194B1C60136869
:108C3000012B28D0184A136801331360E06A01231E
:108C40008340164A11680B43136000EB8000211D1E
:108C5000134B03EB8000FFF74AFCFFF70DFD0D4BB4
:108C60001B687BB10A4B1B68DA6AE36A9A4209D235
:108C70004FF0E0234FF08052C3F8042DBFF34F8F25
:108C8000BFF36F8F10BDFFF785FFD3E7BC5B0020FC
:108C9000BC5C0020B05B0020A05B0020B45B002027
:108CA000305C002010B5044690F8613063B1012BB0
:108CB00011D0022B0ED04FF0500383F31188BFF375
:108CC0006F8FBFF34F8FFEE7006BFFF7C1FE2046AB
:108CD000FFF7BEFE10BDFFF7BBFEFBE70F4B1B68A7
:108CE000D3B110B5FFF7A6FC0D4BDB68DC68201D87
:108CF000FFF721FC0B4A1368013B1360074A136816
:108D0000013B1360FFF7B8FC2046FFF7CBFF034B96
:108D10001B68002BE6D110BD704700BFD45B00205C
:108D2000D85B0020BC5B002008B5FFF7D7FF074BDE
:108D30001B68012BF9D94FF0E0234FF08052C3F8A4
:108D4000042DBFF34F8FBFF36F8FEEE7305C002031
:108D500070B504460D461D4B1E681D4B1868043047
:108D6000FFF7E9FB48B91A4B1B68DB6A01229A40FE
:108D700018490B6823EA02030B60B4F1FF3F0DD0E2
:108D80003444134B1B685C60A64210D9124B186820
:108D90000F4B19680431FFF7B5FB70BD002DEFD004
:108DA0000B4B196804310D48FFF7A1FBF5E70C4B9D
:108DB0001868074B19680431FFF7A4FB094B1B68BF
:108DC000A342EAD9074B1C60E7E700BFB85B00206D
:108DD000BC5C0020B45B0020005C0020C05B002075
:108DE000045C00209C5B002030B587B00B9C7CB1FC
:108DF0000C9DB5B164250495049D642D1AD04FF0E7
:108E0000500383F31188BFF36F8FBFF34F8FFEE7DB
:108E10004FF0500383F31188BFF36F8FBFF34F8F71
:108E2000FEE74FF0500383F31188BFF36F8FBFF35A
:108E30004F8FFEE7049D0C9D2C63022485F8614052
:108E400000240394029505AC01940A9C0094FFF75A
:108E500053FE0C98FFF7D2FE059807B030BD2DE900
:108E6000F04385B00746884614461E469000FFF73B
:108E70006DFD08B381466420FFF768FD0546A8B183
:108E8000C0F83090002380F86130039302900D9B6E
:108E900001930C9B00933346224641463846FFF728
:108EA0002BFE2846FFF7AAFE012007E04846FFF701
:108EB000CFFD4FF0FF3001E04FF0FF3005B0BDE8CF
:108EC000F083000038B50446FFF7B4FB002C34D023
:108ED000251D2846FFF72FFB70B9E26A02EB8203DB
:108EE0009B002749CB583BB9012303FA02F22549DD
:108EF0000B6823EA02030B60A36A1BB104F118009C
:108F0000FFF719FB204A1368013313601F4B1B68DE
:108F1000A34215D01E4A1368013B13602046FFF799
:108F2000C1FEFFF7D3FDFFF7A7FB1A4B1B681BB170
:108F3000164B1B68A3420CD038BD144B1C68C7E706
:108F400029461548FFF7D3FA144A13680133136012
:108F5000E9E7134B1B6843B14FF0500383F31188CB
:108F6000BFF36F8FBFF34F8FFEE74FF0E0234FF05B
:108F70008052C3F8042DBFF34F8FBFF36F8FDBE731
:108F8000305C0020B45B0020A05B0020BC5C0020B3
:108F9000BC5B0020B05B0020D85B0020D45B0020CD
:108FA000945B002010B588B000240594069407AAAD
:108FB00006A905A800F006FF059B0293069B0193F6
:108FC00000942346079A0E490E48FFF70DFF0E4BFB
:108FD000186090B14FF0500383F31188BFF36F8F87
:108FE000BFF34F8F094B4FF0FF321A60084B01223D
:108FF0001A60084B1C60FFF7B7FB08B010BD00BF3C
:10900000E0C40108298D0008985B00209C5B0020CB
:10901000B05B0020B85B0020024A13680133136084
:10902000704700BF945B0020F8B53A4B1B68002BDB
:1090300069D1394B1D6801351D60C5B9374B1B68B7
:109040001B6843B14FF0500383F31188BFF36F8F58
:10905000BFF34F8FFEE7314A1168314B186810603B
:109060001960304A136801331360FFF72FFD2E4B50
:109070001B68AB423DD900272C4B1B68DB6A03EB16
:1090800083039A002A4B9B58012B00D90127294BB7
:109090001B68002B3CD001273AE001271F4B1B68BF
:1090A0001B6843B31D4B1B68DB68DC6863689D422B
:1090B00026D3261D3046FFF73EFAA36A1BB104F102
:1090C0001800FFF738FAE36A01229A401A49086843
:1090D00002430A6003EB83039A00314614481044AC
:1090E000FFF705FAE26A114B1B68DB6A9A42D4D299
:1090F000D4E70027D2E70C4B4FF0FF321A60BBE7F2
:10910000094A1360B8E70D4A13680133136000275A
:109110003846F8BD945B0020B85B0020045C00205A
:10912000005C0020A45B00209C5B0020BC5C002055
:10913000305C0020A85B0020B45B0020AC5B00200A
:1091400038B5354B1B6843B94FF0500383F3118892
:10915000BFF36F8FBFF34F8FFEE7FFF76BFA2E4B16
:109160001A68013A1A601B68002B4FD12B4B1B6801
:109170000BB900244BE00024294B1B681BB3284B80
:10918000DB68DC6804F11800FFF7D5F9251D2846D7
:10919000FFF7D1F9E06A01238340224A11680B43AB
:1091A000136000EB800029461F4B03EB8000FFF7A4
:1091B0009EF9E26A1D4B1B68DB6A9A42DCD31C4BAA
:1091C00001221A60D8E70CB1FFF780FC194B1C682C
:1091D00084B9174B1C68D4B14FF0E0234FF0805294
:1091E000C3F8042DBFF34F8FBFF36F8F01240EE040
:1091F000013C07D0FFF718FF0028F9D00C4B0122E3
:109200001A60F5E70B4B00221A60E2E70024FFF733
:1092100033FA204638BD00BF945B0020BC5B0020C1
:10922000EC5B0020B45B0020305C0020BC5C0020C4
:10923000A85B0020AC5B002010B5A8B10446104B21
:109240001B6843B14FF0500383F31188BFF36F8F56
:10925000BFF34F8FFEE7FFF7DFFE00212046FFF749
:1092600077FDFFF76DFF48B94FF0E0234FF08052D4
:10927000C3F8042DBFF34F8FBFF36F8F10BD00BF36
:10928000945B0020204B1B681BB1204B01221A600D
:1092900070471E4B00221A601D4B1B68B3FA83F304
:1092A000DBB2C3F11F0303EB83018A0019498A581B
:1092B00042B94FF0500383F31188BFF36F8FBFF3B0
:1092C0004F8FFEE7134803EB83018A000244516885
:1092D0004968516003EB830C4FEA8C020832024468
:1092E000914209D003EB83039A000A4B13445B6855
:1092F000DA68094B1A607047486862469100054A6F
:109300000A445060EEE700BF945B0020A85B002099
:10931000B45B0020305C0020BC5C00200369C268A4
:10932000934204D881688A1A1344581E7047981AC9
:10933000013870472DE9F843044688461646C5684B
:109340008768A7EB0509914509D9406828440EF0C4
:1093500071FFBFF35F8F3544E560BDE8F883406877
:109360004A4628440EF066FFED1B35442A4608EBBA
:10937000090160680EF05EFFBFF35F8FE560ECE708
:109380002DE9F843064688461746C5684FF00009A0
:109390001AE05B1B5A1EB3685C1B944228BF14463C
:1093A000BC4228BF3C4670682246414628440EF025
:1093B00041FFA144A0443F1B2544B368AB420BD0FE
:1093C000BFF35F8FF5604FB133699D42E1D3B2685F
:1093D0005B1B1A44013ADEE70025F1E74846BDE889
:1093E000F883000010B5154CA822002120460EF08D
:1093F00021FE032323616361114AA261114BE361E2
:109400004FF4806323620023A3626362E3622266F7
:109410000D4A62661022A2662367E3666367BFF3A4
:109420005F8F06E0C3F10F020849895C034AD154FB
:1094300001330F2BF6D9BFF35F8F10BDD060002032
:10944000E8C40108D05C0020C05C0020F4C401081E
:10945000F8B50F461646451C05EB4505164B03EBC4
:10946000C50500EB400003EBC003DC6A012C11D002
:10947000022C1CD014B100242046F8BD2846FFF76A
:109480004DFF8642F8D8324639462846FFF752FF4C
:109490003446F1E72846FFF741FF3446864228BFAD
:1094A0000446224639462846FFF744FFE4E72846AB
:1094B000FFF766FF0446DFE7D0600020F8B50446FA
:1094C0000D461646094B1B786BB1EFF311874FF031
:1094D000200181F31188324629462046FFF7B8FF64
:1094E00087F31188F8BDFFF77DFFEEE7D06000201D
:1094F00008B5FFF777FF08BD10B504468268531C16
:109500004068834205D820688154A360E368013332
:10951000E360A26863689A4200D010BD21682069A8
:10952000FFF7CCFFA368984203D04FF0FF33E3600E
:10953000F3E70023A360F0E72DE9F84F81460F46DB
:1095400015461E46DDF828A00B9A0B464FF0010881
:1095500003E0B3FBF5F308F10108AB42F9D2B045E3
:1095600000D2B04612F0010B18D1BAF1000F15D09D
:1095700012F0020F02D0BEB1202400E02024BAF184
:10958000000F0BD0C24509D90AF1FF3A21464846DF
:10959000FFF7B2FFD9F80C30002BF0DAD9F80C3015
:1095A000002B25DB012404E03024E8E7013E05FB25
:1095B00004F4012EFAD8B7FBF4F39D42F7D900E08A
:1095C0001C46B7FBF4F304FB1377124AD15C484600
:1095D000FFF792FFD9F80C30002B03DBB4FBF5F357
:1095E000AC42EDD2BBF1000F02D0BAF1000F01D1B5
:1095F000BDE8F88FBAF1000FFAD0C245F8D90AF1E8
:10960000FF3A20214846FFF777FFD9F80C30002BAE
:10961000F0DAEDE708C501082DE9F04782B007460A
:109620008846154699460A9EDDF82CA081EAE17C21
:10963000ACEBE17C012402E09CFBF5FC01346545C8
:10964000FADD4C4500D24C4636B1B8F1000F02DBD2
:109650001AF0040F00D0013E1AF0020F02D0B9F147
:10966000000F03D01AF0010F00D1AEB9FB68002B38
:109670000FDBB8F1000F1CDB1AF0040F20D1FB68E0
:10968000002B06DB0AF00303022B1ED0FB68002B25
:109690002DDA02B0BDE8F087002EE7D0A642E5D96A
:1096A000013E20213846FFF727FFFB68002BF3DA45
:1096B000DCE7C8F100082D213846FFF71DFFDEE783
:1096C0002B213846FFF718FFD9E7B9F1000FDDD19C
:1096D000002EDBD0002ED9D0A642D7D9013E3021B2
:1096E0003846FFF709FFFB68002BF3DACEE7CDF829
:1096F00004A000964B462A4641463846FFF71CFF19
:10970000C7E70000F0B599B006460C46154603AB16
:1097100013934023149300231593179016938BE013
:109720000020012211E040F0010001340CE040F083
:109730000200013408E040F00400013404E040F08D
:109740000800013400E0002212B32378233B0D2BE4
:10975000F9D801A151F823F03F9700084797000876
:109760004797000847970008479700084797000861
:109770004797000847970008379700084797000861
:109780002797000847970008479700082F97000879
:109790002378A3F13001C9B2092907D8013402EBBB
:1097A000820203EB4203A3F13002F1E72E2B02D039
:1097B0000023217814E00134002306E0013403EB98
:1097C000830301EB4301A1F130032178A1F1300CB7
:1097D0005FFA8CFCBCF1090FF0D9EAE714F8011F1D
:1097E0006C29FBD06829F9D025296DD020D37829A0
:1097F0001ED858291CD35839202919D8DFE801F080
:109800003D181818181818181818181127181818AB
:10981000181818181818181857181848183218183F
:109820003D002B681A1D2A60197813A8FFF764FE03
:109830000134169B002B4CDB14F8011B002948D087
:1098400025293FF46DAF13A8FFF756FEF1E729680D
:109850000F1D2F600968019000920A2213A8FFF7DC
:10986000DBFEE5E729680F1D2F6009680190009273
:109870000A2213A8FFF760FEDAE729680F1D2F60A0
:10988000096801900092102213A8FFF755FECFE758
:109890002B681A1D2A601F6817F8011B0029C7D002
:1098A00013A8FFF729FE169B002BF5DAC0E72B68FB
:1098B0001A1D2A60196800230193082300931022BF
:1098C00013A8FFF739FEB3E7252113A8FFF714FE0D
:1098D000AEE7169B002B05DD159A32B9169B159A3B
:1098E00013441693169819B0F0BD03A93046FFF73C
:1098F000E5FDF3E70EB400B582B003AB53F8041BEB
:10990000019301AAFFF7FEFE02B05DF804EB03B07D
:109910007047000000B585B00023009301930293C7
:1099200003931548154A02604FF400324260836089
:109930000361037680F82030C362114A8262C360FB
:109940000122C26180F830304261F7F7DBFB68B971
:1099500010230093012301930023029369460648D4
:10996000F7F7FCFB28B905B05DF804FB00F044FCF8
:10997000EEE700F041FCF6E7D8610020002001404E
:109980000100000F0268184B9A4200D0704710B5D2
:1099900082B0044600230193144A516C41F4807153
:1099A0005164526C02F480720192019A1048114A7B
:1099B000026043608360C3604FF4806202614FF4D1
:1099C000006242614FF400528261C36103624362EC
:1099D000F8F7C2F920B9064BA3639C6302B010BD2F
:1099E00000F00AFCF7E700BF002001400038024009
:1099F000786100207064024008B50E480E4B036089
:109A00000323436000238360C3604FF4102202618C
:109A10004FF4001242610376437683760122C276C8
:109A200003774277F7F764FC00B908BD00F0E4FB68
:109A3000FBE700BF4C6200200064004008B50E4800
:109A40000E4B03600323436000238360C3604FF425
:109A5000102202614FF4001242610376437683764E
:109A60000122C27603774277F7F742FC00B908BDBE
:109A700000F0C2FBFBE700BF24620020006800404A
:109A800010B58AB0002305930693079308930993B2
:109A90000368454A934204D0444A93423CD00AB0FA
:109AA00010BD434A136801331360012B27D00024F3
:109AB0000194404B1A6B42F008021A631B6B03F0CF
:109AC00008030193019B0323059302220692089346
:109AD0000923099305A93848F8F740FC22460521D7
:109AE0001420F8F74DF81420F8F75AF8224605210B
:109AF0001520F8F745F81520F8F752F8CFE70023BE
:109B000000932C4B1A6C42F000721A641B6C03F029
:109B100000730093009BCAE700230293254B1A6C45
:109B200042F080621A641B6C03F080630293029B14
:109B30001F4A136801331360012B28D000240494BA
:109B40001C4B1A6B42F002021A631B6B03F00203F8
:109B50000493049B60230593022306930323089335
:109B60000923099305A91548F8F7F8FB22460521B2
:109B70004020F8F705F84020F8F712F822460521B2
:109B80004120F7F7FDFF4120F8F70AF887E70023A7
:109B90000393084B1A6C42F000721A641B6C03F0BA
:109BA00000730393039BC9E7006400400068004012
:109BB0002062002000380240000C024000040240F5
:109BC00008B50548054B0360F7F7F8FF00B908BD75
:109BD00000F012FBFBE700BF74620020003002407F
:109BE0000268094B9A4200D0704782B0002301936B
:109BF000064B1A6B42F480521A631B6B03F48053BA
:109C00000193019B02B070470030024000380240CF
:109C100000B583B00023009301930C480C4B036004
:109C2000F7F7DBFF58B90023009301931022694630
:109C30000648F7F7E4FF28B903B05DF804FB00F02D
:109C4000DBFAF0E700F0D8FAF6E700BF7C6200200C
:109C50000074004000B589B000230393049305937A
:109C6000069307930268134B9A4202D009B05DF83D
:109C700004FB0021019103F5E2331A6C42F000521B
:109C80001A641A6C02F000520192019A02911A6B46
:109C900042F001021A631B6B03F001030293029B63
:109CA000202303930323049303A90348F8F756FBE7
:109CB000DCE700BF007400400000024010B582B035
:109CC000002400943A4B1A6B42F480021A631A6B18
:109CD00002F480020092009A01941A6B42F400127E
:109CE0001A631B6B03F400130193019B22460521A9
:109CF0000C20F7F745FF0C20F7F752FF224605210D
:109D00000D20F7F73DFF0D20F7F74AFF224605210A
:109D10000E20F7F735FF0E20F7F742FF2246052108
:109D20000F20F7F72DFF0F20F7F73AFF2246052106
:109D30002F20F7F725FF2F20F7F732FF22460521C6
:109D40003820F7F71DFF3820F7F72AFF22460521B4
:109D50003A20F7F715FF3A20F7F722FF22460521B0
:109D60003B20F7F70DFF3B20F7F71AFF22460521AE
:109D70003C20F7F705FF3C20F7F712FF22460521AC
:109D80004420F7F7FDFE4420F7F70AFF224605219D
:109D90004520F7F7F5FE4520F7F702FF224605219B
:109DA0004620F7F7EDFE4620F7F7FAFE02B010BDA9
:109DB0000038024008B501F057FB0120FEF782FB96
:109DC000FBE70000034B0360034B0B608023136031
:109DD000704700BF906400209062002010B588B0EA
:109DE0000DF1040C074C0FCCACE80F0094E8070011
:109DF0008CE80700002101A8FEF731FB024B186038
:109E000008B010BD00C40108F46400202DE9F0433F
:109E10008FB0002409940A940B940C940D94009430
:109E20005F4B1A6B42F002021A631A6B02F00202D5
:109E30000092009A01941A6B42F040021A631A6B66
:109E400002F040020192019A02941A6B42F0010260
:109E50001A631A6B02F001020292029A03941A6BBF
:109E600042F008021A631A6B02F008020392039A86
:109E700004941A6B42F004021A631A6B02F0040293
:109E80000492049A05941A6B42F480721A631A6B56
:109E900002F480720592059A06941A6B42F0200231
:109EA0001A631A6B02F020020692069A07941A6B44
:109EB00042F080021A631A6B02F080020792079A3E
:109EC00008941A6B42F010021A631B6B03F0100324
:109ED0000893089B334F224640213846F8F734FB5D
:109EE000314E012210213046F8F72EFBDFF8C080FA
:109EF000012211464046F8F727FB4023099301252C
:109F00000A950B940C9409A93846F8F727FA082308
:109F100009934FF40419CDF828900B9509A93846F8
:109F2000F8F71CFA09950A940B9509A93046F8F739
:109F300015FA102309930A950B9502270C9709A986
:109F40003046F8F70BFA30230993CDF828900B949C
:109F500009A91648F8F702FA09950A950B950C9786
:109F600009A94046F8F7FAF9224605210920F7F732
:109F700007FE0920F7F714FE224605210A20F7F70D
:109F8000FFFD0A20F7F70CFE224605211720F7F700
:109F9000F7FD1720F7F704FE0FB0BDE8F08300BF10
:109FA0000038024000180240000002400008024051
:109FB0000004024008B50B480B4B03600B4B436099
:109FC00000238360C3604FF4804202614361836178
:109FD000C3610362F8F7A4FC00B908BD00F00CF9F6
:109FE000FBE700BF0C66002000580040801A060006
:109FF00008B50B480B4B03600B4B43600023836099
:10A00000C3604FF48042026143618361C3610362B4
:10A01000F8F786FC00B908BD00F0EEF8FBE700BFDA
:10A02000B8650020005C0040801A06002DE9F04170
:10A030008AB0002305930693079308930993036856
:10A040005D4A934205D05D4A934269D00AB0BDE8AB
:10A05000F081044600250095594E336B43F02003F0
:10A060003363336B03F020030093009B03230593BA
:10A070001222069208930423099305A95148F8F780
:10A080006DF90195336C43F480033364336C03F44E
:10A0900080030193019B4C484C4B03604FF060637D
:10A0A00043608560C5604FF48063036145618561ED
:10A0B000C56105624562F7F74FFE58BB424BA3638B
:10A0C0009C634348434B03604FF06063436040230D
:10A0D00083600023C3604FF4806202614361836147
:10A0E000C36103624362F7F737FEB0B9384B63636D
:10A0F0009C63002205212120F7F742FD2120F7F77C
:10A100004FFD002205212220F7F73AFD2220F7F724
:10A1100047FD9BE700F070F8D0E700F06DF8E5E749
:10A1200000250295264C236B43F004032363236B25
:10A1300003F004030293029B0395236B43F0010396
:10A140002363236B03F001030393039B4FF400731A
:10A1500005934FF01208CDF81880032708970426BE
:10A16000099605A91C48F8F7F9F84FF48073059390
:10A17000CDF8188007950897099605A91748F8F7AC
:10A18000EDF80495236C43F400032364236C03F47B
:10A1900000030493049B2A4605214820F7F7F0FCAE
:10A1A0004820F7F7FDFC2A4605214920F7F7E8FC8F
:10A1B0004920F7F7F5FC49E700580040005C0040F3
:10A1C0000038024000140240586500204060024000
:10A1D000F8640020B860024000080240000002401D
:10A1E00008B50268034B9A4200D008BDF6F7CAFED4
:10A1F000FBE700BF0020004072B6FEE700B595B057
:10A200003022002108A80DF015FF002303930493CA
:10A210000593069307930193204A116C41F08051F6
:10A220001164126C02F080520192019A02931C4B4D
:10A230001A6842F480421A601B6803F48043029358
:10A24000029B012308934FF48033099302230E935A
:10A250004FF480020F9206221092A82211921293BC
:10A260000723139308A8FAF7BDF898B90F230393AF
:10A2700002230493002305934FF4A05306934FF455
:10A2800080530793052103A8FAF7FCFA20B915B00B
:10A290005DF804FBFFF7B0FFFFF7AEFF00380240A8
:10A2A0000070004000B583B0F6F752FEFFF7A6FF3E
:10A2B000FFF7ACFDFFF702FDFFF72CFBFFF79CFB60
:10A2C000FFF7BCFB00F09CF800F08CFD00F0E2FD15
:10A2D00000F026FF00F02EF800F054F800F0F2FC39
:10A2E00000F0CAFE00F002FF00F03AFF00F03CFE72
:10A2F000FFF760FEFFF77CFE00F0A6F8FFF760FCBA
:10A30000FFF786FC02F0E0FB064B0093064B074A82
:10A3100007490020FFF7EEFAFFF760FDFEF79AF815
:10A32000FEE700BF64C5010824C5010828C501086F
:10A3300030C5010808B50548054B0360FAF740FC35
:10A3400000B908BDFFF758FFFBE700BF60660020BB
:10A35000000806500268094B9A4200D0704782B04C
:10A3600000230193064B5A6B42F040025A635B6B29
:10A3700003F040030193019B02B0704700080650B0
:10A380000038024008B50A480A4B036000234360C6
:10A390007C22826040F67F42C26003614361836138
:10A3A000FAF776FC00B908BDFFF726FFFBE700BF10
:10A3B000706600200028004000B585B0002300939F
:10A3C00001930293039302680A4B9A4202D005B0AC
:10A3D0005DF804FB02230093074B03936846FAF7EA
:10A3E00045FB20B9054B0122C3F83C2EEFE7FFF7F0
:10A3F00003FFF7E70028004000031E00000047426B
:10A4000008B50F480F4B03604FF48273436000237D
:10A410008360C36002220261012242614FF4007234
:10A4200082611022C2610362436283620A23C362B3
:10A43000FAF70EFD00B908BDFFF7DEFEFBE700BF2F
:10A44000686800200030014008B50F480F4B0360DA
:10A450004FF48273436000238360C3600222026171
:10A46000012242614FF4007282613822C2610362AC
:10A47000436283620A23C362FAF7EAFC00B908BDAB
:10A48000FFF7BAFEFBE700BF10680020003800406D
:10A490002DE9F0438BB00446002305930693079300
:10A4A000089309930368774A934206D0764A934209
:10A4B00000F082800BB0BDE8F08300250095734B5F
:10A4C0005A6C42F480525A645A6C02F480520092E0
:10A4D000009A01951A6B42F002021A631A6B02F09D
:10A4E00002020192019A02951A6B42F001021A636C
:10A4F0001B6B03F001030293029B182305934FF09B
:10A500000209CDF818904FF00108CDF81C80032601
:10A5100008960527099705A95D48F7F71FFF8023CF
:10A520000593CDF81890CDF81C800896099705A9D9
:10A530005848F7F713FF5848584B03604FF0C06373
:10A5400043608560C5604FF4806303614561856148
:10A55000C5610562042343628662C5620563F7F73D
:10A56000FBFB18BB4C4BE3649C634D484D4B0360B5
:10A570004FF0C0634360402383600023C3604FF407
:10A580008062026143618361C36103624362F7F7E2
:10A59000E3FB70B9424BA3649C6300220521232096
:10A5A000F7F7EEFA2320F7F7FBFA83E7FFF724FE2D
:10A5B000D8E7FFF721FEEDE700250395334B1A6C32
:10A5C00042F480421A641A6C02F480420392039AA5
:10A5D00004951A6B42F002021A631B6B03F002032C
:10A5E0000493049B4FF460430593022306930326D0
:10A5F00008960523099305A92548F7F7AFFE2A48D1
:10A600002A4B036045608560C5604FF48063036139
:10A6100045618561C5610562042343628662C56246
:10A620000563F7F799FB30BB1F4BE3649C6320483D
:10A63000204B03600023436040228260C3604FF4DC
:10A640008062026143618361C361036204224262EA
:10A6500003228262C3620363F7F77EFB70B9144B77
:10A66000A3649C63002205212420F7F789FA2420A3
:10A67000F7F796FA1EE7FFF7BFFDD5E7FFF7BCFD3A
:10A68000EDE700BF003001400038004000380240D4
:10A690000004024000000240B06700201064024045
:10A6A0005067002058640240F06600205860024065
:10A6B000906600207060024010B582B000240094C3
:10A6C000114B5A6C42F480425A645A6C02F4804234
:10A6D0000092009A01941A6C42F080521A641B6C2A
:10A6E00003F080530193019B22460F216FF001007C
:10A6F000F7F746FA224606210420F7F741FA04202C
:10A70000F7F74EFA02B010BD0038024030B589B0FC
:10A71000044600230193214B1A6C42F480721A64A0
:10A720001B6C03F480730193019B02A903A8FAF741
:10A730007FF9069BCBB9FAF75BF90346184AA2FBEF
:10A7400003239B0C013B1748174A026040F2E73293
:10A75000C26043600023036183608361FAF7BAFF3C
:10A76000054630B1284609B030BDFAF741F943003B
:10A77000E4E70C48FAF744FE05460028F2D12D2004
:10A78000F7F70EFA0F2C01D90125EBE7002221463D
:10A790002D20F7F7F5F9054B1C60E3E70038024080
:10A7A00083DE1B43C068002000200040040000201E
:10A7B000FEE7FEE7FEE7FEE7FEE7704708B5F7F7BE
:10A7C000FDFC08BD08B50820F7F7C4FE08BD08B5B4
:10A7D0001020F7F7BFFE08BD08B50248F7F7B4FB35
:10A7E00008BD00BF346B002008B50248F7F7ACFB8A
:10A7F00008BD00BF5865002008B50248F7F7A4FB64
:10A8000008BD00BFF066002008B50248F7F79CFBC2
:10A8100008BD00BF9066002008B50248F7F744F86D
:10A8200008BD00BF4C62002008B50248F7F73CF8AD
:10A8300008BD00BF4C62002008B52020F7F78AFE53
:10A8400008BD000008B50248F8F734FE08BD00BF97
:10A850000C66002008B50248F8F7FCFE08BD00BFF2
:10A860000C66002008B50248FAF76EFC08BD00BF70
:10A870006868002008B50248FAF766FC08BD00BF0A
:10A880001068002008B50248FBF736FD08BD00BF80
:10A89000DC6C002008B50248FBF72EFD08BD00BFA8
:10A8A000986C002008B50348FAF7F3FD0248FAF760
:10A8B000F0FD08BD54690020C068002008B50248BA
:10A8C000F7F742FB08BD00BFF864002008B5024856
:10A8D000F7F73AFB08BD00BFB067002008B5024893
:10A8E000F7F732FB08BD00BFD46A002008B5024864
:10A8F000F7F72AFB08BD00BF5067002008B50248E3
:10A90000F7F722FB08BD00BF7861002008B50248B8
:10A91000F6F7CAFF08BD00BF2462002008B5024850
:10A92000F6F7C2FF08BD00BF2462002008B5024848
:10A93000F9F74AFA08BD00BF2482002008B5024892
:10A94000F7F702FB08BD00BF946B002008B5024872
:10A95000F7F7FAFA08BD00BF746A002008B502488C
:10A96000F7F7F2FA08BD00BFF46B002008B5024803
:10A97000FBF7C2FC08BD00BF546C002008B50248BC
:10A98000F8F798FD08BD00BFB865002008B502487B
:10A99000F8F760FE08BD00BFB865002001207047D1
:10A9A00008B50DF005FC162303604FF0FF3008BD1D
:10A9B00008B54FF0FF31FFF7F3FFFEE770B50C4627
:10A9C0001646002506E0AFF30080214601F8010B92
:10A9D00001350C46B542F6DB304670BD70B50C460D
:10A9E0001646002504E014F8010BAFF30080013592
:10A9F000B542F8DB304670BD4FF0FF3070474FF482
:10AA000000534B60002070470120704700207047C2
:10AA100010B503460C4A0D490D48006840B10C487A
:10AA200000680344521A934206D8094A136010BDC5
:10AA30000748084C0460F2E70DF0BAFB0C230360F2
:10AA40004FF0FF30F3E700BF00000220005000008D
:10AA500008690020D09E0020034AD2F8883043F4D1
:10AA60007003C2F88830704700ED00E000B587B091
:10AA700003682C4A934218D02B4A934224D02B4A85
:10AA800093422ED02A4A934238D02A4A934218D170
:10AA900000230593284B5A6C42F400325A645B6CD5
:10AAA00003F400330593059B0BE000230193224B35
:10AAB0005A6C42F001025A645B6C03F0010301938B
:10AAC000019B07B05DF804FB002302931A4B1A6C3C
:10AAD00042F004021A641B6C03F004030293029B0D
:10AAE000EFE700230393144B1A6C42F008021A6438
:10AAF0001B6C03F008030393039BE2E7002204921C
:10AB00000D4B596C41F0020159645B6C03F0020378
:10AB10000493049B0F212D20F7F732F82D20F7F72F
:10AB20003FF8CEE70000014000080040000C004064
:10AB300000040140004401400038024070B58CB070
:10AB400000230793089309930A930B930368514AD0
:10AB500093420DD0504A934222D0504A93423AD069
:10AB60004F4A934251D04F4A934279D00CB070BDB6
:10AB7000002301934C4B1A6B42F010021A631B6BBB
:10AB800003F010030193019B4FF4D4430793022376
:10AB9000089301230B9307A94448F7F7DFFBE5E788
:10ABA00000230293404B1A6B42F008021A631B6B9E
:10ABB00003F008030293029B4FF4804307930223A0
:10ABC00008930122099203220A920B9307A938489D
:10ABD000F7F7C4FBCAE700230393334B1A6B42F029
:10ABE00080021A631B6B03F080030393039B4FF4F3
:10ABF000E053079302230893012209920A930B93CF
:10AC000007A92C48F7F7AAFBB0E700240494264BC9
:10AC10001A6B42F480721A631A6B02F48072049207
:10AC2000049A05941A6B42F004021A631B6B03F03A
:10AC300004030593059BC02307930226089603256A
:10AC40000B9507A91C48F7F789FB40230793089643
:10AC500009940A940B9507A91848F7F77FFB85E735
:10AC600000230693104B1A6B42F020021A631B6BF1
:10AC700003F020030693069B4023079302230893C7
:10AC8000012209920A9303230B9307A90C48F7F7B3
:10AC900065FB6BE70000014000080040000C00402D
:10ACA000000401400044014000380240001002400E
:10ACB000000C0240001C024000200240000802403C
:10ACC0000014024010B596B000241294139414940A
:10ACD00015941094119409940A940B940C940D9467
:10ACE0000E940F942022214601A80DF0A3F93B48B1
:10ACF0003B4B0360A7234360846044F61F63C3603B
:10AD0000046144618461FAF7E5FC00284BD14FF4FB
:10AD10008053129312A93148FAF742FE002845D118
:10AD20002E48FAF72FFD002843D1002310931193EA
:10AD300010A92A48FAF744FF00283DD1602309935F
:10AD400000220A920B920C920D920E920F9209A978
:10AD50002248FAF7AAFD002831D1042209A91F4888
:10AD6000FAF7A3FD70BB082209A91C48FAF79DFD5C
:10AD700058BB0C2209A91948FAF797FD40BB0023DC
:10AD8000019302930393049305934FF400520692A8
:10AD9000089301A91148FAF759FFE0B90F48FFF7E6
:10ADA000CDFE16B010BDFFF727FAB0E7FFF724FA83
:10ADB000B6E7FFF721FAB8E7FFF71EFABEE7FFF79D
:10ADC0001BFACAE7FFF718FACDE7FFF715FAD0E745
:10ADD000FFF712FAD3E7FFF70FFADFE72C6A00203C
:10ADE0000000014000B58FB000230A930B930C9331
:10ADF0000D9308930993019302930393049305938E
:10AE0000069307932148224A0260A722426083608A
:10AE10004FF6FF72C26003618361FAF75BFC28BBE7
:10AE20004FF480530A930AA91848FAF7B9FD00BBFA
:10AE30001648FAF7A7FCF8B900230893099308A964
:10AE40001248FAF7BDFED0B96023019300230293A4
:10AE500003930593082201A90C48FAF726FD88B947
:10AE60000A48FFF76BFE0FB05DF804FBFFF7C4F96B
:10AE7000D6E7FFF7C1F9DBE7FFF7BEF9DCE7FFF73D
:10AE8000BBF9E1E7FFF7B8F9EAE700BFE4690020A2
:10AE90000008004000B58FB000230A930B930C9379
:10AEA0000D930893099301930293039304930593DD
:10AEB000069307932A482B4A0260436083604FF64B
:10AEC000FF72C26003618361FAF704FC002831D18C
:10AED0004FF480530A930AA92148FAF761FD60BB39
:10AEE0001F48FAF74FFC58BB00230893099308A9A1
:10AEF0001B48FAF765FE30BB6023019300220292E3
:10AF00000392059201A91648FAF7CFFCF0B9042282
:10AF10000DEB02011248FAF7C8FCD0B9082201A9CA
:10AF20000F48FAF7C2FCB8B90D48FFF707FE0FB09B
:10AF30005DF804FBFFF760F9CAE7FFF75DF9CFE7BB
:10AF4000FFF75AF9D0E7FFF757F9D5E7FFF754F9BC
:10AF5000DDE7FFF751F9E1E7FFF74EF9E4E700BF5E
:10AF60009C690020000C004010B596B0002412949B
:10AF70001394149415941094119409940A940B94B6
:10AF80000C940D940E940F942022214601A80DF0EC
:10AF900051F83748374B0360A7234360846044F679
:10AFA0001F63C360046144618461FAF793FB002866
:10AFB00046D14FF48053129312A92D48FAF7F0FCB2
:10AFC000002840D12A48FAF7B1FB00283ED10023DF
:10AFD0001093119310A92648FAF7F2FD002838D1F2
:10AFE000602309934FF4FA630A9300220B920C92A8
:10AFF0000D920E920F9209A91D48FAF727FC58BB33
:10B00000042209A91A48FAF721FC40BB082209A921
:10B010001748FAF71BFC28BB002301930293039304
:10B02000049305934FF400520692089301A9104827
:10B03000FAF70CFEC8B90E48FFF780FD16B010BD38
:10B04000FFF7DAF8B5E7FFF7D7F8BBE7FFF7D4F873
:10B05000BDE7FFF7D1F8C3E7FFF7CEF8D0E7FFF77A
:10B06000CBF8D3E7FFF7C8F8D6E7FFF7C5F8E2E774
:10B07000546900200004014000B589B00023019309
:10B080000293039304930593069307931548164A76
:10B090000260A7224260836041F28732C26003618E
:10B0A0008361FAF717FBA0B90E48FAF76BFB98B962
:10B0B00060230193002202920392059201A909489C
:10B0C000FAF7F3FB58B90748FFF738FD09B05DF808
:10B0D00004FBFFF791F8E7E7FFF78EF8E8E7FFF7E3
:10B0E0008BF8F0E70C6900200044014008B50A48DD
:10B0F0000A4B03604FF46123436000238360C36005
:10B1000003610C2242618361C361FAF703FF00B956
:10B1100008BDFFF771F8FBE7DC6C00200010014070
:10B1200008B50C480C4B03600C4B43604FF4805344
:10B1300083600023C3604FF4806202610C2242618D
:10B140008361C361FAF7E6FE00B908BDFFF754F862
:10B15000FBE700BF986C002000480040A08601007B
:10B1600008B50A480A4B03604FF4E13343600023FB
:10B170008360C36003610C2242618361C361FAF79B
:10B18000C9FE00B908BDFFF737F8FBE7546C002093
:10B19000001401402DE9F0418CB0044600230793D0
:10B1A000089309930A930B9303689D4A93420AD02C
:10B1B0009C4A934200F082809B4A934200F0C380F5
:10B1C0000CB0BDE8F08100250095984B5A6C42F018
:10B1D00010025A645A6C02F010020092009A019513
:10B1E0001A6B42F002021A631A6B02F00202019219
:10B1F000019A02951A6B42F001021A631B6B03F06D
:10B2000001030293029B802307934FF00208CDF8BD
:10B21000208003270A9707260B9607A98448F7F78B
:10B220009DF84FF400730793CDF8208009950A9795
:10B230000B9607A97F48F7F791F87F487F4B03608B
:10B240004FF00063436040238360C5604FF4806328
:10B25000036145618561C5614FF440330362456216
:10B26000F6F77AFD20BB744B63639C637448754B9F
:10B2700003604FF00063436000238360C3604FF4BA
:10B280008062026143618361C3614FF440320262B4
:10B290004362F6F761FD70B9694BA3639C630022BA
:10B2A00005212520F6F76CFC2520F6F779FC87E7C9
:10B2B000FEF7A2FFD7E7FEF79FFFEDE70025039516
:10B2C0005A4B1A6C42F480221A641A6C02F48022DF
:10B2D0000392039A04951A6B42F004021A631B6BE3
:10B2E00003F004030493049B4FF440630793022389
:10B2F000089303230A9307230B9307A95248F7F7F0
:10B300002DF85248524B03604FF000634360856054
:10B31000C5604FF48063036145618561C561056265
:10B320004562F6F719FD58B9484BA3639C630022A8
:10B3300005212720F6F724FC2720F6F731FC3FE70C
:10B34000FEF75AFFF0E700250595384B5A6C42F09E
:10B3500020025A645A6C02F020020592059A069562
:10B360001A6B42F040021A631B6B03F04003069312
:10B37000069B4FF4844307930223089303260A96FF
:10B3800008230B9307A93348F6F7E8FF3248334BFD
:10B3900003604FF0206343608560C5604FF48063B5
:10B3A000036145618561C5614FF400330362042385
:10B3B00043628662C5620563F6F7CEFC50BB264B3E
:10B3C000A3639C632648274B03604FF020634360D0
:10B3D000402383600023C3604FF4806202614361B5
:10B3E0008361C3614FF4003202620422426203228D
:10B3F0008262C3620363F6F7AFFC70B9184B6363F4
:10B400009C63002205214720F6F7BAFB4720F6F798
:10B41000C7FBD5E6FEF7F0FED1E7FEF7EDFEEDE760
:10B420000010014000480040001401400038024074
:10B430000004024000000240F46B0020B8640240A7
:10B44000946B00208864024000080240346B0020A6
:10B450002860024000180240D46A00204064024084
:10B46000746A0020A064024008B500220F49104809
:10B47000FCF70FFA70B90F490D48FCF721FA60B9D3
:10B480000D490B48FCF7C4F950B90948FCF732FAEA
:10B4900048B908BDFEF7B0FEEDE7FEF7ADFEEFE7F9
:10B4A000FEF7AAFEF1E7FEF7A7FEF2E7E0000020B4
:10B4B000206D00204C0000209800002000207047E4
:10B4C0000020704708B5034B1B680BB108889847EC
:10B4D000002008BD0080002038B50C46074D01460D
:10B4E0002846FCF7AEF92846FCF7B7F9044B1B6871
:10B4F0000BB120889847002038BD00BF206D002088
:10B50000FC7F002010B5064C002206492046FCF7BF
:10B510008AF905492046FCF794F9002010BD00BFC8
:10B52000206D0020FC6F0020FC770020024B18608B
:10B53000024B19600248704700800020FC7F002009
:10B54000FC77002030B589B0002303930493059362
:10B55000069307930368B3F1A04F01D009B030BD43
:10B5600000250195164C236B43F001032363236BE5
:10B5700003F001030193019B4FF4E0530393022373
:10B580000493032306930A23079303A90D48F6F7B0
:10B59000E5FE636B43F0800363630295636C43F4E1
:10B5A00080436364636C03F480430293029B2A46E6
:10B5B00005214320F6F7E4FA4320F6F7F1FACDE748
:10B5C000003802400000024008B500F2C441D0F843
:10B5D0000805FCF7A5F908BD08B501EBC10300EBB0
:10B5E0008303D3F88C22D0F80805FCF766FA08BD6F
:10B5F00008B501EBC10300EB8303DA6CD0F8080552
:10B60000FCF7BEFA08BD08B5D0F80805FCF700FA4B
:10B6100008BD10B50446C3683BB1022B01D101211E
:10B6200004E0FEF7E9FD012100E00021D4F808055F
:10B63000FCF7D4F9D4F80805FCF79EF910BD00001A
:10B6400010B50446D0F80805FCF7CBF92268D2F80B
:10B65000003E43F00103C2F8003E236A23B1034ACF
:10B66000136943F00603136110BD00BF00ED00E055
:10B6700008B5D0F80805FCF7BEF908BD08B5D0F844
:10B680000805FCF7EDF908BD08B5D0F80805FCF78A
:10B69000D0F908BD08B5D0F80805FCF7F8F908BDE1
:10B6A00008B5D0F80805FCF7F4F908BD02780AB12E
:10B6B0000020704710B503461548C0F80835C3F898
:10B6C000C8024FF0A0430360042343600222C2601B
:10B6D000002303618261C36103624362C362036347
:10B6E000F8F77EF880B90A4C80212046F8F774FEFE
:10B6F000402200212046F8F749FE80220121204601
:10B70000F8F744FE002010BDFEF776FDEBE700BF22
:10B7100024820020D0F8C83211F0800F08D101F047
:10B720007F0101EBC10103EB810393F87E027047B7
:10B7300001F07F0101EBC10103EB810393F83E00AF
:10B74000704708B5D0F8C802F8F76DFA08BD0000D8
:10B7500000487047048000207047032805D8DFE8C0
:10B7600000F005040205012070470320704708B56A
:10B77000D0F8C802F8F7CBF8FFF7EFFF08BD08B51F
:10B7800094461A466346D0F8C802F8F79FF9FFF7C7
:10B79000E4FF08BD08B5D0F8C802F8F7DCF9FFF7F8
:10B7A000DCFF08BD08B5D0F8C802F8F774FAFFF757
:10B7B000D4FF08BD08B5D0F8C802F8F7B0FAFFF713
:10B7C000CCFF08BD08B5D0F8C802F8F76BF9FFF751
:10B7D000C4FF08BD08B5D0F8C802F8F72DFAFFF786
:10B7E000BCFF08BD08B5D0F8C802F8F7EDF9FFF7BF
:10B7F000B4FF08BD12230B8000487047CC00002026
:10B8000004230B8000487047C800002000239342A7
:10B810001ED200B510E00CF1370C01F813C0000186
:10B820004FEA430C0CF1010C4FF0000E01F80CE054
:10B830000133DBB2934209D24FEA107CB0F1204FC2
:10B84000E9D20CF1300C01F813C0E8E75DF804FB15
:10B850007047000038B50B4BD3F8100AD3F8144AE0
:10B86000D3F8183AC01800D138BD074D0822294630
:10B87000FFF7CCFF042205F110012046FFF7C6FFB9
:10B88000F2E700BF0070FF1FAE00002008B51A23CA
:10B890000B80FFF7DFFF014808BD00BFAC000020B0
:10B8A00008B50A4628B905490548FCF76EFD034866
:10B8B00008BD02490248FCF768FDF8E73087002020
:10B8C00084C5010810B50A46034C21460348FCF71D
:10B8D0005CFD204610BD00BF3087002098C50108E0
:10B8E00008B50A4628B905490548FCF74EFD034846
:10B8F00008BD02490248FCF748FDF8E73087002000
:10B90000A8C5010808B50A4628B905490548FCF745
:10B910003CFD034808BD02490248FCF736FDF8E744
:10B9200030870020B4C50108DFF834D00D480E4937
:10B930000E4A002302E0D458C4500433C4188C4289
:10B94000F9D30B4A0B4C002301E013600432A242EE
:10B95000FBD3FFF781F80CF031FCFEF7A3FC704736
:10B960000000022000000020080D00206CE4010807
:10B97000080D0020D09E0020FEE700001A4BD3EDFA
:10B980000A7A1A4BC3ED007A9FED197AF4EEC77A62
:10B99000F1EE10FA05DD77EEC77A164BC3ED037AA8
:10B9A00070479FED137AF4EEC77AF1EE10FA0ED8D5
:10B9B0009FED117AF4EEC77AF1EE10FA07DB9FEDF6
:10B9C0000C7A77EEC77A0B4BC3ED037A70479FED85
:10B9D000087A77EEC77A9FED097A77EE877A054B7A
:10B9E000C3ED037A704700BF5889002030890020DA
:10B9F0002C70B4429C8A0020D48FB3C20000B443A0
:10BA0000084B1B6893F83B30042B03D80649074AC0
:10BA1000C2F80610042B03D9054A044BC3F80620CC
:10BA2000704700BF34890020000040414089002059
:10BA30000000C8410C4B1A7C0C4B9A700C4AD17810
:10BA40005971917899711279DA720A4A92F88020C4
:10BA50005A72094A1268B2F84420A3F80720074A2C
:10BA6000B2F904209A8170479C8A0020D89900205E
:10BA700040890020A889002034890020948A002071
:10BA800000B583B01A4B1B68B3F90830B3F5967F45
:10BA900002DC184B1B7893B90122164B1A70002058
:10BAA000154B1873154B1874154B1A70DA705870C3
:10BAB000144B0093144B154A1549FDF71BFF0C4B13
:10BAC0001B68DB7A012B02D003B05DF804FB094A46
:10BAD00013700B4A13700F4B5A6A074B1A60094BCD
:10BAE00000930D4B0D4A0E490020FDF703FFEBE7D5
:10BAF000908A002038890020848900209C8A0020B8
:10BB00004089002064C50108C4C50108C8C50108F2
:10BB1000D0C501085889002024C5010828C501089E
:10BB2000F0C5010838B5554B554A1A60554B1A688F
:10BB3000D2F8023007EE903AF5EE407AF1EE10FAC4
:10BB400035D1D2F8063007EE903AF5EE407AF1EEB4
:10BB500010FA2CD1D2F80A3007EE903AF5EE407A7E
:10BB6000F1EE10FA23D1D2F8123007EE903AF5EE4A
:10BB7000407AF1EE10FA1AD1D2F8163007EE903A68
:10BB8000F5EE407AF1EE10FA11D1D2F81A3007EE44
:10BB9000903AF5EE407AF1EE10FA08D13A4B0022D5
:10BBA00083F88020394A13680133136050E0374B23
:10BBB00000211960364B01211970304D324C294655
:10BBC000204604F0CDF9334B187094ED1E1AD4EDD5
:10BBD0001D0A94ED1C0A05F091FC2F4B93ED086AA9
:10BBE00095ED157ADFED2D6A27EE267ADFED2C5ADA
:10BBF000C7EE257A77EEC67A2A4BC3ED007AF4EECB
:10BC0000E67AF1EE10FA24DDDFED276A77EEE66AD8
:10BC1000214B93ED097A37EE267A244B83ED007A97
:10BC2000164A92ED167ADFED1D6A27EE667A9FEDD1
:10BC30001C6AC7EE066AC3ED016AB0EE007AF4EE44
:10BC4000C77AF1EE10FA13D80F4B012283F8802047
:10BC500038BD9FED177AF4EEC77AF1EE10FA04D5ED
:10BC6000DFED116A77EEA66AD2E7F0EE676ACFE7FA
:10BC7000054B002283F88020EAE700BF2C8A0020D1
:10BC80000000D041888A0020A8890020A4890020D3
:10BC9000A1890020A0890020588900200000344399
:10BCA000DB0F49409C8900200000B44384890020B8
:10BCB000000034C338B5734B1B68DA7A022A08D007
:10BCC000032A00F0C580012A09D16F4A0021917032
:10BCD00005E06E4A012111746D4A022111739A7AAE
:10BCE000032A37D06B4A1268D2F8021007EE901A76
:10BCF000F5EE407AF1EE10FA75D1D2F8061007EEA3
:10BD0000901AF5EE407AF1EE10FA6CD1D2F80A10E2
:10BD100007EE901AF5EE407AF1EE10FA63D1D2F800
:10BD2000121007EE901AF5EE407AF1EE10FA5AD1A1
:10BD3000D2F8161007EE901AF5EE407AF1EE10FAEE
:10BD400051D1D2F81A2007EE902AF5EE407AF1EEA2
:10BD500010FA48D1504A002182F880104C4C94EDE2
:10BD6000007AB3F9002007EE902AF8EEE77ADFEDCB
:10BD70004B6A67EEA67A37EE677A84ED007AD4EDE7
:10BD8000016AB3F9023007EE903AF8EEE77A9FEDD8
:10BD9000446A67EE867A76EEE77AC4ED017A414D21
:10BDA00095ED090A37EE400A03F0A4FBD5ED097AB8
:10BDB00077EE807AC4ED007A94ED017AF3EE097A99
:10BDC000B4EEE77AF1EE10FA01DBC4ED017A304B04
:10BDD00093ED017AFBEE087AB4EEE77AF1EE10FA11
:10BDE00001D8C3ED017A274B1B689B7A022B39D00F
:10BDF000244B1B68B3F9042007EE902AF8EEE77A8B
:10BE00009FED277A67EE877A204AC2ED007AB3F970
:10BE1000061007EE901AF8EEE77A67EE877AC2ED21
:10BE2000017AB3F9083013F1640F1EDA164A0121C2
:10BE3000D17013F5FA7F1CDA134B04225A701A4A98
:10BE4000114BC3F80620194B1B78012B15D038BDB8
:10BE50000E4A032111740E4A022111730A4A01216C
:10BE600091703CE7FFF75EFEC2E7074A0021D17000
:10BE7000DFE7054B00225A70E1E7034B01225A70BD
:10BE8000E5E700BF908A0020408900209C8A0020BE
:10BE900084890020888A0020A88900200AD7233BB3
:10BEA0006F12833A58890020000090413C8900209D
:10BEB00038B5904B19688B7C03F00102C3F3400046
:10BEC000121A8D4807EE902AF8EEE77AC0ED017A53
:10BED000C3F3C002C3F38003D21A07EE902AF8EE30
:10BEE000E77AC0ED007A854CD4ED007AB1F90C30D8
:10BEF00006EE903AF8EEE66ADFED815A86EEA57A14
:10BF0000F1EE006A27EE267A77EEC77AC4ED007A62
:10BF100094ED017AB1F90E3006EE103AB8EEC66A29
:10BF2000C6EE256AB1EE086A66EE866A37EE267AB4
:10BF300084ED017A734D95ED090A37EEC00A03F0DE
:10BF4000D9FAD5ED097A77EE807AC4ED007A94EDCE
:10BF5000017AF3EE097AB4EEE77AF1EE10FA01DB3A
:10BF6000C4ED017A654B93ED017AFBEE087AB4EEED
:10BF7000E77AF1EE10FA01D8C3ED017A624B0022A4
:10BF800083F880205B4B1B681A7C5AB15A7C4AB9F3
:10BF90005E4AD278012A0AD15C4A0121117004213B
:10BFA000517004E01A8A12B9584A002151705B7C22
:10BFB000002B45D0564B1B68D3F8022007EE902A81
:10BFC000F5EE407AF1EE10FA30D1D3F8062007EE04
:10BFD000902AF5EE407AF1EE10FA27D1D3F80A2034
:10BFE00007EE902AF5EE407AF1EE10FA1ED1D3F862
:10BFF000122007EE902AF5EE407AF1EE10FA15D1F4
:10C00000D3F8162007EE902AF5EE407AF1EE10FAFA
:10C010000CD1D3F81A3007EE903AF5EE407AF1EEF3
:10C0200010FA03D1394B00225A7009E0FFF77AFD6C
:10C03000354B93F88030012B2FD0344B00225A70AF
:10C040002C4B1B6893F8203013F0010F34D1294B8F
:10C050001B6893F8263013F0010F37D101224FF4FB
:10C0600080712C48F6F770FA224B1B6893F8212058
:10C0700012F0010F31D1254A00211170D1709B7F40
:10C0800013F0010F2ED1214B00221A71FFF7B8FCDB
:10C09000214B1B78012B29D038BD164B1B681B7C0C
:10C0A000002BCAD0194BDB78012BC6D1174B0122CC
:10C0B0001A7004225A70C3E707F078F90D4B1A681A
:10C0C00092F82030013382F82030C0E700224FF48C
:10C0D00080711048F6F738FAC6E70C4A0121117052
:10C0E000D170CCE7094B01221A71CFE7074B01222F
:10C0F0005A70D1E7908A00209C8A00208489002011
:10C100000000254458890020A8890020408900208B
:10C11000888A0020000802403C89002008B5864B30
:10C120001B68997901F00102C1F34001521A83485A
:10C1300007EE902AF8EEE77AC0ED017A9979C1F31B
:10C14000C002C1F38001521A07EE902AF8EEE77A96
:10C15000C0ED007A7A4AD2ED007AB3F9001006EE0B
:10C16000901AF8EEE66A9FED776A86EE867AF1EE2F
:10C17000006A27EE267A77EEC77AC2ED007AD2ED12
:10C18000017AB3F9021006EE901AF8EEE66A86EE2E
:10C19000867AF1EE086A27EE267A77EE877AC2ED84
:10C1A000017AB3EE097AF4EEC77AF1EE10FA01DB08
:10C1B00082ED017A624A92ED017AFBEE087AB4EEE2
:10C1C000E77AF1EE10FA01D8C2ED017A5E4A002159
:10C1D00082F880101A795AB15A794AB95B4AD278F2
:10C1E000012A0AD1594A012111700421517004E039
:10C1F0009A8812B9554A002151705B79002B45D0BD
:10C20000534B1B68D3F8022007EE902AF5EE407AD4
:10C21000F1EE10FA30D1D3F8062007EE902AF5EEB1
:10C22000407AF1EE10FA27D1D3F80A2007EE902ACF
:10C23000F5EE407AF1EE10FA1ED1D3F8122007EE97
:10C24000902AF5EE407AF1EE10FA15D1D3F81620C7
:10C2500007EE902AF5EE407AF1EE10FA0CD1D3F801
:10C260001A3007EE903AF5EE407AF1EE10FA03D16B
:10C27000364B00225A7009E0FFF754FC324B93F81A
:10C280008030012B2CD0314B00225A702A4B1B6876
:10C290001B7D13F0010F32D1274B1B689B7E13F0DF
:10C2A000010F34D101224FF480712A48F6F74CF97E
:10C2B000214B1B685A7D12F0010F2FD1234A002118
:10C2C0001170D1709B7C13F0010F2CD11F4B0022F9
:10C2D0001A71FFF795FB204B1B78012B27D008BD67
:10C2E000154B1B681B79002BCDD0184BDB78012B2D
:10C2F000C9D1164B01221A7004225A70C6E707F002
:10C3000055F80D4B1A68137D01331375C4E70022ED
:10C310004FF480710F48F6F717F9C9E70B4A01216E
:10C320001170D170CEE7094B01221A71D1E7074B8A
:10C3300001225A70D3E700BF8C8A00209C8A00201B
:10C340008489002000002544A8890020408900201D
:10C35000888A0020000802403C89002008B519485E
:10C3600007F07EFF184B186005F0D8F8174B1860DF
:10C37000174807F053FE174B18601749174806F087
:10C38000F9FF174B18600D21164805F041F9164BBF
:10C3900018602C21154805F06BF9154B1860102119
:10C3A000144805F035F9144B18600121134805F0C5
:10C3B0005FF9134B1860134B00225A60124B012295
:10C3C0001A7008BD986C0020908A0020888A00208E
:10C3D000DC6C00208C8A0020D8990020546C00204E
:10C3E0003489002018C601089889002024C6010855
:10C3F0009489002030C60108548900203CC60108F9
:10C4000050890020848900203889002010B53449E3
:10C41000002005F04EF93349334B186805F049F90F
:10C420003249334B186805F044F9FFF703FBFFF777
:10C43000A5FAFFF725FB2F4B1B787BB12E4B1A6813
:10C44000937A023BDBB2012B41D9538940F201328E
:10C4500093423FD040F2011293423ED0274C2368D2
:10C460001878B0FA80F0400905F030F82368B3F886
:10C470004410234AA2F81510B3F84F10A2F8171071
:10C48000B3F851101F4A5181B3F842109181B3F8AB
:10C490004010D18193F8463013F0020F02D1184AB0
:10C4A0000021117413F0010F02D1174B00221A73EF
:10C4B0001349002005F014F91249144B186805F0CF
:10C4C0000FF91149124B186805F00AF910BDFFF772
:10C4D000F1FBC3E7FFF7ECFCC0E7FFF71FFEBDE78A
:10C4E000948A00203C89002050890020588900202F
:10C4F0009489002038890020908A00203489002007
:10C500009C8A0020408900208489002054890020D2
:10C51000988900202DE9F04F2DED028BDDB004F05D
:10C520002FFD05464A4B18604FF0B80B5A460021C4
:10C530000DEB0B000BF07EFD05F124032E9305F1AE
:10C5400008032F93434B3D93DFF85081CDF8F880DB
:10C55000414B3F93DFED418ACDED408A07268DF8B0
:10C5600008619FED3F8A8DED438A3E4B48933E4BD9
:10C570004A93DFF82CA1CDF82CA18DF83461CDF8C9
:10C5800038814FF004098DF84C9106278DF84D71D4
:10C5900001248DF850418DF851418DF85441334BB1
:10C5A000569357948DF86C415A46002168460BF01B
:10C5B00041FD05F1180300934D4401952C4B039365
:10C5C0002C4B0F932C4B1093CDED128A8DF85060AD
:10C5D0008DED158A4FF07E531A93284B1C93CDF89E
:10C5E00074A08DF87C60CDF880808DF894908DF8E3
:10C5F00095708DF896408DF897408DF898408DF89D
:10C6000099408DF89A408DF89C701D4B2893299481
:10C6100003232A938DF8B4400DEB0B0005F03EFA8E
:10C62000184B1860684605F039FA174B18602C2132
:10C63000164804F0EDFF164B18600D21154805F063
:10C6400017F8154B18605DB0BDEC028BBDE8F08F9C
:10C65000088B002000409C458FC2F53C00606A4674
:10C6600000401C46CDCC4C3F0AD7233D4C620020F5
:10C67000B88A00200080BB45000061440AD7A33C73
:10C6800024620020048B0020008B002024C60108B7
:10C69000FC8A002018C60108F88A00200000C84261
:10C6A0000000FA4370B5494C2146494B186805F023
:10C6B00000F8237B012B61D0022B37D06BB3454CA4
:10C6C0002368D3ED067AF1EE677A9FED437A87EE21
:10C6D000870ADFED427A20EE270A08F055F9DFEDF0
:10C6E000407A20EE270A3F4B83ED000A3E4DAC46D0
:10C6F00024680FCCACE80F000FCCACE80F0094E836
:10C7000003008CE80300394B1B685B68AB62294669
:10C71000374B186804F0E4FF70BD344B186805F01F
:10C72000B5F9344B186805F0B1F9C8E72F4D286802
:10C7300005F0B0F92F4C206805F0ACF90122042176
:10C74000286805F085F901220221286805F080F9A2
:10C7500001220421206805F07BF9012202212068D2
:10C7600005F076F9194E96ED000A286805F004FAEE
:10C7700096ED010A206805F0FFF9A0E71B4D286837
:10C7800005F088F91B4C206805F084F9012204218A
:10C79000286805F05DF901220221286805F058F9A2
:10C7A00001220421206805F053F9012202212068AA
:10C7B00005F04EF9054E96ED000A286805F0DCF903
:10C7C00096ED010A206805F0D7F978E7BC8A0020C9
:10C7D000F88A0020088B002000003443DB0F49401A
:10C7E00000409C45B88A0020CC8A0020048B0020A1
:10C7F000FC8A0020008B002000B583B004F0C0FB51
:10C80000174B0093174B184A18490020FDF772F890
:10C810000EE0134B0193164B0093164B164A174923
:10C820000020FDF767F804F0A1FE0120FBF74AFEA7
:10C8300000F01AFE124C84ED000A04F043FD00F0F3
:10C8400013FED4ED007A30EE670A094B83ED000A3F
:10C85000F7EE007AB4EEE70AF1EE10FAD9DCE2E77F
:10C8600064C5010824C5010828C5010848C6010897
:10C87000248B0020C4C50108C8C501086CC6010886
:10C88000288B002000B583B0164B0093164B174A37
:10C8900017490020FDF72EF80CE0124B0193154BC1
:10C8A0000093154B154A16490020FDF723F8012087
:10C8B000FBF708FE00F0D8FD124C84ED000A05F0ED
:10C8C000E5FC00F0D1FDD4ED007A30EE670A094BAB
:10C8D00083ED000AF7EE007AB4EEE70AF1EE10FA03
:10C8E000DBDCE4E764C5010824C5010828C50108AC
:10C8F000A4C601081C8B0020C4C50108C8C50108D6
:10C90000CCC60108208B002000B583B001F030F8C0
:10C91000174B0093174B184A18490020FCF7EAFF01
:10C920000CE0134B0193164B0093164B164A174914
:10C930000020FCF7DFFF0A20FBF7C4FD00F094FDA8
:10C94000134C84ED000A03F079FB01F02FF800F09E
:10C950008BFDD4ED007A30EE670A094B83ED000AB7
:10C96000F2EE047AB4EEE70AF1EE10FAD9DCE2E76F
:10C9700064C5010824C5010828C5010808C70108C5
:10C98000148B0020C4C50108C8C5010830C70108C0
:10C99000188B002000B583B00C4D0D4C0D4E009649
:10C9A0002B4622460C490020FCF7A4FF06F0FEFCB3
:10C9B00000962B46224609490020FCF79BFF06F013
:10C9C000E9FC0120FBF77EFDF9E700BF24C5010863
:10C9D00028C5010864C501086CC7010890C7010893
:10C9E00008B5A82000F054FC00F0BCFD08BD000014
:10C9F00010B5A4B02E4C0DF1740CA646BEE80F0085
:10CA0000ACE80F009EE807008CE8070000211DA895
:10CA1000FBF725FD274B18600DF1580C04F11C0E97
:10CA2000BEE80F00ACE80F009EE807008CE80700A6
:10CA3000002116A8FBF713FD1F4B18600DF13C0CED
:10CA400004F1380EBEE80F00ACE80F009EE80700C6
:10CA50008CE8070000210FA8FBF701FD174B1860B9
:10CA60000DF1200C04F1540EBEE80F00ACE80F00ED
:10CA70009EE807008CE80700002108A8FBF7EFFC00
:10CA80000F4B18600DF1040E04F1700CBCE80F00A0
:10CA9000AEE80F009CE807008EE80700002101A81F
:10CAA000FBF7DDFC074B186005F014FB24B010BD4C
:10CAB0001CC401083C8B0020348B0020308B0020EC
:10CAC000388B00202C8B002008B572B6FFF788FF4A
:10CAD000FFF744FCFFF71EFD00F04EF8FFF788FF5C
:10CAE00062B608BD08B5FFF791FCFFF7DBFD00F06B
:10CAF0001DF908BD00B583B0164B0093164B174ABD
:10CB000017490020FCF7F6FE0CE0124B0193154B81
:10CB10000093154B154A16490020FCF7EBFE012047
:10CB2000FBF7D0FC00F0A0FC124C84ED000AFFF7EC
:10CB3000D9FF00F099FCD4ED007A30EE670A094B7A
:10CB400083ED000AF7EE007AB4EEE70AF1EE10FA90
:10CB5000DBDCE4E764C5010824C5010828C5010839
:10CB6000DCC701080C8B0020C4C50108C8C501083A
:10CB700008C80108108B00202DE9F041E2B04FF009
:10CB8000B8084246002134A80BF054FA384B3B93C6
:10CB900001248DF8F440374E3E964FF07F52439279
:10CBA000354A449246938DF82041499602258DF8E6
:10CBB00064518DF865518DF86C51304B5C935D95E7
:10CBC00034A804F06BFF2E4B186003275D978DF897
:10CBD000664134A804F062FF2A4B186042460021E7
:10CBE00006A80BF027FA284B0D938DF83C401093C4
:10CBF0004FF08042159218968DF868401B93234A97
:10CC00002092234A219223938DF8AC5006238DF86D
:10CC1000AD308DF8B4701F4B2E932F9506A804F0FD
:10CC20003DFF1D4B186021461C4804F0F1FC1C4BD5
:10CC3000186010211B4804F01BFD1B4B18600023DB
:10CC40008DF80C30194A0492059303A805F028FBCF
:10CC5000174B18606B46174A07CA83E80700184647
:10CC600005F01EFB144B186062B0BDE8F08100BFF8
:10CC700000606A4600401C46CDCC4C3E2462002039
:10CC80007C8B0020788B002000409C450000FA43FC
:10CC90000000C8424C620020748B00203CC6010892
:10CCA000688B002030C60108548B00205469002096
:10CCB000708B0020A8C401086C8B002008B500F020
:10CCC000D3FB144B83ED000A134BD3ED007A30EE07
:10CCD000670ADFED127AB4EEE70AF1EE10FA03D438
:10CCE0000F4B5B78042B00D008BD0E4B1B68B3F9CB
:10CCF0000C30002BB8BF5B429BB242F21B529342F6
:10CD000002D9094B01221A7000F0AEFB024B83EDF1
:10CD1000000AE9E7448B0020408B002000004843D4
:10CD2000588B0020748B0020508B002010B52DED07
:10CD3000028B6D4C21466D4B186804F0BAFC2378C9
:10CD400003BB6B4B186804F0A5FE694B186804F030
:10CD5000A1FE684B93ED008A674BD3ED007A38EE65
:10CD6000278A00F081FBB4EEC08AF1EE10FA3EDCB7
:10CD70005D4B5B78042B00F29B80DFE803F00883B7
:10CD80003B5269005A4B186804F084FEDDE7584CAA
:10CD90000221206804F0EEFE9FED580A206804F09E
:10CDA000EBFE514BDB78012B00F083809FED538A23
:10CDB000B0EE480A524B186804F0DEFEB0EE480AA6
:10CDC000504B186804F0D8FE4FF47A714E4B186837
:10CDD00005F0A2FA4FF47A714C4B186805F09CFAF2
:10CDE000FFF76CFF4A494B4B186804F079FCBDEC27
:10CDF000028B10BD3E4C0421206804F0BBFE20686D
:10CE000090ED040ADFED447A30EE670A04F0B4FED8
:10CE100000F02AFB374B83ED000A374B3F4A1A607C
:10CE2000BFE7334C0421206804F0A4FE206890ED95
:10CE3000040ADFED3B7A30EE670A04F09DFE00F055
:10CE400013FB2C4B83ED000A2B4B364A1A60A8E7E4
:10CE5000274C0221206804F08DFE234BD3F80630C6
:10CE600007EE903A9FED307A67EE877A9FED2F7A42
:10CE700067EE877AB4EE000A20EE670A206804F0B5
:10CE80007BFE8EE71A4C0221206804F073FE9FEDB2
:10CE9000280A206804F070FE00F0E6FA154B83EDD6
:10CEA000000A154B234A1A60194B00221A7078E7C2
:10CEB000FEE79FED218AB0EE480A114B186804F096
:10CEC0005BFEB0EE480A0F4B186804F055FE4FF4B5
:10CED000FA610D4B186805F035FA4FF4FA610B4B07
:10CEE000186805F02FFA7BE7588B0020548B002040
:10CEF000748B00204C8B0020488B00200000000029
:10CF00007C8B0020788B0020708B00206C8B0020A5
:10CF1000508B0020688B00200080CA44000016431C
:10CF200000E0974500007A440000B443000010423E
:10CF300000804A460000C8420058184710B50C4C03
:10CF40002046F4F717FB02212046F4F790FC10214D
:10CF50002046F4F78CFC074C2046F4F70BFB02212B
:10CF60002046F4F784FC10212046F4F780FC10BD25
:10CF70004C6200202462002000B58BB00123069390
:10CF800000230793C36913F0010F0CBF0123002393
:10CF900004930E230993436B5B01019302680B4BCF
:10CFA0009A420DD00A4A1378591C11700593012337
:10CFB000089369460068F4F741FA0BB05DF804FB8A
:10CFC000044A1378591C1170F0E700BF4C6200202E
:10CFD000FC000020A48B002070B582B005460E46F0
:10CFE00031462846F4F730FC48B36B46154A3146C3
:10CFF0002846F4F784FB002400E00134124B1B7830
:10D00000A342EDD9114B53F824301A68AA42F4D147
:10D010000C4A11685A6B9142EFD1D3F8392072B1A2
:10D02000084A126983F83820084D184669462C30A2
:10D030000BF000F955F82400D0F83930984702B0C9
:10D0400070BD00BF808B0020A58B0020A88B002026
:10D0500030B585B00446314B1B7873B12F4B93F834
:10D0600000C0BCF10F0F2FD92D4B00932D4B2E4A32
:10D070002E490020FCF73EFCF6E7FFF75FFF284B48
:10D0800000932B4B2B4A2C490020FCF733FCE5E79F
:10D0900001339C451AD9294A52F82320506BA168C4
:10D0A0008842F5D1116822689142F1D11C4B02935C
:10D0B00004F108030193231D00931A4B1A4A2049D7
:10D0C0000020FCF717FCF1E70023E2E741200AF01B
:10D0D000FBFB0546412200210AF0ACFF62686A6052
:10D0E0000023082129756B75AB75EB7523682B60E0
:10D0F000EA61A3686B63E368C5F839302369C5F852
:10D100003D302846FFF738FF044A1378591C117048
:10D110000A4A42F82350284605B030BDA58B0020AE
:10D1200064C50108C4C50108C8C50108A4C8010830
:10D1300024C5010828C501087CC80108A88B002067
:10D14000FCC8010810B52DED028B82B00446F0EE4C
:10D15000408A00F089F9B0EE408A2068F4F7B6FA08
:10D16000D8B900F081F930EE480AB4EEE80AF1EEE1
:10D1700010FAF2DD1A4B01931A4C236800931A4BF4
:10D180001A4A1B490020FCF7B5FB236801332360D2
:10D19000002002B0BDEC028B10BD00F065F930EE4E
:10D1A000480A144B83ED000A214651F8040B04F1A0
:10D1B000200304F12402F4F70BFA08B90120E8E790
:10D1C000074B0193074C23680093074B074A0A4912
:10D1D0000020FCF78FFB2368013323600020D8E791
:10D1E00064C50108A08B002048C901084CC901088A
:10D1F00054C901089C8B0020A4C901084B1EDBB256
:10D20000072B0AD900B583B0054B0093054B064A9E
:10D2100006490020FCF76EFBF6E74161704700BF4E
:10D2200064C50108C4C50108C8C50108CCC9010806
:10D2300008B50021FFF7D0FE08BD08B50121FFF7B2
:10D24000CBFE08BD0E4B1B78C3B982B00C4B01223C
:10D250001A700C4B5B680193019A0B4B1B689A4246
:10D2600003D20A4A136801331360064B5A68064B0F
:10D270001A60034B00221A7002B07047704700BF5B
:10D28000008C0020001000E0108C0020148C002086
:10D2900008B5124AD2F8FC3043F08073C2F8FC3073
:10D2A0000F4B002159601A6842F001021A600D4BC1
:10D2B00003FB00F00C4B18600C4BA3FB00239B09F5
:10D2C0000B4A13600B4BA3FB0030800C0A4B186019
:10D2D0000A4B1960FFF7B6FF08BD00BF00ED00E084
:10D2E000001000E040420F00208C0020D34D62105F
:10D2F0001C8C002083DE1B43188C0020148C002023
:10D3000000B52DED028B83B00D4B5B680193019B43
:10D3100002689B1A07EE903AF8EE677A094B93ED94
:10D32000007AB8EE477A87EE878A019B0360FFF7A1
:10D3300089FFB0EE480A03B0BDEC028B5DF804FB38
:10D34000001000E0208C00202DE9F04182B0294B34
:10D350005B680193FFF776FF274B1C680026650882
:10D36000E3071B1B65F10005DB186D411C1945F136
:10D370000005019BE41845F10005204B1C605D6031
:10D380001F4BD3F800804246334620462946F3F728
:10D3900003FC07461B4B1860596042463346204643
:10D3A0002946F3F7F9FB10461C461546164B1A6042
:10D3B0005C60DFF86480C8F80070144B1F683A4660
:10D3C00033462146F3F7E8FB80B2A8F8040000FBDF
:10D3D00007F7E81B64F100010D4B186059600D4B15
:10D3E0001A683346F3F7D8FBA8F8060002B0BDE888
:10D3F000F08100BF001000E0148C0020088C002099
:10D40000208C0020F88B0020F08B00201C8C00204A
:10D41000E88B0020188C0020248C002008B5FFF732
:10D4200093FF0E4B9A8807EE902AF8EEE77A9FED6D
:10D430000C7A67EE877A93ED007AB8EE470A30EE01
:10D44000270ADB8807EE903AF8EEE77A9FED057A37
:10D4500067EE877A30EE270A08BD00BF248C0020D3
:10D460006F12833ABD37863508B5FFF76DFF0B4A5B
:10D47000116893884FF47A7000FB013300EE103A84
:10D48000B8EE400AD38807EE903AF8EEE77A9FEDBF
:10D49000047A67EE877A30EE270A08BD248C0020D4
:10D4A0006F12833A0A4B5968094B5B685B1A094A49
:10D4B000D2ED007AF8EE677A67EE807A07EE103ADE
:10D4C000B8EE477AB4EEE77AF1EE10FAECD4704792
:10D4D000001000E0208C002008B5002300E001339C
:10D4E000074A12789A420AD9064A52F82320D1886C
:10D4F0008142F4D191680029F1D01046884708BDD7
:10D50000548C00202C8C0020002306E013690BB102
:10D510001046984710BD0133DBB20E4A12789A428A
:10D5200017D90D4A52F8232011688142F3D110B562
:10D53000446C11798C42E9D00133DBB2054A127890
:10D540009A42E7D9044A52F8232011688142F3D164
:10D55000EEE77047608C0020588C002008B5FFF77C
:10D56000D3FF08BD08B5FBF7C3FF08BD08B50368C6
:10D5700003F14042B2F5005F0FD903F13F4202F5DB
:10D580007F02B2F5806F17D9A3F14023A3F5803352
:10D59000B3F5006F10D9002008BDF7F729FA0E4B3C
:10D5A0009B68C3F382230D4AD35C1BB9012303FBA1
:10D5B00000F0F1E70223FAE7F7F72AFA064B9B6837
:10D5C000C3F38223054AD35C1BB9012303FB00F09C
:10D5D000E2E70223FAE700BF003802406CC5010809
:10D5E00008B5002301E00133DBB20C4A12789A42FD
:10D5F00013D90B4A52F8232011688142F3D190F8D5
:10D600001CE051684FEA910C012101FA0CF18E45A2
:10D61000E9D153690BB11046984708BDA48C00208E
:10D62000648C0020836801684A680132B3FBF2F31E
:10D6300007EE903AF8EE677A67EE807A0B68FCEEB8
:10D64000E77AC3ED0B7A836801684A680132B3FB5D
:10D65000F2F307EE903AF8EE677A27EE800ABCEE16
:10D66000C00A81ED030A7047436863B903681B6809
:10D67000D3ED0B7AF8EE677A27EE800ABCEEC00A8B
:10D6800083ED0D0A7047042B0ED0082B19D00368C8
:10D690001B68D3ED0B7AF8EE677A67EE807AFCEEC2
:10D6A000E77AC3ED107A704703681B68D3ED0B7AF5
:10D6B000F8EE677A67EE807AFCEEE77AC3ED0E7AD1
:10D6C000704703681B68D3ED0B7AF8EE677A67EE54
:10D6D000807AFCEEE77AC3ED0F7A704738B51C4BC1
:10D6E0001B780F2B00D9FEE705461C200AF0ECF84A
:10D6F00004460023036043608360C36003614361A9
:10D700008361286820606B686360AB68E360EB68E6
:10D7100023612B6963616B69A361FFF727FFA06039
:10D7200061682068F8F7CAF994ED030A2046FFF70C
:10D7300079FF94ED040A2046FFF796FF044A137818
:10D74000591C1170034A42F82340204638BD00BFDF
:10D75000A48C0020648C002010B5044690F80021B1
:10D760000146D0F80401F8F7B1FFD4F804319B6BFF
:10D770001A68136823F00803136010BD70B582B0F7
:10D78000214B1D78022D1DD9204B0093204B214A9F
:10D7900021490020FCF7AEF8F6E70133DBB29D42E9
:10D7A00013D91E4A52F82320D2F80411626891421C
:10D7B000F3D1164B0093164B164A19490020FCF77B
:10D7C00099F8F6E704460023E9E74FF486700AF07B
:10D7D0007BF806464FF4867200210AF02BFC636842
:10D7E000C6F80431237886F80031A368C6F80831FA
:10D7F0006A1C054B1A70094B43F825603046FFF749
:10D80000ABFF304602B070BDB48C002064C5010887
:10D81000C4C50108C8C5010810CA0108A88C0020A9
:10D8200048CA010808B5022B0AD0032B0DD0012BE2
:10D8300000D0FEE76423D0F80401F8F79AFB08BD96
:10D84000D0F80401F8F701FCF9E7D0F80401F8F783
:10D8500023FCF4E738B50C46002301E00133DBB2CA
:10D86000154A92F800C09C4525D91D46134A52F826
:10D870002320D2F804118142F0D1D2F808313BB113
:10D880009847224600210D4B53F825000AF0D2FBA1
:10D890000A4C54F8251091F80021D1F80401F8F74A
:10D8A00015FF54F82530D3F804319B6B1A681368C0
:10D8B00023F00803136038BDB48C0020A88C00202E
:10D8C00010B582B00246002401E00134E4B2124BEC
:10D8D0001B78A3421ED9114B53F82410D1F8040130
:10D8E0009042F2D191F80021F8F7F0FE0B4B53F87B
:10D8F0002430D3F804319B6B1A68136823F00803B3
:10D900001360074B01930094064B074A0749002018
:10D91000FBF7F0FF02B010BDB48C0020A88C0020F3
:10D9200064C5010848C901084CC9010884CA010836
:10D9300010B584B004AB03E90300FDF7F7FD064C16
:10D940002060064B0093064B064A07490020FBF770
:10D95000D1FF206804B010BDB88C002064C5010858
:10D9600024C5010828C50108CCCA01087047000079
:10D9700000B587B0002300930193029303930493AF
:10D980000593074B009308230193064B02936846C7
:10D99000FFF7A4FE044B186007B05DF804FB00BF5E
:10D9A000E46900206F12833AD08C002038B500243F
:10D9B00040E095ED000A284B1868FFF755FE2B79DB
:10D9C000062B0BD8DFE803F0040B121920272E00DA
:10D9D0009FED220A204B1868FFF724FE38BD9FED0B
:10D9E000200A1D4B1868FFF71DFEF7E79FED1D0A83
:10D9F000194B1868FFF716FEF0E79FED1B0A164B50
:10DA00001868FFF70FFEE9E79FED180A124B186838
:10DA1000FFF708FEE2E79FED160A0F4B1868FFF7C5
:10DA200001FEDBE79FED130A0B4B1868FFF7FAFDC9
:10DA3000D4E70134042CD1D80F4B53F824506B7920
:10DA4000042BF6D8AB79002BB3D19FED0C0A024B17
:10DA50001868FFF709FEECE7D08C00209D9DFA3A8C
:10DA6000934ADF3A32E5C63A41C8BB3A052FA73A96
:10DA700009F2943AFAA9843ABC8C00200000000014
:10DA8000F6EE007A60EE277A10EE103A074AA2EB23
:10DA9000630307EE103A67EE277A67EE277AB7EE50
:10DAA000080A30EE670A27EE000A7047865A375F89
:10DAB00010B52DED048B0446D0F8EC3093ED009AB0
:10DAC0005C4A82ED009A93ED018A5B4A82ED008AFE
:10DAD000D3ED028A594AC2ED008AD3ED039A584B1E
:10DAE000C3ED009A69EE097A28EE087A77EE877A14
:10DAF00028EEA87A77EE877A29EEA90A37EE800A0F
:10DB0000FFF7BEFF4F4B83ED000A00230BE0D4F874
:10DB1000EC2002EB8302D2ED007A60EE277AC2EDB0
:10DB2000007A0133DBB2032BF1D9474B93ED6F7AC7
:10DB300028EE077AD4F80021F6EE007A27EE277A4D
:10DB400082ED047A93ED6F7A28EE877AD4F800217B
:10DB500027EE277A82ED057A93ED6F7A29EE477AE0
:10DB6000D4F8002127EE277A82ED0A7A93ED6F7AB6
:10DB700029EE877AD4F8002127EE277A82ED0B7AF6
:10DB800093ED6F7A69EEC79AD4F8002169EEA79AEF
:10DB9000C2ED109A93ED6F7A29EE479AD4F80021DE
:10DBA00029EE279A82ED119A93ED6F7A68EE878AB3
:10DBB000D4F8002168EEA78AC2ED168A93ED6F7A39
:10DBC00028EE478AD4F8002128EE278A82ED178AAA
:10DBD000D4F8F820D2ED1C6A93ED747AC6EE877AF9
:10DBE000C2ED1C7AD4F8F820D2ED236A93ED747A52
:10DBF000C6EE877AC2ED237AD4F8F83093ED1C7A1A
:10DC0000DFED127AB4EEE77AF1EE10FA01DDC3ED42
:10DC10001C7AD4F8F83093ED237ADFED0C7AB4EE69
:10DC2000E77AF1EE10FA01DDC3ED237ABDEC048B47
:10DC300010BD00BFF48C0020F08C0020EC8C002084
:10DC4000E88C0020E48C0020A88D002000401C46B9
:10DC500038B504469022D0F8F81008480AF0EAFADD
:10DC600048252A46D4F81C1105480AF0E3FA2A464A
:10DC7000D4F80C1103480AF0DDFA38BD0001002089
:10DC8000608D0020188D00202DE9F84F044600F12A
:10DC9000780500F180073946284606F055FB84F8E0
:10DCA000C800B4F87830A4F8A830B4F85A30A4F812
:10DCB000AA3004F1580A04F1A80842465146284601
:10DCC00006F008FC84F8C800B4F8A830A4F8B03016
:10DCD000B4F88230A4F8B23004F1B0094A463946AB
:10DCE000404606F0F7FB84F8C800B4F89030A4F87A
:10DCF000A030B4F89230A4F8A23004F1A0052A466E
:10DD000004F19001484606F08FFD84F8C8004946AA
:10DD1000284606F07FFC84F8C800D4F8EC30D3ED38
:10DD2000007AC54AC2ED007A93ED016AC34A82EDDA
:10DD3000006AD3ED026AC24AC2ED006A93ED037A2B
:10DD4000C04B83ED007AB4F87830A4F8B8300123E2
:10DD5000A4F8BA3066EE075A27EEA65A75EEC55AF1
:10DD6000D4F82C3175EEA55AC3ED005A67EE865AE9
:10DD700026EE875A75EE855AD4F82C3175EEA55AE1
:10DD8000C3ED015A67EEA77A26EE066A77EEC67AE9
:10DD900066EEA66A77EEE67A27EE077AD4F82C319B
:10DDA00077EE877AC3ED027A002512E0D4F82C31A1
:10DDB00003EB850393ED000AB0EEC00A06F018FFEE
:10DDC00005F16002A04B03EB820383ED010A0135EC
:10DDD000EDB2022DEAD9B4F84830A4F8C0304FF0C3
:10DDE000010BA4F8C2B004F1B80504F1C006324634
:10DDF000294604F1480006F003FB84F8C800B4F893
:10DE0000C030A4F8A830A4F8AAB04246314648462B
:10DE100006F060FB84F8C800A4F8B8B0B4F8C030CD
:10DE2000A4F8BA302946304606F08EFA84F8C800C5
:10DE3000DFF828B25A464146284606F04BFB84F8E4
:10DE4000C8009BED027ADBED037AABF5E07BF6EEE2
:10DE5000006A67EEA66AB4EEE67AF1EE10FA02D531
:10DE600001228BF83821B4EEE77AF1EE10FA45DDA5
:10DE7000754B93F83831002B40D0734B93F8393100
:10DE8000DBB1714AD2F84031D2F84411013341F18B
:10DE90000001C2F84031C2F844116B4BD3F8402165
:10DEA000D3F84431332A73F100030CD30023664ABC
:10DEB00082F8383184F82C3046E0634B0020002192
:10DEC000C3E95001E9E7227B604D2B8803FB02F296
:10DED000D4F8EC10D4F8E8000AF0ACF9227B2B88D7
:10DEE00002FB03F303FB02F2D4F8FC10D4F8F800B1
:10DEF0000AF0A0F9012384F82C309AE0DFED546A8F
:10DF000067EEA66AB4EEE67AF1EE10FA0FDD4E4B3C
:10DF100093F838315BB137EEC77ADFED4E6A67EEC2
:10DF2000A67AC7EE276A484BC3ED676A04E0464B02
:10DF30004FF07E52C3F89C21434B00200021C3E9DF
:10DF40005001002384F82C30B4F85830A4F8A830DD
:10DF5000B4F88230A4F8AA3042463946504606F05A
:10DF6000B9FA84F8C80004F198073A464946404691
:10DF700006F0B0FA84F8C80000230EE0D4F81C21A3
:10DF800002EB8302D2ED007A2F4991ED677A67EEBA
:10DF9000877AC2ED007A0133DBB2B4F89820B4F886
:10DFA0009A1001FB02F29342E8DB042201E0013205
:10DFB000D2B2052A1DD80023022BF8D8D4F81C11A0
:10DFC00002EB4200184401EB8001D1ED007A02F12E
:10DFD0005C0C1D4800EB8C0090ED016ADFED1E6AC1
:10DFE00086EE267A67EE877AC1ED007A0133DBB2DE
:10DFF000E2E7B4F89830A4F8B8300123A4F8BA30B6
:10E000002A463146384606F065FA84F8C8000E4BB9
:10E0100093F83831002B50D1D4F8BC300022DA60AC
:10E0200004F13002294604F1380006F0FDFB84F8C3
:10E03000C800BDE8F88F00BF148D0020108D0020AF
:10E040000C8D0020088D0020A88D0020928F0020CC
:10E05000CDCCCC3D6666663FDA0FC93F688F0020A5
:10E060000133DBB2052BD7D8D4F8BC20990002EBE2
:10E07000830292ED007A1248D0ED6F7ADFED116ADB
:10E0800067EEA67AB4EEE77AF1EE10FA01DDC2EDA2
:10E09000007AD4F8BC200A4492ED007A0849D1ED08
:10E0A0006F7ADFED096A67EEA67AB4EEE77AF1EEF1
:10E0B00010FAD5D5C2ED007AD2E70423D2E700BF2B
:10E0C000A88D00200AD7233C0AD723BC10B52DED1C
:10E0D000048B0446D0F8EC3093ED009A39EE099A9F
:10E0E0002E4A82ED009A93ED018A38EE088A2C4A76
:10E0F00082ED008AD3ED029A79EEA99A294AC2EDFF
:10E10000009AD3ED038A78EEA88A274BC3ED008AE4
:10E11000827B264B1B8802FB03F3027B03FB02F28C
:10E120000021D0F80C0109F085FFD4F80C31F1EE94
:10E13000697AC3ED007AD4F80C31C3ED018AD4F8C2
:10E140000C31B1EE497A83ED027AD4F80C3183EDCB
:10E15000038AD4F80C3183ED068AD4F80C3183EDB0
:10E16000079AD4F80C31C3ED088AD4F80C31C3ED0A
:10E17000099AD4F80C3183ED0C9AD4F80C31B1EE35
:10E18000488A83ED0D8AD4F80C31C3ED0E7AD4F8A9
:10E190000C31C3ED0F8ABDEC048B10BD048D002043
:10E1A000008D0020FC8C0020F88C0020928F002035
:10E1B00038B504462F4B01221A7083ED6C0AC3ED6B
:10E1C0006D0A83ED6E1A2C4AC3F8CC21002283F825
:10E1D000382100200021C3E95001C3E95201F7EEC4
:10E1E000007AF4EEE71AF1EE10FA01DDF0EE671AAC
:10E1F000204DC5ED741A85ED642A03230022062103
:10E20000281D00F013FD05F5E4730122114605F504
:10E21000E07006F005FB002309E0164AD2F8EC2076
:10E2200002EB830204EB8301096811600133032BC5
:10E23000F3DD104C114BC4F8D030114BC4F8D4307E
:10E24000104BC4F8D830104BC4F8DC30012384F8EC
:10E250002E3084F82F3090252A460C49D4F804013A
:10E2600009F0E8FF2A460A49D4F8FC0009F0E2FF69
:10E2700038BD00BFA88D002077CC2B3251DC0008C0
:10E28000B1DA0008CDE0000889DC0008E8CA01081E
:10E290000001002010B52DED088BF0EE61AAB0EE64
:10E2A00042AAF0EE629A804C84ED6F3AD4ED587A2F
:10E2B00030EE670A84ED5B0AD4ED597A70EEE70A16
:10E2C000C4ED5C0AD4ED5A7A31EE671A84ED5D1A1A
:10E2D000F6EE007A20EE270A20EE039A734B83EDC8
:10E2E000009A60EEA70A20EE838A714B83ED008AC4
:10E2F00021EE271A61EE038A6E4BC3ED008A90224D
:10E300006D49D4F8040109F095FFD4F80431F1EE19
:10E31000497AC3ED017AD4F80431F1EE486AC3EDCD
:10E32000026AD4F80431B1EE687A83ED037AD4F846
:10E33000043183ED069AD4F80431C3ED088AD4F889
:10E340000431C3ED096AD4F8043183ED0C8AD4F8A2
:10E35000043183ED0D7AD4F8043183ED0F9AD4F8AB
:10E360000431C3ED128AD4F8043183ED138AD4F852
:10E370000431C3ED147AD4F84831D4F84C21134356
:10E3800005D1C4ED5EAA84ED5FAAC4ED609A464B48
:10E3900093ED5E7AD3ED645A27EE257A93ED6F6A9A
:10E3A00075EE866AC7EE267A66EE2AAA8AEEA67A05
:10E3B00077EE877AC3ED5E7A93ED5F5A25EE855A44
:10E3C00085EE267A26EE0AAA8AEE265A37EE057AD6
:10E3D00083ED5F7A93ED605A65EE855A85EEA60A65
:10E3E00026EE296AC6EE265A30EE250A83ED600A2B
:10E3F00067EEA77A27EE077A77EE877A20EE000A93
:10E4000037EE800AFFF73CFBB0EE408A2B4B83EDE2
:10E41000000A00230FE0244903F15E0201EB8202AF
:10E42000D2ED007A8A6802EB830268EE277AC2EDA9
:10E43000007A0133DBB2022BEDD91B4C94ED5B0A61
:10E4400020EE000AD4ED5C7A67EEA77A70EE277AA8
:10E4500094ED5D0A20EE000A37EE800AFFF710FB0C
:10E46000B7EE007AC7EE007AC4ED657AC7EE086AA7
:10E47000C4ED666A9FED127AF4EEC77AF1EE10FAF7
:10E4800024D5DFED107AF4EEE76AF1EE10FA1DDD27
:10E49000DFED0D7AF4EEE76AF1EE10FA16D50122FF
:10E4A00084F8392116E000BFA88D0020E08C002000
:10E4B000DC8C0020D88C0020E8CA0108D48C002015
:10E4C0009A99993ECDCC1441CDCC2441744B002275
:10E4D00083F83921724CD4ED6C7A94ED6F7AD4F8CC
:10E4E000183167EE877AC3ED007AD4ED6C7A94ED3B
:10E4F0006F7AD4F8183167EE877AC3ED077AD4EDD6
:10E500006C7A94ED6F7AD4F8183167EE877AC3EDA0
:10E510000E7AD4ED6C7A94ED6F7AD4F8183167EEF8
:10E52000877AC3ED157AD4ED6D7A94ED6F7AD4F8CD
:10E53000183167EE877AC3ED1C7AD4ED6D7A94EDCD
:10E540006F7AD4F8183167EE877AC3ED237AD4F85E
:10E550001C21D4F8B8311360D4F81C211361D4F80D
:10E560001C31D4F8B8211A62201D00F0E3FE636864
:10E57000D3ED008AC4ED548A93ED018A84ED558A67
:10E58000D3ED02AAC4ED56AA93ED03AA84ED57AACF
:10E590001A69C4F860215B69C4F864310023C4F8C7
:10E5A000683128EE8A0A68EE2A7A30EE270A28EEC9
:10E5B000A89A68EE080A79EE200A70EEA00AF7EE33
:10E5C00000BA70EEEB0A30EE000A06F069FB9FED30
:10E5D00035BA60EE0B9AC4ED6A9A28EE880A6AEEA4
:10E5E0008A7A30EE270A6AEE0A7A39EE279A39EEED
:10E5F000099A79EE6B0A30EE000A06F051FB20EE24
:10E600000B0A84ED690A28EE0A8A68EEAA8A38EEB7
:10E61000688AB8EE000A28EE000A06F015FB20EE24
:10E620000B0A84ED680AD4ED767A79EEE77A9FEDED
:10E630001E7AF4EEC77AF1EE10FA23DDB4F9D43184
:10E64000013BA4F8D431164BB3F9D42107EE902A3C
:10E65000F8EEE77A9FED157A67EE877A79EEA77A7A
:10E66000C3ED6B7AC3ED769AD3F84821D3F84C11F9
:10E67000013241F10001C3F84821C3F84C11BDEC4F
:10E68000088B10BD9FED0A7AF4EEC77AF1EE10FA0E
:10E69000D9D5034AB2F9D4310133A2F8D431D2E743
:10E6A000A88D0020E12E6542000034430000B443F1
:10E6B000000034C3D0ED017A90ED0D7AD0ED0E6AF2
:10E6C00037EE267AF6EE006A27EE267A67EE877A2C
:10E6D00090ED197A67EE877AC0ED137A7047D0ED26
:10E6E0000D7A90ED117A27EE877AB5EEC07AF1EEC9
:10E6F00010FA26DDF5EEC07AF1EE10FA1CDD90ED91
:10E70000087AB4EEE77AF1EE10FA1ADAD0ED076A79
:10E7100037EE266AB4EEE76AF1EE10FA0FDB90ED01
:10E72000136A76EEE77A37EE277AC7EE267A66EE38
:10E73000277AC0ED137A7047F1EE677ADFE700239E
:10E74000C3647047D0ED116A90ED137A36EE877A84
:10E750001F4B83ED007AD0ED107A76EEA77A90ED1C
:10E76000126A77EE867A1B4BC3ED007AF5EEC07A1B
:10E77000F1EE10FA28DD90ED036AB4EEE76AF1EEEF
:10E7800010FA0AD5D0ED0D7A66EEA76AF5EEC06AEA
:10E79000F1EE10FA01DD0023C364D0ED067AB4EE89
:10E7A000E77AF1EE10FA03DD0023C364C0ED117ABD
:10E7B000F1EE677AB4EEE77AF1EE10FA03D50023B2
:10E7C000C364C0ED117A7047F1EE677AD3E700BFFA
:10E7D0008C8F0020888F0020D0ED027A90ED0C7A8B
:10E7E000D0ED0B6A37EE667A67EE877AD0ED196A5C
:10E7F00087EEA67A80ED127A704790ED126AD0ED1E
:10E80000197A26EE276A90ED0A7A77EE877AC6EEB5
:10E81000276A90ED166A27EE067A87EE276A76EE6B
:10E82000867AC0ED127A704790ED146AD0ED197AAD
:10E8300026EE276A90ED097A77EE877AC6EE276A88
:10E8400090ED156A27EE067A87EE276A76EE867ACD
:10E85000C0ED147A704790ED147AD0ED037AB4EEDF
:10E86000E77AF1EE10FA01DDC0ED147A90ED147A3A
:10E87000F1EE677AB4EEE77AF1EE10FA01D5C0ED69
:10E88000147A704790ED147AB0EEC77AD0ED037A1F
:10E89000DFED1D6A67EEA67AB4EEE77AF1EE10FAC4
:10E8A0002BD4D0ED177AB0EEE77ADFED186AB4EE2C
:10E8B000E67AF1EE10FA20D4D0ED0B6A77EEE67A24
:10E8C000F0EEE77AC7EE876ADFED117AF4EEE76AD9
:10E8D000F1EE10FA12DD836EC26E013342F10002D6
:10E8E0008366C266816EC36E40F2F512914273F187
:10E8F000000302D3012380F8703070470022002308
:10E90000C0E91A23EEE700BF6F12833A17B7D13878
:10E910003333733F38B505460C467822002109F0A1
:10E9200089FB23462A462034D3F800E0D3F804C0FC
:10E930009868D968C2F800E0C2F804C09060D1605D
:10E9400010331032A342EFD1186859689B681060E9
:10E950005160936005F16000FEF7D2FC38BD10B540
:10E960002DED028B0446F0EE408AB0EE608A90F9FD
:10E970001430002B71DB04F16000FEF7C1FC84ED64
:10E98000190AC4ED0B8A84ED178A78EE680AC4ED83
:10E990000D0AF5EEC00AF1EE10FA61DDF0EE607AD4
:10E9A00094ED047AB4EEE77AF1EE10FA73D5D4ED73
:10E9B000007A60EEA77AC4ED107AD4ED017A60EEA9
:10E9C000A77A60EE277AC4ED137AD4ED027A94ED3B
:10E9D0000E7A70EEC70A67EEA07A87EE807A84ED31
:10E9E000127A237D13F0040F3DD1237D13F0200F05
:10E9F0003DD1237D13F0020F3DD1237D13F0400F55
:10EA00003DD1237D13F0010F3DD1D4ED117A94ED6A
:10EA1000137A77EE877AC4ED117A94ED107A77EE57
:10EA2000877A94ED127A77EE877AC4ED147A237D93
:10EA300013F0100F2BD12046FFF70DFFE36A23637D
:10EA400094ED140A84ED150AA36CA365636BA363AC
:10EA5000E36CE363BDEC028B10BDFFF713FF8AE7A5
:10EA6000F1EE607A9CE72046FFF724FEBDE72046E2
:10EA7000FFF735FEBDE72046FFF7AEFEBDE72046B7
:10EA8000FFF7BBFEBDE72046FFF75CFEBDE7204673
:10EA9000FFF7CAFECFE700232365E364CEE700005B
:10EAA000034690B14FF6FF7009E013F8012B424086
:10EAB000D2B2074931F8122082EA102061464A1E7C
:10EAC0001FFA82FC0029F0D170474FF6FF707047A3
:10EAD00090010020D8B138B50C460546022918D956
:10EAE000023989B2FFF7DCFF2B1913F8023CC2B2DE
:10EAF0009A4201D0002038BDC0F30F202B1913F823
:10EB0000013C984201D00020F5E70120F3E7002006
:10EB100070470020EFE7000070B50446002505743B
:10EB2000827B414E338803FB02F24168D0F8F40047
:10EB300009F080FBA27B338803FB02F22946606860
:10EB400009F078FAA27B338802FB03F303FB02F29D
:10EB50002946D4F8180109F06DFA227B338802FBAC
:10EB600003F3A27B03FB02F22946D4F80C0109F05F
:10EB700061FA294601E00131C9B2A37B8B422AD94F
:10EB8000D4F8F4304FEA810C03EB8102D2ED007A25
:10EB9000F5EE407AF1EE10FAEDD0227C03EB820321
:10EBA000C3ED007A626A237CD154A069D4F80C21A9
:10EBB00094F80CE0257C63695B5C05FB0E3303F184
:10EBC0008043013B02EB8302604403681360237CB3
:10EBD00001332374CFE700230FE0E069616A11F885
:10EBE00003C0D4F8181102FB033201EB820100EBE1
:10EBF0008C0002680A600133DBB2227C9A42ECD8B6
:10EC0000A4F87820237BA4F87A30A4F88030A4F804
:10EC10008220A4F89020A4F89220A4F89830A4F8B8
:10EC20009A20A4F8482070BD928F00202DE9F0476B
:10EC300004460D4691461E46DFF8B8830423A8F823
:10EC40000030EB4B08221A80017380F80D90867318
:10EC500000270774304608F037FE606132463946B7
:10EC600009F0E8F9B8F800A006FB0AFA504608F0E7
:10EC70002BFEA0615246394609F0DCF9B8F800A035
:10EC800006FB0AFA504608F01FFEE061524639467C
:10EC900009F0D0F9B8F800A005FB0AFA504608F0D0
:10ECA00013FE20625246394609F0C4F9304608F096
:10ECB0000BFE60623246394609F0BCF9B8F800A094
:10ECC00005FB0AFA504608F0FFFD2060524639461F
:10ECD00009F0B0F9B8F800A006FB0AFA504608F0AF
:10ECE000F3FD60605246394609F0A4F9B8F800A077
:10ECF00009FB0AFA504608F0E7FDA0605246394683
:10ED000009F098F9B8F800A005FB0AFA504608F097
:10ED1000DBFDC4F8E8005246394609F08BF9D4F817
:10ED2000E8300122217B04F1300005F079FDB8F8CC
:10ED3000008005FB08F8404608F0C6FDC4F8EC006A
:10ED40004246394609F076F9D4F8EC300122217BAD
:10ED500004F1380005F064FDB9F1000F40F04C817A
:10ED6000DFF89082B8F8007006FB07F7384608F025
:10ED7000ABFDC4F8F4003A46002109F05BF9D4F881
:10ED8000F4300122A17B04F1480005F049FDB8F8F8
:10ED9000007005FB07F705FB07F7384608F094FD00
:10EDA000C4F8F8003A46002109F044F9217BD4F870
:10EDB000F8300A4604F1500005F032FDB8F8007052
:10EDC00005FB07F705FB07F7384608F07DFDC4F89B
:10EDD000FC003A46002109F02DF9217BD4F8FC30E3
:10EDE0000A4604F1580005F01BFDB8F8007005FB59
:10EDF00007F705FB07F7384608F066FD8246C4F8BA
:10EE00000001384608F060FDC4F804013A460021CC
:10EE1000504609F00FF9B8F8002005FB02F205FB97
:10EE200002F20021D4F8040109F004F9217BD4F89E
:10EE300000310A4604F1600005F0F2FC217BD4F8B1
:10EE400004310A4604F1680005F0EAFCB9F1000F4C
:10EE500040F0E880674FB7F800A00AFB06F909FB0D
:10EE600005F9484608F030FD8046C4F80C010AFB5D
:10EE700005F006FB00F008F027FDC4F810014A4633
:10EE80000021404609F0D6F83A8805FB02F206FB5D
:10EE900002F20021D4F8100109F0CCF8D4F80C31BA
:10EEA000227BA17B04F1780005F0BAFCD4F8103184
:10EEB000A27B217B04F1800005F0B2FCB7F8008052
:10EEC00005FB08F808FB05F8404608F0FDFCC4F80F
:10EED00014014246002109F0ADF8217BD4F8143129
:10EEE0000A4604F1880005F09BFCB7F8008006FB99
:10EEF00008F808FB06F8404608F0E6FCC4F81801DC
:10EF00004246002109F096F8A17BD4F818310A4650
:10EF100004F1900005F084FC3B8805FB03F303FB40
:10EF200006F6304608F0D0FCC4F81C013246002139
:10EF300009F080F8D4F81C31A27B217B04F1980001
:10EF400005F06EFC94F80C803E8808FB06F606FB84
:10EF500008F5284608F0B8FC0746C4F82001284602
:10EF600008F0B2FCC4F82401284608F0ADFCC4F84F
:10EF70002801304608F0A8FCC4F82C01304608F0FF
:10EF8000A3FCC4F830013B464246414604F1A000D0
:10EF900005F046FC217BD4F824310A4604F1A80090
:10EFA00005F03EFC217BD4F828310A4604F1B0007C
:10EFB00005F036FCD4F82C310122217B04F1B80095
:10EFC00005F02EFCD4F830310122217B04F1C00081
:10EFD00005F026FC002384F8283084F8293084F8D2
:10EFE0002A3084F82B3084F82C30BDE8F08700BF3D
:10EFF000908F0020928F0020164B1F8809FB07F787
:10F00000384608F061FCC4F8F0003A46002109F0E7
:10F0100011F8D4F8F0300122617B04F1400005F0D2
:10F02000FFFB9DE6B8F8003005FB03F303FB09F98D
:10F03000484608F049FCC4F808014A46002108F097
:10F04000F9FFD4F80831627B217B04F1700005F0F0
:10F05000E7FBFFE6928F002038B50446C37B63B11F
:10F06000FFF75AFD627B0E4B1B8803FB02F2A1687F
:10F07000D4F8F00009F0DEF838BD827B084D2B880B
:10F0800003FB02F24168D0F8F40009F0D3F8A27B48
:10F090002B8803FB02F20021606808F0CBFFE1E758
:10F0A000928F002090F82830B3BB70B50446437BA4
:10F0B00043B3037BA0F8B8300126A0F8BA6000F192
:10F0C000B8052A4600F13001603005F003FA84F8F3
:10F0D000C800237BA4F8C030A4F8C26004F1C006C5
:10F0E000324604F1400104F1700005F0F3F984F8B0
:10F0F000C80004F138023146284605F095FB84F833
:10F10000C80070BD00F1380200F13001603005F038
:10F11000E1F984F8C800F4E77047F8B590F82930B1
:10F1200003B1F8BD044600F1600600F168073946F6
:10F13000304605F009F984F8C80004F158052A465C
:10F1400004F15001304605F0C5F984F8C800B4F860
:10F150005830A4F8A830B4F86A30A4F8AA3004F102
:10F16000A80632463946284605F0B4F984F8C800A6
:10F170002A4604F18801304605F056FB84F8C800A1
:10F18000CFE72DE9F84390F82A300BB1BDE8F883BA
:10F19000044600F1780600F180073946304605F054
:10F1A000D3F884F8C800B4F87830A4F8A830B4F8DC
:10F1B0005A30A4F8AA3004F1580804F1A8052A46E8
:10F1C0004146304605F086F984F8C800B4F8A83006
:10F1D000A4F8B030B4F88230A4F8B23004F1B0062C
:10F1E00032463946284605F075F984F8C800B4F867
:10F1F0009030A4F8A030B4F89230A4F8A23004F112
:10F20000A0094A4604F19001304605F00DFB84F850
:10F21000C8003146484605F0FDF984F8C800B4F846
:10F220005830A4F8A830B4F88230A4F8AA302A469E
:10F230003946404605F04EF984F8C80004F19802BA
:10F240003146284605F046F984F8C8009EE790F854
:10F250002B3003B170472DE9F0410446B0F8783007
:10F26000A0F8B8300126A0F8BA6000F1380700F124
:10F27000B8052A463946783005F02CF984F8C800DC
:10F28000B4F84830A4F8C030A4F8C26004F1C00853
:10F290004246294604F1480005F0B2F884F8C80057
:10F2A000B4F89830A4F8B830A4F8BA602A464146B9
:10F2B00004F1980005F00EF984F8C80004F130025A
:10F2C0002946384605F0B0FA84F8C800BDE8F08158
:10F2D000F8B590F82C3003B1F8BD0446B0F898307A
:10F2E000A0F8A830B0F87A20A0F8AA20A0F8B03092
:10F2F000B0F85A30A0F8B23000F1A8073A4600F151
:10F300007801983005F0E6F884F8C80004F1580553
:10F3100004F1B00632462946384605F0DBF884F899
:10F32000C80004F150023146284605F069F884F817
:10F33000C800D1E738B50446FFF78EFED4F8CC30CC
:10F340000BB1204698472046FFF7ACFED4F8D030EA
:10F350000BB1204698472046FFF7DFFED4F8D430A3
:10F360000BB120469847237C0BB9E37BCBB92046F1
:10F37000FFF707FFD4F8D8300BB120469847204656
:10F38000FFF765FFD4F8DC300BB1204698472046E4
:10F39000FFF79EFFD4F8E0300BB1204698470023DA
:10F3A00019E0227B204D2B8803FB02F2D4F8EC10ED
:10F3B000D4F8E80008F03EFF227B2B8802FB03F321
:10F3C00003FB02F2D4F8FC10D4F8F80008F032FF86
:10F3D000E0E70133DBB2227B9A4214D9D4F8F8106B
:10F3E00002FB033201EB820292ED007A216A01EB0B
:10F3F0008301D1ED007AB4EEE77AF1EE10FAE8D5A8
:10F40000C2ED007AE5E7084B1B8803FB02F2D4F853
:10F41000E810206808F00EFFD4F8E4300BB1204665
:10F420009847206838BD00BF928F0020F0EE405A08
:10F43000B5EEC00AF1EE10FA1ED9F6EE007A20EE13
:10F44000270A9FED0F6A25EE866A60EE007A77EE56
:10F45000E57A70EE006A87EEA67A30EE470AB4EEDF
:10F46000E76AF1EE10FAF0D4B1EE467AB4EEE77A3C
:10F47000F1EE10FAE9DC70479FED020A704700BF19
:10F480006F12833A00000000B4EEE00AF1EE10FAC9
:10F4900007D4B4EEC10AF1EE10FA04DDB0EE410A71
:10F4A0007047B0EE600A7047B4EEE01AF1EE10FA61
:10F4B0001ED4B4EEC01AF1EE10FA0AD571EE600A4D
:10F4C00001E030EE600AB4EEC10AF1EE10FAF8DCA9
:10F4D0007047F4EEC00AF1EE10FA09DD31EE601A61
:10F4E000B4EEE00AF1EE10FA02D530EE010AF7E7C9
:10F4F0007047000008B59FED031ADFED030AFFF720
:10F50000D3FF08BD00003443000034C3FDEEC07AD1
:10F510000C4BC3ED007AB8EEE77A30EE470A0A4B9F
:10F5200083ED000AB6EE007AB4EEC70AF1EE10FAE7
:10F5300004DD17EE903A0133024A1360014B18685C
:10F54000704700BF988F0020948F002010B52DEDDC
:10F55000048B044690ED009A69EE097AD0ED018A99
:10F5600028EEA87A77EE877A90ED028A28EE080ACC
:10F5700037EE800AFFF75AFFC9EE007AC4ED007A31
:10F58000C8EE807AC4ED017AC8EE007AC4ED027A42
:10F590002046BDEC048B10BDD0ED017A91ED027ACE
:10F5A00067EE877A90ED027AD1ED016A27EE267A2E
:10F5B00077EEC77AC2ED007AD0ED027A91ED007A4B
:10F5C00067EE877A90ED007AD1ED026A27EE267A0F
:10F5D00077EEC77AC2ED017AD0ED007A91ED017A2B
:10F5E00067EE877A90ED017AD1ED006A27EE267AF0
:10F5F00077EEC77AC2ED027A7047D0ED007A91EDCE
:10F60000007A67EE877A90ED017AD1ED016A27EEF4
:10F61000267A77EE877A90ED020A91ED027A20EE53
:10F62000070A37EE800A704731EE601A30EE600A42
:10F6300001238340013B07EE903AF8EEE77A20EE93
:10F64000270AC0EE017AFCEEE77A17EE903A98B2FC
:10F6500070470000000000002DE9F04F2DED068BF3
:10F6600085B00446D1ED0A7A91ED0C7A77EE877A6F
:10F67000C0ED1F7A90ED038AD0ED078A67EEA87A75
:10F6800038EE278A80ED038A90F82D30022B05D0C2
:10F69000032B00F00F8100250127CAE10025012D71
:10F6A00034DCD4ED038A07EE905AB8EEE78ADFED3A
:10F6B000D87A28EE278A78EE888AD4ED089A94EDD5
:10F6C000009AB0EE680A05F05FF920EE290A39EEDB
:10F6D000409AEE1C04EB061686ED009A94ED019A12
:10F6E000B0EE680A05F00AF920EE290A39EE409AD0
:10F6F00086ED019AA26804EB05139A63D4ED037AB0
:10F7000038EE278A83ED0F8A0135C8E7F0EE000A4C
:10F7100094ED0C0A05F0C6FAF0EE408AF0EE000A0D
:10F7200094ED0D0A05F0BEFA78EE808AF0EE000A3C
:10F7300094ED100A05F0B6FAB0EE408AF0EE000A39
:10F7400094ED110A05F0AEFA38EE008AF4EEC88A9C
:10F75000F1EE10FA00F3A382002572E218EE100A0F
:10F76000F0F79AFE06460F462846F0F783FEA6A35A
:10F77000D3E90023F0F7E8FE02460B46304639464F
:10F78000F0F72CFDF1F7B8F9834644E0666A46E0ED
:10F79000D4ED027A94ED0A7A77EE877A04EB0518B5
:10F7A000C8ED0E7A18EE100AF0F776FE06460F4600
:10F7B0002846F0F75FFE94A3D3E90023F0F7C4FED8
:10F7C00002460B4630463946F0F708FDF1F794F94A
:10F7D000C8F83C008AF0010A0135022D6EDCF5EE16
:10F7E000C08AF1EE10FAB9D918EE100AF0F754FEFB
:10F7F00006460F462846F0F73DFE83A3D3E90023D3
:10F80000F0F7A2FE02460B4630463946F0F7E4FC1C
:10F81000F1F772F98346BAF1000FB7D0266A206873
:10F82000F0F73AFE804689463046F0F735FE064648
:10F830000F465846F0F730FE41EC190BB0EE490A7E
:10F84000F0EE690A05F02CF953EC102B30463946DE
:10F85000F0F77AFE02460B4640464946F0F7BCFCFC
:10F86000F1F74AF905F1030B04EB0B1BCBF8000091
:10F870006068F0F711FE80468946B0EE490AF0EE66
:10F88000690A05F061F953EC102B30463946F0F760
:10F890005BFE02460B4640464946F0F79DFCF1F7F9
:10F8A0002BF9CBF80400BAF1000F3FF471AFD4ED9F
:10F8B000027A73E700254FF0010A8EE7002518E071
:10F8C000EE1C04EB0616F0EE000A96ED000A05F0B9
:10F8D000E9F9B0EE408AF0EE000A96ED010A05F073
:10F8E000E1F938EE008A04AB03EB850303ED048AEB
:10F8F0000135022DE4DD00252E46012302E03546C8
:10F900001E460133022B1ADC04AA02EB830252EDDD
:10F91000047A04AA02EB860212ED047AF4EEC77AA6
:10F92000F1EE10FAEBD404AA02EB850212ED047A90
:10F93000F4EEC77AF1EE10FAE3D51D46E1E794ED57
:10F94000008AF0EE000AB0EE480A05F0ABF9B0EE1E
:10F95000409AD4ED018AF0EE000AB0EE680A05F094
:10F96000A1F939EE000A05F0F5F9B0EE409AF31C62
:10F9700004EB031393ED000A68EE009AD3ED01AA9D
:10F9800068EEAA7A79EEA79AF0EE000A05F08AF9F5
:10F99000B0EE40AAF0EE000AB0EE6A0A05F082F975
:10F9A0003AEE000A05F0D6F920EE090A89EE80AA9F
:10F9B000EB1C04EB031393ED000A28EE008AD3ED51
:10F9C000019A68EEA98A38EE288AF0EE000A05F05E
:10F9D00069F9F0EE408AF0EE000AB0EE690A05F02F
:10F9E00061F938EE800A05F0B5F920EE090AC8EE93
:10F9F000007AB4EEE7AAF1EE10FA40F32281354620
:10FA00001FE194ED099A39E00000004052C1004026
:10FA1000DB0F4940D4ED027A94ED0A7A77EE877ACB
:10FA200004EB0513C3ED0E7A83ED0F8A87F001070F
:10FA30000135032D42DCE068F0F72EFD8046894653
:10FA400007EE905AF8EEE77A1FED0F7A67EE877AA5
:10FA500017EE900AF0F720FD0022924BF0F774FDAC
:10FA600002460B4640464946F0F7B8FBF1F744F82A
:10FA700008EE100A002FC4D094ED089AD4ED008A45
:10FA8000B0EE480A04F080FF20EE090A78EEC08A42
:10FA9000EE1C04EB0616C6ED008AD4ED018AB0EE2A
:10FAA000480A04F02BFF20EE090A78EEC08AC6ED62
:10FAB000018A002FAED0D4ED027AB1E7002518E01C
:10FAC000EE1C04EB0616F0EE000A96ED000A05F0B7
:10FAD000E9F8B0EE408AF0EE000A96ED010A05F072
:10FAE000E1F838EE008A04AB03EB850303ED048AEA
:10FAF0000135032DE4DD9DED007ADDED017AB4EEF4
:10FB0000E77AF1EE10FA1ADC01210023DDED027A2A
:10FB100004AA02EB830212ED047AF4EEC77AF1EE46
:10FB200010FA0FD404AA02EB810212ED047AF4EE6B
:10FB3000C77AF1EE10FA20D41D460B4603E00021EF
:10FB40000123E3E70225DDED037A04AA02EB850237
:10FB500012ED047AF4EEC77AF1EE10FA10D404AA8A
:10FB600002EB830212ED047AF4EEC77AF1EE10FA9A
:10FB700000F192802E461D4603E01D460223E2E777
:10FB8000032694ED008AF0EE000AB0EE480A05F074
:10FB900089F8B0EE409AD4ED018AF0EE000AB0EE9A
:10FBA000680A05F07FF839EE000A05F0D3F8B0EEE8
:10FBB000409AF31C04EB031393ED000A68EE009ADD
:10FBC000D3ED01AA68EEAA7A79EEA79AF0EE000AC0
:10FBD00005F068F8B0EE40AAF0EE000AB0EE6A0A4E
:10FBE00005F060F83AEE000A05F0B4F820EE090AD4
:10FBF00089EE80AAEB1C04EB031393ED000A28EEB8
:10FC0000008AD3ED019A68EEA98A38EE288AF0EED0
:10FC1000000A05F047F8F0EE408AF0EE000AB0EE78
:10FC2000690A05F03FF838EE800A05F093F820EEF7
:10FC3000090AC8EE007AB4EEE7AAF1EE10FA00DD88
:10FC40003546EB1C04EB031393ED007AD4ED046A04
:10FC5000D4ED1F7A66EEA76A37EE267A84ED1C7A19
:10FC600093ED017AD4ED056A67EEA66A37EE267A3F
:10FC700084ED1D7A04EB051393ED0E7AD4ED066A3C
:10FC800067EEA67A77EE277AC4ED1E7A284605B08D
:10FC9000BDEC068BBDE8F08F2E46032571E70125EC
:10FCA000CFE700BF0000E03FF8B52DED048B10EE6C
:10FCB000107AF0EE609AB0EE419A0026DFED268AC7
:10FCC0003EE09FED268A29EE088A28EE288AF7EE84
:10FCD000007A38EE278A18EE100AF0F7DDFB41ECC7
:10FCE000100B04F09DFE51EC100B19A3D3E9002377
:10FCF000F0F754FD04460D463846F0F7CDFB0246BA
:10FD00000B4620462946F0F767FA04460D4668EE92
:10FD1000A97A17EE900AF0F7BFFB02460B46204681
:10FD20002946F0F759FAF0F7E7FE06EE900AC9EE19
:10FD3000087A77EEE97A86EEA77A78EEC78A0136F6
:10FD4000042EBEDDB0EE680ABDEC048BF8BD00BF2A
:10FD5000000000204A7BB33F0000000051DA9B3DC9
:10FD60002DE9D0432DED028B044600F14002022123
:10FD70001C3004F0A3FA94ED100AB5EEC00AF1EEBF
:10FD800010FAC0F2D98004F0E5FF84ED0F0AE06BB1
:10FD9000F0F782FB6AA3D3E90023F0F71DFAF0F72E
:10FDA000ABFE00EE900AE06394ED090A04F078FFE0
:10FDB00084ED0D0AD4ED070A94ED080A04F070FFF3
:10FDC00084ED060A94ED018A04F0DEFD28EE008A37
:10FDD000D4ED028A94ED060A04F090FD68EE808A64
:10FDE00038EE288A84ED048A94ED018AB1EE488ABF
:10FDF00094ED060A04F082FD28EE008AD4ED028A12
:10FE000094ED060A04F0C0FD68EE808A38EE288A78
:10FE100084ED058A94ED008A94ED0D0A04F0B4FD9A
:10FE200028EE008A94ED0D0A04F068FDB0EE481A41
:10FE3000D4ED040A94ED0F0AFFF736FF2046283070
:10FE400080ED000A04F12C02012104F037FAD4ED10
:10FE5000097A94ED037AD4ED0A6A27EE267A77EED2
:10FE6000877AC4ED147A636BA363002384F8483067
:10FE700094F84830092B51D894ED008A94ED0E0A7D
:10FE800004F03CFD28EE008AD4ED0A7A67EE887A09
:10FE900017EE900AF0F700FB06460F46E06AF0F70F
:10FEA000FBFA29A3D3E90023F0F74EFB02460B46E9
:10FEB00030463946F0F790F9F0F71EFE07EE900A4B
:10FEC000E06494ED148A38EE678A84ED118AA06BA1
:10FED000F0F7E2FA8046894618EE100AF0F7DCFAED
:10FEE00006460F461AA3D3E90023F0F72DFB02467E
:10FEF0000B4640464946F0F771F9F0F7FDFDA06367
:10FF000094F84830013384F8483013A3D3E9002330
:10FF100030463946F0F78AFD0028A9D0D4ED070A0B
:10FF200094ED080A04F0BCFE84ED150AA36BA365EA
:10FF3000BDEC028BBDE8D0830023E36327E700BF5D
:10FF40009A9999999999C93F9A9999999999134028
:10FF50009A9999999999B93F7B14AE47E17A743F80
:10FF600070B504460D46204B0B635378C3F3420330
:10FF700080F82C305378C3F3021380F82D30D2F878
:10FF800002300360D2F806304360D2F80A30836052
:10FF9000D2F812300361D2F816304361D2F81A3029
:10FFA0008361D2F80E30C360D2F81E30C361D2F83C
:10FFB00022300362D2F826304362D2F82A308362BC
:10FFC000FFF74AFB0646236FEB61636F2B62A36F5B
:10FFD0006B6223696B606369AB60A369EB60284661
:10FFE000FFF7BEFE304670BDCDCCCC3C10B504460C
:10FFF000102007F069FC0023036043608360C36046
:020000040801F1
:10000000A368C360238803B96423038063684360E3
:10001000638803B96423038123880381034A137827
:10002000591C1170024A42F8230010BD9C8F002019
:10003000A08F0020038803817047000010B50024C2
:1000400004E053680BB1D06898470134064B1B7825
:10005000A34208D9054B53F824201389002BF0D074
:10006000013B1381F1E710BD9C8F0020A08F002081
:1000700008B5002210210248F2F766FA08BD00BF59
:100080000000024008B5012210210248F2F75CFA94
:1000900008BD00BF0000024008B50022012102484F
:1000A000F2F752FA08BD00BF0004024008B5012271
:1000B00011460248F2F748FA08BD00BF00040240AA
:1000C00000B587B08DF80F004FF47A7300930123C9
:1000D0000DF117020DF10F0104480068F4F717FF46
:1000E0009DF8170007B05DF804FB00BFA09000204A
:1000F00038B50D46144640F08000FFF7E1FF06E0FA
:100100005520FFF7DDFF05F8010B013CE4B2002CA0
:10011000F6D138BD10B50C46FFF7D2FF2046FFF7E9
:10012000CFFF10BD10B50C4640F08000FFF7C8FFB0
:100130005520FFF7C5FF207010BD000030B52DED34
:10014000048B8BB00446CB4B93E803000890ADF8CA
:100150002410090C8DF8261000238DF82730FDF7A8
:100160005DF9C54B83ED000AFDF758F9C24BD3ED9D
:10017000007A30EE670AF2EE087AB4EEE70AF1EEA2
:1001800010FA0ADC9FEDBD0AFDF78CF9002323630A
:100190006362A362E3620025E1E0B94B6362B94B9D
:1001A000A362E362B84B2363B84BA361B84B0093DF
:1001B000B84BB94AB9490020F9F79CFB94ED0C7A89
:1001C000DFEDB76AC6EE877AC4ED087A0BB0BDECF6
:1001D000048B30BD9DF823301B021BB29DF82220FA
:1001E000134307EE903AAF4B93ED007AF8EEE77ABF
:1001F00067EE877AC4ED037AD4ED096A77EEA67AC2
:10020000C4ED097A9DF825301B021BB29DF824200D
:10021000134307EE903AF8EEE77A67EE877AC4ED7B
:10022000047AD4ED0A6A77EEA67AC4ED0A7A9DF8CC
:1002300027301B021BB29DF82620134307EE903A8D
:10024000F8EEE77A67EE877AC4ED057A94ED0B7ADB
:1002500077EE877AC4ED0B7AE5E00023022B0DD808
:100260009A1C04EB820251680AAA02EB830242F84C
:10027000141C42F8201C0133DBB2EFE7B0EE688AB1
:1002800078EEC86A884BC3ED006A00233BE0013377
:10029000DBB2022B24D819469A1C04EB8202D2ED61
:1002A000017A0AAA02EB830212ED057AF4EEC77A0C
:1002B000F1EE10FA04DD0AAA02EB830242ED057AA0
:1002C0000AAA02EB810212ED087AF4EEC77AF1EE87
:1002D00010FADCD50AAA02EB810141ED087AD6E7D3
:1002E000F0EE498ACCE70AAA02EB830252ED057AC6
:1002F00012ED087A77EEC77A6C4A02EB8302C2ED00
:10030000007A0133DBB2022BEDD9F6EE007AF4EE7F
:10031000E76AF1EE10FA00F39980644B93ED007AEE
:10032000DFED637AB4EEE77AF1EE10FA00F38E8037
:1003300093ED017AB4EEE77AF1EE10FA00F38680DD
:1003400093ED027AB4EEE77AF1EE10FA7EDC9FEDDF
:10035000590AFDF7A7F80135ADB2B0EE689A41F23F
:100360006F739D427CD8FFF783FE9220FFF7A8FEB3
:10037000062208A91220FFF7BBFEFFF783FE9DF8B7
:1003800021301B021BB29DF82020134307EE903A48
:10039000F8EEE77A484A92ED007A67EE877AC4ED84
:1003A000007A9DF823301B021BB29DF822100B43EC
:1003B00007EE103AD2ED006AB8EEC77A27EE267A39
:1003C00084ED017A9DF825301B021BB29DF8242094
:1003D000134300EE103AB8EEC00A20EE260A84ED70
:1003E000020A67EEA77A27EE077A77EE877A20EE81
:1003F000000A37EE800A04F0ADFCF0EE408AD4ED3E
:100400000C7A77EE807AC4ED0C7AFFF745FE08226D
:1004100008A90020FFF76CFEFFF748FE9DF820308A
:100420000F2B3FF4D7AE002D3FF417AFB4EEE89A90
:10043000F1EE10FA01D5B0EE689AB4EEE88AF1EE6A
:1004400010FA01DDB0EE688A002322E7104B00931A
:100450001A4B1B4A1B490020F9F74CFAB0EE689A78
:10046000D4ED0C6A9FED187AC6EE877AC4ED0C7A4B
:10047000002339E0B4C40108B09000200AD7A33BA0
:10048000AC38223BB016CE393F161B41000020424B
:1004900064C50108C4C50108C8C5010878CB0108B6
:1004A000C3F51C4194030020EC900020F090002044
:1004B0009A99193E6F12033A9803002048C901081F
:1004C0004CC90108B0CB01080080BB4503F108020C
:1004D00004EB8202D2ED016A1FED057AC6EE877A3F
:1004E000C2ED017A0133DBB2022BEFD9FFF7C0FD79
:1004F000A220FFF7E5FD022208A92220FFF7F8FD60
:10050000FFF7C0FD9DF820209DF821305B0943EAEC
:10051000C203B3F5806F01DBA3F5006307EE903AE9
:10052000F8EEE77AB4EE007A67EE877AB3EE077AF0
:1005300077EE877AC4ED067A2D4A1388013313804B
:100540002C4B93ED007AF6EE007AB4EEE77AF1EEFA
:1005500010FA3FF709AED4ED0C7A9FED277A77EECB
:10056000C77AF0EEE77AB6EE007AF4EEC77AF1EEEB
:1005700010FA3FF7F9AD214B93ED007ADFED207AC9
:10058000B4EEE77AF1EE10FA3FF7EEAD93ED017AB3
:10059000B4EEE77AF1EE10FA3FF7E6AD93ED027AAA
:1005A000B4EEE77AF1EE10FA3FF7DEADD4ED097A5A
:1005B000F0EEE77A9FED137AF4EEC77AF1EE10FAD7
:1005C0003FF7D2ADD4ED0A7AF0EEE77AF4EEC77ACF
:1005D000F1EE10FA3FF7C8ADD4ED0B7AF0EEE77A02
:1005E000F4EEC77AF1EE10FA3FF7BEADE6E500BFD4
:1005F000E8900020EC900020CDCC1C41F090002031
:100600009A99193E0AD7233C70B52DED028B82B022
:10061000FFF72EFD8020FFF753FD5520FFF750FD1B
:100620005520FFF74DFD514C2070FFF72BFD9FED3E
:10063000508AB0EE480AFCF735FFFFF719FD80201D
:10064000FFF73EFD5520FFF73BFD5520FFF738FD36
:100650002070FFF717FDB0EE480AFCF723FFFFF705
:1006600007FDB6217E20FFF755FDFFF70BFD9FED3F
:10067000410AFCF717FFFFF7FBFC8020FFF720FD86
:100680005520FFF71DFD5520FFF71AFD2070FFF7DD
:10069000F9FCB0EE480AFCF705FFFFF7E9FC802003
:1006A000FFF70EFD5520FFF70BFD5520FFF708FD66
:1006B0002070FFF7E7FCB0EE480AFCF7F3FE237862
:1006C0001E2B03D12C4B00221A7011E02B4B0093F0
:1006D0002B4B2C4A2C490020F9F70CF9FF2041E064
:1006E000A2782A49087802430A700133224A13701B
:1006F000214B1B78052B34D8FFF7BAFC1E4D2B7805
:10070000234C03EB4303E2185178E05CFFF702FD52
:10071000FFF7B8FC9FED168AB0EE480AFCF7C2FE60
:10072000FFF7A6FC2B7803EB4303E05C40F080006E
:10073000FFF7C6FC5520FFF7C3FC5520FFF7C0FCB0
:100740000A4E3070FFF79EFCB0EE480AFCF7AAFE96
:100750002B7803EB43021444617832789142BFD185
:10076000C3E7002002B0BDEC028B70BDFE900020FC
:100770006F12833A0AD7A33DFD90002064C501089B
:10078000C4C50108C8C50108E0CB0108FC900020E1
:100790005CCC010870B52DED028B82B0FFF77CFCBC
:1007A000494C21460020FFF7BDFCFFF77FFC9FED81
:1007B000478AB0EE480AFCF775FEFFF76DFC21464C
:1007C0000020FFF7AFFCFFF771FCB0EE480AFCF722
:1007D00069FEFFF761FCB6211420FFF79BFCFFF7D1
:1007E00065FC9FED3B0AFCF75DFEFFF755FC2146DB
:1007F0000020FFF797FCFFF759FCB0EE480AFCF722
:1008000051FEFFF749FC21460020FFF78BFCFFF764
:100810004DFCB0EE480AFCF745FE23780F2B03D1C0
:100820002C4B00221A7019E02B4B00932B4B2C4AB7
:100830002C490020F9F75EF8FF2041E0013BDBB2D4
:100840002B7003EB4303284A13449B78274A117803
:100850000B4313701F4A1378013313701D4B1B7821
:10086000052B2CD8FFF718FC1A4D2B78204C03EBE6
:100870004303E2185178E05CFFF74CFCFFF716FCED
:100880009FED128AB0EE480AFCF70CFEFFF704FC5D
:100890000D4E2B7803EB43033146E05CFFF742FC3F
:1008A000FFF704FCB0EE480AFCF7FCFD2B7803EBE5
:1008B00043021444617832789142BFD1CAE70020E4
:1008C00002B0BDEC028B70BDFE9000206F12833A27
:1008D0000AD7A33DFD90002064C50108C4C50108E6
:1008E000C8C5010814CC01085CCC0108FC900020AC
:1008F00048CC010838B50D46114B1860114C002347
:100900002370FFF781FE237818432070FFF742FF22
:1009100023781843207075B90B4B0C4A5A620C4A65
:100920009A62DA620B4A1A630B4A1A620B4A9A619C
:10093000044B187838BD0448FFF700FCF8E700BF07
:10094000A0900020FC900020B4900020AC38223B06
:10095000B016CE393F161B41C48B813F00002042A8
:1009600038B50546FFF784FB9220FFF7A9FB734CCF
:10097000062221461220FFF7BBFBFFF783FB6378BB
:100980001B021BB2227813436D4A138007EE903A84
:10099000F8EEE77A6B4991ED007A67EE877A95ED8C
:1009A000087A67EE877AC5ED007AE3781B021BB2FE
:1009B000A07803431380D1ED006A07EE903AF8EE79
:1009C000E77A67EEA67A67EE277AC5ED017A637952
:1009D0001B021BB221790B43138007EE903AF8EE0D
:1009E000E77A67EEA67A27EE277A85ED027AFFF797
:1009F00053FB082221460020FFF77AFBFFF756FB46
:100A000023780F2B2BD0FFF733FBA220FFF758FBE7
:100A10004A4C022221462220FFF76AFBFFF732FBF5
:100A2000227863785B0943EAC203454A1380B3F531
:100A3000806F02DBA3F500631380414BB3F90030F4
:100A400007EE903AF8EEE77AB4EE007A67EE877A2E
:100A5000B3EE077A77EE877AC5ED077A38BD3A4B61
:100A60001B78002B3AD0E3781B021BB2A1780B4312
:100A700033490B80354890ED007A07EE903AF8EE56
:100A8000E77A67EE877AD5ED096A77EEE67AC5ED03
:100A9000037A63791B021BB2207903430B8007EEB4
:100AA000903AF8EEE77A67EE877AD5ED0A6A77EE44
:100AB000E67AC5ED047AE3791B021BB2A2791343EF
:100AC0000B8007EE903AF8EEE77A67EE877A95EDBD
:100AD0000B7A77EEC77AC5ED057A94E7174AD37893
:100AE0001B021BB291780B4315490B80174890ED00
:100AF000007A07EE903AF8EEE77A67EE877AC5ED6E
:100B0000037A53791B021BB2107903430B8007EE63
:100B1000903AF8EEE77A67EE877AC5ED047AD379F2
:100B20001B021BB2927913430B8007EE903AF8EE4A
:100B3000E77A67EE877AC5ED057A64E7A89000202A
:100B4000A49000209803002090030020940300202C
:100B5000014B1B68586370470C69002070B52DED80
:100B6000028B8AB006460024079408940994002357
:100B7000049305934FF07E530693019402940394DB
:100B800021E0354D2846FFF7EBFE95ED027ADDEDCD
:100B9000077A77EEC77ACDED077A95ED017ADDED2C
:100BA000087A77EE877ACDED087A95ED007ADDED5B
:100BB000097A77EE877ACDED097A9FED280AFCF75E
:100BC00071FC0134E4B2632CDBD900230CE00AAAE7
:100BD00002EB830252ED036A9FED217AC6EE877A1B
:100BE00042ED037A0133DBB2022BF0D907A8FEF7FE
:100BF000ADFC04A907A8FEF700FD03F0F9FFB0EE75
:100C0000408A01AA04A907A8FEF7C6FC01A8FEF7BE
:100C10009DFCF6EE007A28EE278AB0EE480A04F032
:100C2000B7F886ED000A002410E00AAB03EB84035A
:100C300053ED098AB0EE480A04F0F6F8013406EBE9
:100C4000840368EE808AC3ED008AE4B2012CECD9FB
:100C50000AB0BDEC028B70BDB49000206F12833AD5
:100C60000000C84270B52DED068B86B004460D46D7
:100C7000164690ED040A9F4BD3ED007A70EE677A2A
:100C8000F0EEE77A9FED9C7AF4EEC77AF1EE10FA77
:100C900022DCD0ED057A994B93ED007A77EEC77A96
:100CA000F0EEE77A9FED947AF4EEC77AF1EE10FA5F
:100CB00012DCD0ED067A924B93ED007A77EEC77A8C
:100CC000F0EEE77A9FED8C7AF4EEC77AF1EE10FA47
:100CD00002DC0378002B6ED09FED8AAA80EE0A0A10
:100CE00003F052FEB0EE409A94ED050A80EE0A0A37
:100CF00003F04AFEF0EE408A94ED060A80EE0A0AFE
:100D000003F042FEF0EE40AA94ED040A80EE0A0AD7
:100D100003F0F4FDB0EE408A94ED050A80EE0A0A75
:100D200003F0ECFDF0EE409A94ED060A80EE0A0A1C
:100D300003F0E4FD69EE2A6A28EE297A27EE007AAC
:100D400036EE877A704B83ED007A28EE887A6F4B07
:100D500083ED007A29EE007A2AEE886A66EE295A37
:100D600037EE657A6A4B83ED007A29EE297A27EE11
:100D7000007A37EE467A674B83ED007A29EE289A9F
:100D8000654B83ED009A28EE408A66EEA96A38EE3C
:100D9000668A624B83ED008A68EEC07A604BC3EDD1
:100DA000007A604BC3ED009A68EEAA8A5E4BC3EDF1
:100DB000008A00232370002310E005EB8302D2EDAC
:100DC000007A04EB830292ED017A67EE877A06AA35
:100DD00002EB830242ED037A0133DBB2022BECD942
:100DE000DDED037A484B93ED006A27EE867A9DEDA0
:100DF000045A464BD3ED002A65EE226A37EE267A76
:100E0000DDED055A424B93ED003A65EE836A37EE0D
:100E1000267A85ED007A3F4BD3ED006A27EEA67A5D
:100E20003D4BD3ED003A65EE234A37EE247A3B4B37
:100E300093ED004A65EE844A37EE247A85ED017A17
:100E4000374B93ED007A67EE877A364BD3ED004A45
:100E500025EE245A77EE857A334B93ED005A65EEF2
:100E6000855A77EEA57AC5ED027A002309E006EBF4
:100E70008302116806AA02EB830242F8181C0133B0
:100E8000DBB2022BF3D99DED002A26EE026ADDEDDE
:100E9000015A62EEA52A36EE226ADDED027A23EED1
:100EA000273A36EE036A86ED006A66EE826A63EEE2
:100EB000A53A76EEA36A24EE274A76EE846AC6ED5A
:100EC000016A27EE027A64EEA54A37EE247A25EE0F
:100ED000275A37EE057A86ED027A2269054B1A60A9
:100EE0006269064B1A60A269054B1A6006B0BDEC38
:100EF000068B70BD2C9100206F12833A2891002040
:100F000024910020E12E6542209100201C910020B8
:100F10001891002014910020109100200C910020C5
:100F200008910020049100200091002010B50F4C82
:100F3000DFED0F0A0F4B93ED070A2046FDF70FFD7B
:100F400094ED140AFEF7E2FA00EE100A9FED0A1A79
:100F5000DFED0A0AB8EEC00AFEF796FABCEEC00A48
:100F600010EE103A98B2FFF7F3FD10BD409100204B
:100F700000002042B49000200000804F00000000DC
:100F80002E4B93F880300BB12D48704730B52DEDC6
:100F9000028B91B0294B012283F88020002129483F
:100FA000F4F78CFD01212848FFF7A4FC0028F9D1B3
:100FB000264BB7EE008A83ED018A83ED028A83ED2A
:100FC000038ADFED238AC3ED048AC3ED058AC3EDEE
:100FD000068A01251D7000240C940D940E940F9424
:100FE0000CA8FFF7BBFDB0EE682AF0EE481A9FEDA3
:100FF000191ADFED190AB2EE040A0CA8FDF7D8F8A9
:101000002C22214601A807F015F8144B0193144B2C
:101010000293144B04938DF81850134B079301A9B6
:101020001248FDF777FC054B114A9A621148FCF70C
:1010300067F9034811B0BDEC028B30BDD49100209C
:10104000249200200C69002068680020B8910020DC
:1010500000000000002474496F12833A00007A44B3
:101060000000A0410000FA44000096434091002097
:1010700096430B3C3C91002092ED026A66EE067AA4
:10108000F6EE006A76EEE77A92ED037A67EE075A9B
:1010900077EEE57AD0ED005A67EEA57AD2ED014AF7
:1010A00066EE245A92ED005A27EE054A75EEC45AB0
:1010B00090ED014A65EE845A77EEA57A27EE247A00
:1010C00026EE056A37EE067A90ED026A27EE067A7A
:1010D00077EE877A77EEA77AC1ED007AD2ED015AE2
:1010E00092ED027A65EE877AD2ED004A92ED035ACC
:1010F00024EE856A77EE867A90ED006A67EE867A4E
:1011000025EEA56A36EEC66A25EE054A36EE446A35
:1011100090ED014A26EE046A77EE867A27EE057A8C
:1011200065EEA45A37EE657A90ED026A27EE067AEC
:1011300077EE877A77EEA77AC1ED017AD2ED015A80
:1011400092ED037A65EE877A92ED005A92ED026A8B
:1011500065EE064A77EEE47AD0ED004A67EEA47AAF
:1011600027EE067A25EE855A37EE057A90ED015A7C
:1011700027EE057A77EE877A65EEA55A76EEE56A70
:1011800026EE066A76EEC66A90ED027A66EE876A09
:1011900077EEA67A77EEA77AC1ED027A704792EDE4
:1011A000026A66EE067AF6EE006A76EEE77A92ED6D
:1011B000037A67EE075A77EEE57AD0ED005A67EECC
:1011C000A57AD2ED014A66EE245A92ED005A27EE36
:1011D000054A75EE845A90ED014A65EE845A77EE21
:1011E000A57A27EE247A26EE056A37EE467A90ED48
:1011F000026A27EE067A77EE877A77EEA77AC1ED54
:10120000007AD2ED015A92ED027A65EE877AD2ED3C
:10121000004A92ED035A24EE856A77EEC67A90ED85
:10122000006A67EE867A25EEA56A36EEC66A25EE76
:10123000054A36EE446A90ED014A26EE046A77EEDE
:10124000867A27EE057A65EEA45A37EE257A90ED78
:10125000026A27EE067A77EE877A77EEA77AC1EDF3
:10126000017AD2ED015A92ED037A65EE877A92ED1A
:10127000005A92ED026A65EE064A77EEA47AD0ED46
:10128000004A67EEA47A27EE067A25EE855A37EEF5
:10129000457A90ED015A27EE057A77EE877A65EE6A
:1012A000A55A76EEE56A26EE066A76EEC66A90EDF7
:1012B000027A66EE876A77EEA67A77EEA77AC1EDB4
:1012C000027A704770B586B0002303930493564B9F
:1012D00005935648FCF714F8554E86ED000A554B19
:1012E000D3ED007A77EE807AC3ED007A524D28462E
:1012F000FFF736FBD5ED027AF1EE677A4F4CC4ED7D
:10130000177A6B6823662B686366D5ED057AF1EE74
:10131000677AC4ED147A2B696365EB68A36504F101
:101320005C0204F150014648FFF79CFC96ED003A40
:10133000D4ED192A94ED182AD4ED171A94ED161A43
:10134000D4ED150A94ED140AFCF7A4FF3D4B0FCB26
:1013500084E80F00224604F12C013B48FFF78CFE85
:10136000224604F138013948FFF786FE224604F18F
:1013700044013748FFF780FE2246694603A8FFF77D
:101380000EFF002327E02D4A03F1160102EB810135
:1013900091ED017A06A901EB830151ED067A37EE52
:1013A000677A2349D1ED007A27EE277AD2ED0A6ACF
:1013B00077EEA67A87EE276A191D02EB810292ED7D
:1013C000007A66EE876A86EEA77A76EE077AC2ED35
:1013D000007A0133DBB2022BD5D9184C224604F136
:1013E0001C0104F11000FFF747FE1A4B93ED6A0A47
:1013F00084ED1C0AD3ED690AC4ED1B0AD3F8A021C1
:10140000A266D3F8AC31636700F06CF8124B1B682E
:1014100013F0010F05D0104A13680133136006B0B2
:1014200070BDFFF783FDF6E7C3F51C413C9100203A
:101430003891002034910020B4900020D4910020F5
:10144000B8910020F88E002088CC01087CCC0108DF
:1014500070CC0108A88D00203091002000B583B029
:10146000054B0093054B064A06490020F8F742FA5F
:1014700003B05DF804FB00BF64C5010848C901085A
:101480004CC9010894CC010838B50E4B1868037894
:10149000A52B00D038BD3021FDF71CFB0028F9D06A
:1014A000084B1C68084D04F1300EAC46206861689A
:1014B000A268E368ACE80F00103465467445F4D1C7
:1014C000E8E700BF7092002090920020044B5A7809
:1014D00060F300025A70D2B26FF347025A7070473D
:1014E00078920020044A10EE103AC2F8063010EE4E
:1014F000903AC2F80230704778920020064B10EE06
:10150000102AC3F80A2010EE902AC3F80E2011EE1C
:10151000102AC3F8122070477892002010B586B0C8
:1015200004AB0024049405940B4A059293E803004D
:10153000FCF7FEF9094B186001940294039405230B
:10154000ADF80430064B029301A8FEF74FFD054BA2
:101550001860054806B010BD89140108709200207B
:101560005D140108749200209092002038B50C4C54
:101570005A23237016212046FDF792FAE082094D86
:10158000AE46A446BCE80F00AEE80F009CE803009E
:101590008EE8030018212846FCF7E8F938BD00BFA3
:1015A000789200205892002010B582B00446212184
:1015B00006F057FD1F2801D802B010BD044B01935F
:1015C0000094044B044A05490020F8F793F9FEE71C
:1015D00064C50108C4C50108C8C50108D0CC01080C
:1015E000884200D1704700B585B0054B0293019148
:1015F0000090044B044A05490020F8F77BF9FEE708
:1016000064C50108C4C50108C8C50108F4CC0108B7
:10161000F8B505460F46FFF7C7FF144C2646A46AE7
:1016200074B129462046EFF72FFC0028F6D194F834
:1016300021103846FFF7D4FF012384F82C3012E044
:10164000302006F041F9B0623022002106F0F2FCB1
:10165000B36A83F821702946B06A06F0E3FD0123DE
:1016600086F82C30B46A2046F8BD00BF9C030020E9
:10167000F8B50E46FFF7CCFF07460C2006F024F91C
:1016800005460024046044608460067144B17B6AAE
:101690006BB11A469B68002BFBD195602846F8BDBC
:1016A000304606F011F945F824000134EEE77D627A
:1016B000F4E710B50446C07900B910BD0B46617956
:1016C000227954F82110184606F0B4FD63790133ED
:1016D000637100236371E379013BE3710120ECE75F
:1016E00070B505460E46426A0F4B1A600FE0A379AB
:1016F00095F82120314654F8230006F09BFD002385
:10170000A371E3790133E371A268074B1A60064BBA
:101710001C683CB1E379012BE9D100226271013BE5
:10172000E371E4E7012070BDC092002000B585B0F0
:10173000D0F8A83119680A4A91420ED0022209490C
:101740000291DB6901930092074B084A0849002087
:10175000F8F7D0F805B05DF804FB0122EFE700BF11
:101760004C62002064C5010848C901084CC9010841
:1017700018CD010830B585B00C4609794A1ED2B2A1
:1017800090F8AE31012B57D05DB2002D00F0BC8037
:10179000023BDBB2012B00F2B780032A14D8216888
:1017A0005F4B99420DD01346042102F20122A26040
:1017B0005C4A0125555480F8AD3180F8AC11002306
:1017C0000FE013460121F0E74B1FDBB225685449B7
:1017D0008D4201D00321E8E70021E6E701251FE063
:1017E0000133514A12789A4240F297804F4A52F898
:1017F0002320D2F8A821106821688842F0D1516BCB
:10180000A2689142ECD14A4B00934A4B4A4A4B4959
:101810000020F8F76FF82268414B9A42DED002258B
:10182000434B02930195A3680093424B424A4449BB
:101830000020F8F75FF8F3E790F8AF31012B13D0F1
:10184000032A2AD82168364B994223D01346032114
:1018500002F20522A260334A0125555480F8AD31C9
:1018600080F8AC11002325E0032A09D821682C4B0D
:10187000994202D013460821EAE713460621E7E71A
:101880004B1FDBB2256826498D4201D00921DFE7D5
:101890000721DDE713460021DAE74B1FDBB225689D
:1018A0001F498D4201D00521D2E70221D0E7012551
:1018B0001EE001331C4A12789A422ED91B4A52F874
:1018C0002320D2F8A821106821688842F1D1516BF9
:1018D000A2689142EDD1164B0093164B164A174958
:1018E0000020F8F707F822680D4B9A42DFD0022556
:1018F0000F4B02930195A36800930E4B0E4A1049BB
:101900000020F7F7F7FFF3E7094B0093094B0A4A6A
:101910000C490020F7F7EEFFF6E705B030BD00BF39
:101920004C620020C4920020E8920020D092002057
:1019300064C50108C4C50108C8C5010854CD010823
:10194000C4CD0108F0CD010838B50546D0F83D40BA
:10195000D4F8B401FEF76EFB04F5DC70FBF7D0FCA5
:1019600084ED6F0A6188218095F82C3095F82D2040
:1019700042EA0322628007EE902AF8EE676ADFED02
:101980002F7A66EEA76AC4ED016AD4ED027A9FED64
:101990002C7A27EE877A95F82E0095F82F3043EAB7
:1019A00000231BB207EE903AF8EEE77A9FED256A26
:1019B00067EE867A77EE277AC4ED027AB4F90C30B6
:1019C00007EE903AF8EEE77A9FED1F7A67EE877A96
:1019D00095F8300095F8313043EA00231BB207EE4A
:1019E000103AB8EEC77A9FED196A27EE067A77EEBD
:1019F000877AFDEEE77A17EE903AA38195F83230B8
:101A0000A373521AB2F5805F10DD6369013B636115
:101A100063694FF4B47202FB03F307EE903AF8EEF9
:101A2000E77A77EEA67AC4ED047A38BD12F5805FC6
:101A3000EEDA636901336361EAE700BFACFF333D6F
:101A40009899193E3433A340D0CCCC3D6666663FAE
:101A5000042903D0022903D14277704702777047E7
:101A600000B583B0054B0093054B064A064900209C
:101A7000F7F740FF03B05DF804FB00BF64C5010841
:101A8000C4C50108C8C5010844CE0108002380F878
:101A9000B0317047012380F8B031704770B584B021
:101AA00005464FF4E07005F00FFF04464FF4E07276
:101AB000002106F0BFFA95F89C3084F8AE3104F1AD
:101AC000180305F1940292E8030083E8030095F8F7
:101AD000B43084F8AF3105F1100104F13000FCF7A7
:101AE00019FF05F13C0104F1A800FCF713FF05F113
:101AF000680104F59070FCF70DFF2B6823626B689A
:101B00006362EB68E362AB68A36205F1A00631464D
:101B10002046FFF72FFE134BC5F8AC30C5F8B04098
:101B20003046FBF795FAC4F8A8010023019302930D
:101B300003936423ADF804300B4B0293039401A884
:101B4000FEF754FAC4F8B4012046FFF7A3FF074A92
:101B50001378591C1170064A42F82340204604B0FD
:101B600070BD00BF491901082D170108E892002037
:101B7000D09200200176704780ED660A7047000021
:101B800070B52DED028B002553E0B1EE400A5DE00B
:101B9000237F012B0AD0D4ED047AF0EE400AB0EE98
:101BA000670A04F59070FCF7DAFE56E0236AD3ED7D
:101BB000007AF2E7636AD3ED007AF0EE400AB0EE05
:101BC000670A04F1A800FCF7CAFEA37F13F0010F17
:101BD00004D0E36AD3ED007A30EE270AE37E012BCE
:101BE0005AD0E37F012B5AD09FED711ADFED710AB5
:101BF000FDF74AFCFDEEC07A17EE901A94F8AC217E
:101C000094F8ADC14FEA4C00C1F3072602EB821EE7
